:100000005555AAAA182000000000000000000000BA
:10001000B783000000000000000000004161B35FF2
:100020000002100021080000A5020000BB02000031
:10003000D1020000E7020000FD0200000000000005
:100040000000000000000000000000004528000043
:100050004928000000000000130300004B280000A6
:100060004D2800006D25000085280000A525000012
:1000700067280000692800006D2800007128000032
:100080007528000077280000792800007B280000F0
:100090007D2800008728000000000000000000000C
:1000A000892800008B2800000000000000000000EC
:1000B000000000008D2800008F280000B9250000F6
:1000C000912800009F28000025030000B9280000A7
:1000D000BB2800000000000000000000000000003D
:1000E0001820000000F002F800F068F80AA090E87C
:1000F000000C82448344AAF10107DA4501D100F0E3
:100100005DF8AFF2090EBAE80F0013F0010F18BF47
:10011000FB1A43F001031847D08501001086010047
:100120000A444FF0000C10F8013B13F0070408BF1D
:1001300010F8014B1D1108BF10F8015B641E05D0BB
:1001400010F8016B641E01F8016BF9D113F0080F70
:100150001EBF10F8014BAD1C0C1B09D16D1E58BF02
:1001600001F801CBFAD505E014F8016B01F8016B39
:100170006D1EF9D59142D6D370470000103A24BFC6
:1001800078C878C1FAD8520724BF30C830C144BFFC
:1001900004680C607047000000230024002500263E
:1001A000103A28BF78C1FBD8520728BF30C148BFDA
:1001B0000B6070471FB51FBD10B510BDDFF80CD028
:1001C000FFF7F8FF02F0ABFC17F0D0FF00021000C1
:1001D00003B4FFF7F1FF03BC17F0D0FF0A484FF05C
:1001E000FF0101704FF0000080F311884FF0000014
:1001F00080F3098805484FF00201017062B6044897
:100200004FF080510160704722ED00E000021000C5
:1002100004ED00E002484FF080510160704700009B
:1002200004ED00E04FF0200080F31188EFF3098027
:1002300098B11248006812490968884217D0EFF354
:1002400009800E49096820E9F00F886000B50B4865
:10025000006800F0F2F85DF804EB084808490A6805
:10026000026000688168B1E8F00F81F309884EF000
:10027000040E4FF0000080F3118870470402100054
:1002800008021000EFF311804FF0200181F3118874
:10029000704700004FF0000080F3118870470000A5
:1002A00062B6704772B6704740BA7047C0BA7047BE
:1002B000401E0028FCDC704700BE704740BA704703
:1002C000C0BA70471EF0040F0CBFEFF30880EFF3C5
:1002D00009804FF0010102F0E6B91EF0040F0CBFD7
:1002E000EFF30880EFF309804FF0020102F0DBB971
:1002F0001EF0040F0CBFEFF30880EFF309804FF0FE
:10030000030102F0D0B91EF0040F0CBFEFF3088018
:10031000EFF309804FF0040102F0C5B91EF0040F9D
:100320000CBFEFF30880EFF309804FF0050102F0F6
:10033000BAB94FF0000000B503F0CBFD5DF804EB57
:10034000FFF770BF1EF0040F0CBFEFF30880EFF350
:1003500009804FF0000102F0A6B90000194910B55C
:1003600001200870184900200860184908601849E1
:1003700008601849086000F0B9F900F04BF900F086
:1003800063F8002010BD10B5114800F02AF90F499C
:1003900008600D490968884207D00A480078022899
:1003A00003D1BDE81040FFF735BF10BD10B5FFF712
:1003B000EAFF044902200870FFF710FF4FF0FF30FA
:1003C00010BD00000002100004021000080210001E
:1003D0000C0210001002100070B50D460446C169F1
:1003E0008068CC2217F0F7FDE169A0680844403826
:1003F0004FF08071C163216A816300214163016311
:10040000C1628162C0E908514FF00B31C1614FF008
:100410000A3181614FF0093141614FF008310161CA
:100420004FF00731C1604FF0063181604FF0053168
:1004300041604FF00431016070BD82698168914272
:1004400001D802F018BC704710B54FF4B4714F4892
:1004500017F0EBFD002010BD70B5054600EBC5019F
:100460004A4800EB8104FFF70DFF0646207828B1CB
:100470003046FFF70FFF6FF0010070BD03202070C2
:1004800000206560206204F11C0000F083F8304613
:10049000FFF700FF002070BD2DE9F0410F463B49FA
:1004A000002500EBC00001EB80042E46FFF7EAFEBA
:1004B0008046206A3843206204F11C00074600F0A1
:1004C00090F80CE0216A026C114203D000F066F94A
:1004D000012600E06D1C2946384600F078F8002817
:1004E000F0D1012E01D1FFF74EFF4046FFF7D2FEBB
:1004F0000020BDE8F08170B50D46244900EBC00036
:1005000001EB8004FFF7BEFE216AA9432162FFF7D9
:10051000C1FE002070BD70B50C461C4900EBC00048
:1005200001EB800500202060FFF7ACFE296A216006
:10053000FFF7B0FE002070BD2DE9F0410D461349D4
:1005400000EBC0001E46904601EB8004FFF79AFEC8
:1005500007460F4800680564216A294203D104F167
:100560001C0100F02DF93846FFF794FEFFF78AFED4
:10057000216A29403160B8F1010F02D1216AA943F3
:100580002162FFF787FE0020B3E70000E0041000BF
:1005900004021000002101600846704730B50A6867
:1005A00012B10B46C46B09E000220860C0E90321C8
:1005B0000BE000BF02F10C03D26812B1D56BA5426B
:1005C000F8DC1A68C0E903211860002030BD00681B
:1005D000002201E0C068521C8A4201D00028F9D1F3
:1005E00070470068704702690AB1116831B96FF04D
:1005F0000400704701F10C02C96839B18142F9D198
:10060000C968116000210161084670476FF003005E
:100610007047000010B54FF4C871324817F005FD5F
:10062000002010BD2DE9F041884605462D4900EB1C
:100630008500174601EBC004FFF724FE064620782C
:1006400030B13046FFF726FE6FF00100BDE8F081C3
:1006500002202070E7611422414604F10800656021
:1006600017F042FC0020206204F12400FFF792FF03
:100670003046FFF70FFE0020E8E770B5194900EBA0
:10068000800001EBC004FFF7FDFD0546D4E907013A
:10069000814205DB144804F12401006800F090F861
:1006A000206A401C20622846FFF7F4FD002070BD40
:1006B00070B50C4900EB800001EBC004FFF7E2FDD0
:1006C0000546206A08B1401E206204F12400FFF7AD
:1006D00088FF10B1606A00F011F82846FFF7DAFDD4
:1006E000002070BD480610000402100010B54FF441
:1006F0002A71404817F099FC002010BD10B504463F
:1007000090F8380002280BD02046FFF76CFF02203B
:1007100084F8380038492046FFF740FFFFF733FEE2
:10072000002010BD2DE9F05F8B460646314900EBF5
:1007300006109046DDE90AA911F820201D461AB1DD
:100740006FF00100BDE8F09F01EB8004FFF79AFD18
:10075000074601202070C4E90165C4E90585C4E9A4
:1007600007A91422594604F1240017F0BDFB00200C
:1007700084F8370084F838006169E0602061C4E9DA
:100780000F1020460C99FFF727FEA0602046FFF7C8
:10079000B5FF3846FFF77EFD0020D3E710B50446CD
:1007A00090F83800022809D02046FFF71CFF0220ED
:1007B00084F8380010492046FFF7F0FE002010BDF5
:1007C00070B5044690F838000D4602280BD120463B
:1007D000FFF709FF032084F8380029462046FFF779
:1007E000DDFEFFF7D0FD002070BD044800684068C2
:1007F00070470000D80710000C021000040210001F
:10080000F0B58446002004460C4F14E05CF82460E8
:100810000323DD0046FA05F280EA0260082500287D
:1008200002DA87EA400000E040006D1E002DF6DC91
:100830005B1EEED5641C8C42E8DBF0BD1B00008023
:100840001248804712480047FEE7FEE7FEE7FEE752
:10085000FEE7FEE7FEE7FEE7FEE7FEE7FEE7FEE770
:10086000FEE7FEE7FEE7FEE7FEE7FEE7FEE7FEE760
:10087000FEE7FEE7FEE7FEE7FEE7FEE7FEE7FEE750
:10088000FEE7FEE7FEE7FEE7FEE70000C90800001E
:10089000C5000000244800684FF00051002891F87E
:1008A000210000F01C000DD0042805D0082805D038
:1008B0000C2805D096200CE011200AE0252008E045
:1008C0004B2006E0042809D0082809D00C2809D0BC
:1008D0007020401E01F82C0F087070470C20F8E7BC
:1008E0001B20F6E73720F4E770471049D320087043
:1008F0000D4901200860CDE70C490B2008700A491A
:1009000001200860C6E7084801684FF0005090F8E1
:10091000210011B1F32804D001E0932801D0002078
:10092000704701207047000034040022210000209D
:1009300010B5042000F0D4F9052000F0D1F906200C
:1009400000F0CEF9072000F0CBF9082000F0C8F93C
:10095000182000F0C5F9192000F0C2F91A2000F0A3
:10096000BFF9F14A00201060EF4B40331860EE49A8
:1009700018390860EC4908310860EC49C871EA4C44
:10098000143C2060E84C0C3420600872E64C103CAB
:100990002060E54C103420604872E34C0C3C206031
:1009A000E14C143420608872DF4C083C2060DE4C3F
:1009B00018342060C872DC4C283420608873241DF1
:1009C0002060C873241D2060087401201060186026
:1009D00008700621042000F09BF90621052000F094
:1009E00097F90621084600F093F90621072000F048
:1009F0008FF90621082000F08BF90621182000F05D
:100A000087F90621192000F083F904211A2000F04B
:100A10007FF9042000F070F9052000F06DF9062040
:100A200000F06AF9072000F067F9082000F064F987
:100A3000182000F061F9192000F05EF91A2000F08A
:100A40005BF9042000F040F9052000F03DF9062094
:100A500000F03AF9072000F037F9082000F034F9E7
:100A6000182000F031F9BDE810401A2000F02CB930
:100A700000EB8000AC494000002218390A60AB4A04
:100A8000521F1070012008607047A74900201839D4
:100A90000860704700EB8000A34940000022143931
:100AA0000A60A24A121F10700120086070479E4918
:100AB000002014390860704700EB80009A4940001C
:100AC000002210390A60994AD21E10700120086075
:100AD00070479549002010390860704700EB80008E
:100AE0009149400000220C390A60904A921E107011
:100AF0000120086070478C4900200C39086070475D
:100B000000EB800088494000002208390A60874ACB
:100B1000521E107001200860704783490020083978
:100B2000086070478249097848430A21B0FBF1F117
:100B30008048491E80F86010582181761121C176C5
:100B4000042280F860205C228276C1767047794862
:100B5000002180F860105C2181761121C1767047F8
:100B6000714A10B5283214680123D10664B10024FB
:100B7000146081F8350091F83F0000BF91F83F40C4
:100B80008442FBD0136010BD81F83500FAE700EB1A
:100B9000C00101EB00106FF0030101EB800010B504
:100BA0006549664C0978B0FBF1F0401E80B2FF2821
:100BB0000CD9010A2170494200EB01206070FF202E
:100BC000FFF7CEFF2078401E207010BD002121705D
:100BD0006170BDE81040C0B2C2E7534828300168D8
:100BE00000290DD000210160C00690F83F1090F858
:100BF0003F20FF2A04D000BF90F83F208A42FBD05C
:100C0000704710B54D4C2178607851EA000207D04A
:100C100051B1FF20FFF7A4FF2078401E207010BDC7
:100C2000BDE8104007F012BCFFF79AFF002060708B
:100C300010BD3D4A10B5303214680123590794B1F4
:100C40000024146081F8370091F83F0091F83F408C
:100C50008442FBD0136091F83F0000BF91F83F2021
:100C60008242FBD010BD81F83700F3E72E483030C8
:100C7000016800290AD0002101604FF0005191F86D
:100C80003F0000BF91F83F208242FBD0704700EB4D
:100C9000800040001921B0FBF1F028490004000C4D
:100CA000488001D01920E3E6704710B5234C00239B
:100CB000608830B11920FFF7DBFE6088401E60803D
:100CC00000E00123184610BD00F01F0201219140F1
:100CD00040094FF0E02202EB8000C0F8001170479D
:100CE00000F01F020121914040094FF0E02202EB89
:100CF0008000C0F88011704700F01F020121914070
:100D000040094FF0E02202EB8000C0F880127047EB
:100D10004907090E002803DA00F00F00084A00E036
:100D2000084A8154704700001C050022330000204F
:100D3000AA02100000100020A902100014021000E6
:100D400014ED00E000E400E04948012101600021C9
:100D50000160704747480121016000210160704730
:100D600010B5002000F06BF8FFF7F4FFFFF7ECFF81
:100D70004149002008604149A0200870002000F08F
:100D80006AF8BDE81040002000F04DB83A48012153
:100D90001C38016000210160704710B5002000F090
:100DA0004EF8334901200860002000F054F8BDE8F7
:100DB0001040002000F037B82D4901201C39086090
:100DC00070472F4800782E49491C0978401A00F0D6
:100DD0003F0070472B4902780A7042784A70827847
:100DE0008A70C278CA7002790A7142794A7182792E
:100DF0008A71C079C8717047234800684178827849
:100E00004FF00050437A0374204B1B78437443899E
:100E10001B0A83744389C37401754275C179817556
:100E2000017AC175704700F01F020121914040090D
:100E30004FF0E02202EB8000C0F80011704700F094
:100E40001F020121914040094FF0E02202EB800097
:100E5000C0F88011704700F01F0201219140400945
:100E60004FF0E02202EB8000C0F8801270470000D3
:100E70005C840022A00000227C04002200E400E048
:100E80002004002000020020280210009D02100013
:100E900010B5092000F02BF80A2000F028F80920EE
:100EA00000F031F80A2000F02EF80521092000F0AA
:100EB00036F805210A2000F032F81E487F214170E3
:100EC0007C2282700171002100F848191A490968D2
:100ED00091F8C810CA0709D08A0707D510F84A2F19
:100EE000C1F38203012199408A43027010BD00F0D2
:100EF0001F020121914040094FF0E02202EB8000E7
:100F0000C0F88011704700F01F0201219140400994
:100F10004FF0E02202EB8000C0F8801270474907D2
:100F2000090E002803DA00F00F00044A00E0044A2A
:100F300081547047480000202802100014ED00E0A2
:100F400000E400E0704710B5044602462A21002064
:100F500000F074F9221D2B21002000F06FF904F13C
:100F600008022C21002000F069F904F10C020F2185
:100F7000032000F063F92068000E032825D304F154
:100F800014022D21002000F059F904F110022E2145
:100F9000002000F053F904F11C022F21002000F082
:100FA0004DF904F118023021002000F047F904F156
:100FB00024023121002000F041F904F12002322105
:100FC000BDE81040002000F039B910BD08B5072178
:100FD0006A46084600F032F9009808BD10B5C44CC6
:100FE000072060700020207044F2C000608000BFC5
:100FF00000BF00BF00BF4CF2C000608000BF00BF58
:1010000000BF00BF4CF2E00060800A20FFF750F9FB
:1010100044F2E000608000BF00BF00BF00BF4FF49B
:101020008040608010BDF0B500252E464FF0005482
:10103000E02717E0883401F03F016070217067807D
:1010400000BF00BF00BF00BFD4F808C043F825C0F0
:101050006680883C00BF6D1C521E491C3F2901D987
:10106000401CC0B2002AE5DCF0BD2DE9F047A04DE0
:101070000026AD1C04462E80DFF878920121C9F8C5
:1010800080104FF4C058A5F8008000BF00BF00BF1B
:1010900000BF00BF00BF4FF480572F803C20FFF7F8
:1010A00007F92E80FFF79AFF00F0DEF85C2000F0D1
:1010B000EDF82346012208210020FFF7B4FF231D8D
:1010C000012209210020FFF7AEFF04F108030122ED
:1010D0000A210020FFF7A7FF04F10C0301220B21D6
:1010E0000020FFF7A0FF04F1100301220C210020D3
:1010F000FFF799FF04F1140301220D210020FFF7EF
:1011000092FF00F0B1F8FFF769FF2F8000BF00BF2A
:1011100000BF00BF00BF00BF00BF00BF00BF00BFD7
:1011200000BF00BFA5F8008000BF00BF00BF00BF28
:1011300000BF00BF4FF440602880C9F88060BDE860
:10114000F087F0B54FF0000C059C0CB14FF0800C0F
:10115000C5B200264FF00057664C27E087F889504B
:101160004FEAC05EBEF1000F01F03F0E4EEA0C0EDA
:1011700001DA4EF0400E87F888E053F826E0C7F811
:101180008CE04FF0010EC4F8B0E04FF0000EC4F850
:10119000B0E0491CC9B2402902D36D1CEDB2002158
:1011A000D4F8C0E0BEF1000FFAD1761C9642D5DB30
:1011B000F0BD4FF0005282F88900002309B1802071
:1011C00002E0C00503D5402082F8880001E082F8E3
:1011D000883048480121C0F8AC10C0F8AC3000BFDE
:1011E000D0F8C0100029FBD17047F8B50C46054671
:1011F0004FF4F47600213046FFF7DBFF0020014674
:1012000000902B4622463046FFF79BFFF8BDF8B50D
:101210000C4605464FF4F87600213046FFF7C9FF2B
:1012200000214FF4FC70FFF7C4FF0020014600903E
:101230002B4622463046FFF784FFF8BD2C4B5870F2
:1012400041F0800003F888092A480021B430016089
:10125000012140F8B41900BFD0F8C0100029FBD11B
:10126000D3F890001060704710B5214C4FF48040C7
:10127000A41C20800420FFF71BF80020208000BF62
:1012800000BF00BF00BF00BF00BF10BD70B5184C4D
:101290002126A41C268000BF00BF00BF00BF00BFE6
:1012A00000BF40F02105258000BF00BF00BF00BF88
:1012B00000BF00BF44F22101084320800420FEF754
:1012C000F7FF258000BF00BF00BF00BF00BF00BF09
:1012D000268000BF00BF00BF00BF00BF00BF0020CE
:1012E000208000BF00BF00BF00BF00BF00BF70BDB7
:1012F0008800002000100022F8B5FF4C002635467B
:101300002670E6700120A66000F08EFC0C2000F034
:101310008BFC032000F088FC172000F085FC0120E6
:1013200000F08EFC0C2000F08BFC032000F088FC09
:10133000172000F085FC00F0DFFC6A460221EF4830
:1013400001F00DF9EE499DF80000EE4A08709DF895
:1013500001101170542800D0042600F0C7FE0521AA
:10136000012000F079FC05210C2000F075FC06211D
:10137000032000F071FC0621172000F06DFC012015
:1013800000F046FC032000F043FC172000F040FC76
:10139000A57065703046F8BD9065704738B50C464D
:1013A000009015460421684601F0A5FDD6498978CC
:1013B000C90604D5062C01D0032C00D1401C00998D
:1013C000296585F84E0038BD2DE9F041CE4C054623
:1013D000CE4E002084F8460030682246294690F818
:1013E00045076075E06AFFF7D9FF206BA065E5202F
:1013F0004FF0E90C042D08D0052D06D0012D33D077
:10140000022D31D00A2D7BD099E03168A37891F874
:10141000A8219B0622F0060201D542F0040201F544
:10142000D57184F84D200A8824F8342F4A886280C8
:101430000A7922714A796271CA88E2800A89228116
:101440008A7AA272CA7AE272497B6174A17C41F005
:101450000401A174AE49C1F30E01A182343C042DF4
:101460004FD0052D50D06AE0326892F81B1421F05D
:10147000060361888F0601D543F0040384F84D30DC
:10148000B2F81C3424F8343FB2F81E34638092F86A
:101490002034237192F82134637192F8223492F847
:1014A000B171C90543EA0723E38092F8243492F826
:1014B000B37143EA0723238192F82634A37292F88A
:1014C0002734E37292F82834A373A4F1340403D4CC
:1014D00092F82B1484F8441092F8291404F8451F4C
:1014E000617841F0040161708949F831C1F30E015E
:1014F000A4F80310453C012D03D0022D04D01EE0BA
:1015000005E084F84A001AE084F84AC017E0316820
:10151000A27891F85817920621F0060101D541F002
:10152000040184F84D1014F8461F41F004012170A5
:101530007749F839C1F30E0161802071463CA078EB
:1015400080070028306890F8660701DA20F0030071
:1015500084F84B00607D20F004006075664845709B
:10156000BDE8F041684800F0BCBE6848624A0068C7
:10157000127900F2073100F2FB2031F812206249A3
:101580004A830278CA7542780A7680788877002084
:101590000875887570472DE9F0475B4C05460020BB
:1015A00084F84600594EE12084F84A003168DFF89B
:1015B0006491594B91F845074F4F6075072D06D040
:1015C000082D17D0062D3ED0032D3CD034E091F8E5
:1015D00015C00A7D94F85C800CF1010C0CFB02F044
:1015E000B8F1010F03D902FB08F000FB0CF009EB86
:1015F000400008E0FFF7B9FF31683A79087D5043B1
:10160000464A02EB4000C0F30E00A4F8480091F8EF
:1016100053071A7800F0F00002F00F021043E07751
:1016200091F8550784F82100374A29465FF00100F8
:10163000FFF7B4FE2069A06560884107617D21D570
:1016400021F0040124E04A7DB7F808C0087D521C4F
:1016500002FB0CF2504309EB4000C0F30E00A4F86B
:10166000480091F853071A7800F0F00002F00F02DA
:101670001043E07791F8550784F82100224A294663
:10168000E068D5E7326892F8452702F0040211437A
:10169000617594F84A10072D14D021F0020100BFA3
:1016A000800784F84A100028306890F8660701DA4D
:1016B00020F0030084F84B007D70BDE8F04712482D
:1016C00000F07ABD41F00201EAE706282DD0092892
:1016D0002BD0072829D0082827D0032825D00C286C
:1016E00022D00D2820D00B281ED00A281CD0042878
:1016F0001AD0052818D013E018021000041000209A
:101700009C0210009D021000800A100028021000A8
:10171000F89F012000800120F6FF0100009E0120BB
:10172000012801D0022801D14EE634E7704730B5D8
:10173000FF4D8BB004460122FE48042C008808D0DF
:10174000052C06D0012C0ED0022C0CD00A2C07D070
:1017500022E0E97804291FD005291DD080071BD07D
:101760008DF800200CE0E978012915D0022913D06A
:10177000410702D410F0050F0ED002208DF80000B2
:10178000684601F049FD684600F090FB684600F0AD
:1017900046FB684600F048FEEC700BB030BDF8B573
:1017A000E34D0746012901D1002068716C79E24EB2
:1017B000641C07E056F82420694638469047012803
:1017C00004D0641C0E2CF5D90020F8BD6C719DF876
:1017D0000000F8BD70B5018800292BD001466022B9
:1017E000D44816F0C6FBFFF700F8D14C0025C4E939
:1017F00002502571607800281CD10121CD48FFF7E7
:10180000CEFF060016D0CD4901200870CC480068F4
:1018100090F8101149070ED590F8430780070AD4B5
:1018200000F064FE0220A07000F064FE192000F0B9
:101830008EFE667070BD25703046FFF778FF30462B
:10184000BDE8704041E700207047C268120006D032
:101850000088C00503D507200870012070470020CC
:101860007047C268120006D00088800503D50820A2
:1018700008700120704700207047C268120006D02F
:101880000088400403D50320087001207047002021
:101890007047C268120006D00078C00703D0062047
:1018A00008700120704700207047426A120006D07D
:1018B0000078000703D50920087001207047002038
:1018C0007047C26A120008D0026B32B100788006FD
:1018D00003D50A2008700120704700207047C26AB3
:1018E000120006D00078C00603D50B200870012036
:1018F000704700207047C26A120006D00078800747
:1019000003D50C2008700120704700207047026B3F
:1019100032B10078400703D50D20087001207047D0
:1019200000207047C26A120007D0026B2AB10088FB
:10193000C00402D501200870704700207047C26AB9
:10194000120008D0026B32B10088800403D5022057
:1019500008700120704700207047C26A120008D04A
:10196000026B32B10088400503D5042008700120C5
:10197000704700207047C26A120008D0026B32B173
:101980000088000503D5052008700120704700205D
:101990007047002008700120704700B589B0012011
:1019A0008DF8000000F075F96648019000F5F850D8
:1019B000039000F53A7004905E4881686846884755
:1019C00009B000BD5A4910B54A780120082A10D143
:1019D0000B795B1CDCB25A4B0C711B6893F8063315
:1019E00003F00F035B1C9C4204D21046FFF76DFE10
:1019F000002010BD00220A7110BD70B54C4C0120B2
:101A00006178062922D1A1684A4D491CA16095F848
:101A10005C2091421BDAE8682A4620F0010006218A
:101A2000FFF7BCFC464822890168487D097D401CBF
:101A30005043401C4843434901EB4000C0F30E00B3
:101A4000A5F84800284600F026FC002070BD0021C3
:101A5000A16070BD70B53A4909684B7D097D5B1C7A
:101A60004B4334490C460A7894F85C40D2071FD0A7
:101A7000012C1DD9498849051AD50020314A14E0A6
:101A8000012109E001FB030632F8105032F816601C
:101A9000491C354422F810508C42F3DC32F9101006
:101AA00091FBF4F122F81010401C9842E8D370BD6D
:101AB000047770BD70B588B0FFF784FF00280ED0A2
:101AC000FFF79BFF00280AD000211A48FFF767FEA6
:101AD000040006D0FFF72BFE2046FFF7F6FD08B006
:101AE00070BD134D154800246C7017490470A42074
:101AF0000873134E306890F81001400702D5AC709F
:101B000000F0E2FC2878012837D08DF80040012051
:101B10008DF81C006846FFF79DFF064C0B4D208892
:101B2000400518D53068407D420005EB40010FE0CC
:101B300018021000800A100068810100A70210003E
:101B4000280210000080012000100020F89F0120D2
:101B5000284616F0C9F94648019000F5F050029069
:101B600000F58070039000F53A70CDE90405F8386F
:101B70000690A16868468847B1E703208DF8000009
:101B8000C5E770B53B483C4E3C4C00684FF0000543
:101B900090F8101149070AD590F84307800706D43A
:101BA000A078012808D002280FD0032803D1A570FF
:101BB000FFF7F3FE357070BD0220A07000F09AFCB4
:101BC000BDE87040322000F0C2BC0320A0706078F5
:101BD000FFF7ADFD6078BDE8704076E5F0B5002216
:101BE0004D1E12E0531C1F460BE000BF30F8126080
:101BF00030F81340A64203D920F8136020F81240B1
:101C00005B1C9BB28B42F1D3BAB2AA42EADBF0BDB5
:101C100000F01F020121914040094FF0E02202EB49
:101C20008000C0F80011704700F01F0201219140B0
:101C300040094FF0E02202EB8000C0F880117047AD
:101C400000F01F020121914040094FF0E02202EB19
:101C50008000C0F8801270474907090E002803DA97
:101C600000F00F00064A00E0064A81547047000069
:101C70000080012028021000A702100018021000A6
:101C800014ED00E000E400E0FE4801680029FCD10A
:101C90007047FD4800220260FB481C380260FB4888
:101CA0000261012101618260816002600160026065
:101CB000F449A0F574700B68002BFCD1F4490B7B40
:101CC00043F020030B730B7B23F040030B730B7B60
:101CD00023F080030B730B7B23F020030B73C0F8FE
:101CE000D823C0F8E023EB4802707047E54818306D
:101CF00001680029FCD1704730B5E44800247430F5
:101D00000460E24880300460E048C4600121C160A2
:101D1000C460046001600460DF4D2020287068709A
:101D2000DB49593D0873A4200873D6481830016870
:101D30000029FCD1FFF7ADFFD848046085F8344096
:101D400030BDF0B518260022CE4DD1484FF4F83101
:101D50005C270C465FF0000303EB000E11F803C094
:101D60005B1C8EF860C00C2BF6DB2B68002BFCD1C3
:101D70008276C77604F10C0103EB000E11F803C064
:101D80005B1C8EF860C00C2BF6DB29680029FCD1A7
:101D9000511C8176C776921C04F13001B2EB460FDC
:101DA000D7DBF0BD2DE9F0479246089E5B1EC6F1D9
:101DB00008010022B64C01F0FF0C154600218946AF
:101DC0009A420BDA00EB0208875C98F8018027FA48
:101DD00006F708FA0CF847EA080703E007D1875C22
:101DE00027FA06F701EB040888F8607003E001EBBE
:101DF000040888F8609001F1010102F101020C2948
:101E0000DEDBA0490F68002FFCD10AEB0501A176AB
:101E10005C21E1766D1C022DD0DBBDE8F08738B582
:101E2000002504460095006A112330222946FFF759
:101E3000B9FF0095182335220021606AFFF7B2FF31
:101E400038BD00B58BB000208DF80000684601F069
:101E5000E3F96846FFF7E3FF0BB000BD2DE9F0475B
:101E60000024DFF820828A498246254626464FF024
:101E70005C0900209C4206DA00EB010C1AF80470A1
:101E80008CF8607002E0471887F86060641C401CA2
:101E90000C28EFDBD8F800000028FBD15019887619
:101EA00081F81B906D1C032DE3DBB6E710B50446EB
:101EB0004069182332220021FFF7D0FFA0692023B8
:101EC0003722BDE810400021C8E700B58BB00020E4
:101ED0008DF80000684601F09FF96846FFF7E6FFBD
:101EE000BAE7F0B500246A4D05E0165D6719641C79
:101EF00087F8606064B29C42F7DB624A1468002C89
:101F0000FCD1A976184340F01000E876F0BD70B51A
:101F100000235F4C05E0CD5C1E195B1C86F8605009
:101F20005BB29342F7DB57490B68002BFCD1A076DC
:101F300042F01000E07670BD30B5594C0722022007
:101F4000216801F24271FFF7E2FF2168022201F2EB
:101F50004A710920FFF7DBFF2168062201F24D716B
:101F60000B20FFF7D4FF20684E494F4D90F85307E0
:101F7000097800F0F00001F00F01084328700122F9
:101F800029461120FFF7C3FF2168032201F2577190
:101F90001620FFF7BCFF43480122401E007800F0E6
:101FA0000F01206890F85A0761F31F102870294626
:101FB0001920FFF7ACFF2168012201F25B711A20A2
:101FC000FFF7A5FF2168042201F25C711B20FFF7D7
:101FD0009EFF34480222C01C2946007828703148F0
:101FE000401C007868701F20FFF791FF21680222D3
:101FF00001F5EC612120FFF78AFF2A480222001D2B
:102000002946007828702748801C007868702720AF
:10201000FFF77DFF2168012201F263712A20FFF79B
:1020200076FF2168072201F266713D20FFF76FFFFE
:102030002068022290F86E17297090F86F07687078
:1020400029464420FFF763FF2168022201F5EE6173
:102050004620FFF75CFF2168082201F272714820D8
:10206000FFF755FF2168082201F27A715020FFF72F
:102070004EFF2168052201F284715820FFF747FFC7
:10208000226813E0040B00221C0C0022D003002263
:102090000010002019021000590000204005002205
:1020A00028021000F6FF0100E00A1000F84D92F837
:1020B0008F072870012302F28A72FA210020FFF7AD
:1020C00010FF2268012302F28C720E21C020FFF75C
:1020D00008FF2268012302F28D721421C020FFF74D
:1020E00000FF332068740B20A87430BD10B5FFF7D3
:1020F00023FFFFF7EAFEFFF7A4FEBDE8104020E64D
:1021000038B50546E34C006D00906073010AA17379
:10211000010CE173000E2074042269462B20FFF7A6
:10212000F6FE012205F14E012F20FFF7F0FE95F893
:102130004E00A074A86D0090E074010A2175010C96
:102140006175000EA075042269463520FFF7DFFE99
:102150000098800F84F84000CF4901220870392090
:10216000FFF7D5FE38BD00EBC00101EB00106FF0AA
:10217000030101EB800010B5C849C94A0978146809
:1021800090FBF1F0401EC1B20123580764B1002456
:10219000146080F8341090F83F1000BF90F83F4072
:1021A0008C42FBD0136010BD80F83410FAE7BD48B4
:1021B00001680129FCD170477CB5044600208DF8E8
:1021C00004002046FFF79CFFB148B4F84810401CBB
:1021D0000180217D00F8011C94F84A104173AD4E36
:1021E000A07D86F83600B04D286890F842078DF83B
:1021F00000006188890503D520F012008DF80000E9
:10220000012269460220FFF782FE042204F1150133
:102210000520FFF77CFE2968022201F24A7109209D
:10222000FFF775FE022204F11A010C20FFF76FFE82
:10223000022204F11C010E20FFF769FE052204F1C1
:102240001E011020FFF763FE286890F80907C007F9
:102250000AD0012201A94420FFF759FE022204F10D
:1022600040013F20FFF753FE012204F14B013D20C6
:10227000FFF74DFE012204F14C014420FFF747FE19
:10228000884801680129FCD194F84A003073232062
:10229000FFF769FF7CBD38B504467E4D006D0090A8
:1022A0006873010AA973010CE973000E28740422F3
:1022B00069462B20FFF72BFE012204F14E012F204F
:1022C000FFF725FE4834A079A87471482188401C86
:1022D0000180A1784173A07828732320FFF743FF82
:1022E00038BD7EB50446FFF70BFF6948B4F84810C7
:1022F000401C018094F8431000F8011C94F84A1027
:102300004173694D286890F842078DF80000618894
:10231000890503D520F012008DF8000001226946DE
:102320000220FFF7F4FD012204F115010520FFF75B
:10233000EEFD94F84600574EC00708D0286800F21A
:10234000957190F8950786F83600012206E094F81A
:10235000440086F83600012204F144010620FFF70C
:10236000D6FD012204F142010720FFF7D0FD012232
:1023700004F145010820FFF7CAFD2968022201F295
:102380004A710920FFF7C3FD286890F80907C007C4
:1023900007D000208DF80800012202A94420FFF791
:1023A000B6FD012204F14D011720FFF7B0FD94F8AE
:1023B0004A00400701D5042000E002208DF8040007
:1023C000012201A91820FFF7A2FD022204F1340125
:1023D0001B20FFF79CFD022204F136011D20FFF7B0
:1023E00096FD012204F138012120FFF790FD012222
:1023F00004F139012220FFF78AFD012204F13F0197
:102400002A20FFF784FD012204F14B013D20FFF754
:102410007EFD244801680129FCD194F84A003073FC
:102420002320FFF7A0FE7EBD30B50446C0691A4DDB
:102430000122007800F00F011B48006890F85A074D
:1024400061F31F10287029461920FFF760FDE0682E
:1024500002222946007828706068007868701F2082
:10246000FFF755FD20692946022200782870A068F0
:1024700000786870BDE83040272048E50A490A68BE
:1024800092F84D270270096891F85517017370474B
:102490005300002000100020E00A1000A9021000E4
:1024A00040050022000B00222802100010B504464F
:1024B000014601220B20FFF72AFD04F10C01012245
:1024C000BDE81040132022E5674908B504200873D1
:1024D000664801226946006890F8430720F008002A
:1024E0008DF800000320FFF712FD08BD5E49202093
:1024F0000873CCE718B55E4C01226946207840F09D
:10250000F0008DF800001046FFF701FD5649C0208D
:10251000087320788DF80000012269461046FFF705
:10252000F6FC18BD534900200860B0E75148403020
:1025300001680029ABD0002101604FF0005191F8F3
:102540003F0000BF91F83F208242FBD09FE74949FE
:1025500000220A60484A10700120086097E770B5B1
:10256000464C2368002BFCD11D4603E0C6185B1CBB
:1025700086F880508B42F9D32368002BFCD102E00F
:10258000C45CD4545B1C8B42FAD370BD10B501F00F
:10259000BBFCFFF7CBFF3A48007878B137481838D2
:1025A00001680029FCD13048C078400602D5354981
:1025B00001200870BDE81040FFF77CBA32490020C6
:1025C000087010BD10B501F09FFC2A49002008607A
:1025D000BDE81040FFF7D5BA10B501F095FCFFF744
:1025E000A5FFBDE81040FFF7CCBA1F4B10B5987699
:1025F000DA76224818380468002CFCD1012083F8D0
:10260000E0001E480468002CFCD1002005E0C4183E
:1026100094F860400C54401C40B29042F7DB10BD6F
:1026200008B543F6FF70ADF80000022269463F206E
:10263000FFF76DFC0220ADF80000012269463D2045
:10264000FFF765FC0849E02008734FF44870FDF778
:102650002FFE022269468720FFF7C7FFFFF734FFEE
:10266000BDF8000008BD0000001000202802100086
:102670005C021000000500222D0000201C0B00222F
:102680001902100018021000A7021000704800681C
:1026900090F8F007C00605D5ED214EF6ED5208463C
:1026A00005F0E3FFFEE705460E46012005F09FFF1B
:1026B000694C6848C4E900062868A0606868E06062
:1026C000A8682061E86860612869A0616869E061C4
:1026D000A8692062614EE869606230685F4FA0625D
:1026E000103F386807F10408E062D8F8000008F1EC
:1026F00004092063D9F8000006F1040A6063DAF8DF
:102700000000DFF858B1A063ABF1340BDBF8000038
:10271000E063381F00682064FEF767F86064504883
:1027200000210068A0640F202A6805F078FF0121CD
:102730000F206A6805F073FF02210F20AA6805F0D8
:102740006EFF03210F20EA6805F069FF0C210F20BE
:102750002A6905F064FF0E210F206A6905F05FFF0A
:102760000F210846AA6905F05AFF20210F20EA69C7
:1027700005F055FF326821210F2005F050FF3A681F
:1027800022210F2005F04BFFD8F8002023210F2035
:1027900005F045FFD9F8002024210F2005F03FFF68
:1027A000DAF8002025210F2005F039FFDBF80020A2
:1027B00026210F2005F033FF381F026827210F2044
:1027C00005F02DFFFEF711F8024630210F2005F02D
:1027D00026FFFFF75BFF012807D002280FD0032850
:1027E00005D0042805D004210AE0012108E00321D6
:1027F00006E00021032005F0FAFEFFF747FF022163
:10280000032005F0F4BE10B504460146042005F08F
:10281000EEFE012C01D1FFF739FF10BD0146082063
:1028200005F0E5BE0146062005F0E1BE10B5044600
:102830000146072005F0DBFE012C03D0022C01D05D
:10284000032C01D1FFF722FF10BD0320EEE70000AB
:1028500028021000AF0550FA5C00012038ED00E0BE
:102860006802100001F050BB704770471B4810B55C
:10287000016821F00401016001F046FBBDE8104051
:1028800014F0B2B87047704701F03EBB01F03CBB9A
:1028900001F03ABB704770477047704701F034BB96
:1028A0007047704770477047704770477047704770
:1028B00010B501F029FBBDE81040FEF7A2B910B534
:1028C00001F022FB06480078012801D102F065F9E9
:1028D00004490020086010BD7047704710ED00E00B
:1028E000A60210004805002210B55C219E4815F094
:1028F0007AFB9D489D499E4A018082809D49418086
:102900009D4BC3809D4C04819D4C44839D4C84838E
:102910009D4CC4839D4C04849D4C44849D4C848474
:102920009D4CC4841A309D4CC481838401844284AC
:102930009B49C1849B499D4B0968B1F87920028568
:10294000B1F85F214285B1F88D208285B1F8D6209B
:10295000C2850022028642868286934A5B1E1288C6
:10296000C2864A7D02870A7D4287904A1B78127888
:1029700042EA0322C287B1F84B2052BAA0F84020A5
:10298000874891F84E274280B1F85C17C1800181D9
:1029900010BD8648113001788548552901D019218C
:1029A00002E0824913310978017070472DE9F04740
:1029B000FF2228217F4815F00EFB7E48FEF7C3FA60
:1029C0007C480E2401254268072645F2AA518A4216
:1029D00002D082688A423CD180460068D8F808203C
:1029E000070E89464A4506D1032F01D1C0F30135B0
:1029F000C0F3032602E00120FFF714FFD8F804100B
:102A0000494504D198F8000000F01F0402E00220BC
:102A1000FFF708FF032F22D1D8F814304946664A41
:102A200040468B4201D1036900E0644B1360C369E7
:102A3000634A8B4201D1836900E0624B1360436AB1
:102A4000614A4B4502D1D8F8200000E05F48106091
:102A500005E00120FFF7E6FE0220FFF7E3FE05F0A8
:102A6000030040EA061020F00C014E48006890F880
:102A70004107C0F3C00241EAC201C0F3800041EA4D
:102A8000800153480170534880F86010012181761D
:102A90001121C1765048017864F304010170BDE84A
:102AA000F08770B5FDF721FFFEF75AF93D4D286814
:102AB0000078A52802D00120FFF7A5FE4FF00850AE
:102AC0000124C0F898432868444A817C01F0010140
:102AD0001160807C111DC0F340000860FEF732FADF
:102AE000FDF726FFFEF708FC042801D1FFF773FE6F
:102AF000FEF782F9FEF7CCF93648802180F86010A5
:102B0000042181761121C176FFF750FFFFF741FFC5
:102B100032486C38046031480C38046070BD10B520
:102B20004FF0005142F218004881FFF7BAFFFFF75B
:102B3000DBFE2B495F2008602A49002008602B48F3
:102B40002949016001F5086029490860294800F019
:102B500021FFFDF7A7FB00F04FF8FDF7A1FBFDF704
:102B600025FC012010BD0000000001200080012094
:102B700000DB012080D3012060A20120009F012002
:102B8000100801204C080120740B0120B00B01201B
:102B9000E8040120240501206C040120A804012080
:102BA0000425100028021000C4021000E1FF0100FB
:102BB000A9021000302E1000B402100040A5AE0291
:102BC000B802100000879303BC02100000366E01AB
:102BD0005C02100000100020200000208804002269
:102BE000700B012098021000EC121000700210000F
:102BF00074021000EC2310007FB5FDF7AFFB274DEA
:102C0000002400BF05EB441000F11002017F4CCA04
:102C1000CDE90261CDE900230FC8FDF783FD10B1B6
:102C20000220FFF703FE641C082CEBDB1C4D002484
:102C300004EB440005EB8001091D55F8200006C98E
:102C4000FDF7F0FC10B10220FFF7F0FD641C072C2B
:102C5000EEDB134D0024543505EBC400416855F8F4
:102C60003400FDF7F9FB10B10220FFF7DFFD641C13
:102C7000072CF1DB7FBD4068FFF7E7BD38B50C4698
:102C80000546012A01D1FDF707FC69462846FDF7F4
:102C900042FC00992142F8D138BD0000A481010016
:102CA000A48201002DE9F04300245F1EDDF81C9092
:102CB00028E02546661C07E030F915C030F916807B
:102CC000C44500DB3546761C9E42F5DB30F81460C7
:102CD00030F815C020F814C020F81560B9F1000FC5
:102CE0000FD031F8146031F815C021F814C021F864
:102CF000156032F8146032F815C022F814C022F8BA
:102D00001560641CBC42D4DBBDE8F08310B5002420
:102D10000388012A06D05BB15B1E1904090C0180EF
:102D200006D007E05B1C9AB202808A4202D9048076
:102D3000012010BD002010BD01EB8010801001EBC0
:102D400041014900182291FBF2F300EB400000F52D
:102D5000F83002FB1311006820F07F40C84000F0FB
:102D60003F0070472DE9F04F88B0074600200190E2
:102D7000029003900490059006900790F848012572
:102D8000F64E80462AE0022420E0087D04FB005035
:102D900036F91000B84218DD01200090032305AA7F
:102DA00003A901A8FFF77EFFD8F80000BDF90410C1
:102DB000007D04FB005036F91000814205DAADF8C1
:102DC0000400ADF80C50ADF81440641CD8F80010A5
:102DD00040464A7D521EA242D7DC6D1C0168097D27
:102DE000491EA942CFDC00240DF10C0BB246C146AE
:102DF0005FF0000505A83BF914C030F91430D9F88C
:102E00000000017D504603FB01C63AF91660BE4240
:102E100035DDD44E76571E4406FB01C2731C03FBFE
:102E200001C130F812203AF811006146101A0FFA69
:102E300080F8701EFFF780FF009061463046FFF774
:102E40007BFF01460098401A002807D0D9F80000FF
:102E50000EDAB0F8651441450FDB1CE0D9F800002C
:102E6000B0F861144A42424515DAB0F8651402E040
:102E7000B0F86104414241450DDD012007906D1C11
:102E8000EDB2022DB6D3641CE4B2032CB0D3079884
:102E900008B0BDE8F08F0020FAE7F0B50546002045
:102EA0004FEA254C4FEA2146BCEB060400D56442AC
:102EB0009C421FDA4FEA2247BCEB070400D564426C
:102EC0009C4217DAF41B00D564429C4212DA2DB200
:102ED0000CB2291B00D5494299420BDA12B2A91A49
:102EE00000D54942994205DAA11A00D549429942D2
:102EF00000DA0120F0BD70B50346002002469A4C6E
:102F000009E09D5C521C05F00F0604EB1515A65D4B
:102F10002D78304428448A42F3DB70BD884200D3C8
:102F200008467047884200DB08467047884200D850
:102F300008467047884200DC08467047884200D344
:102F40000846904200D310467047F0B50025059F13
:102F500014E000240EE000BF05FB03F600EB860C36
:102F600001EB86065CF824C09CFBF7FC46F824C005
:102F7000641C64B29C42EFDB6D1C6DB29542E8DBD1
:102F8000F0BDF0B50025059F14E000240EE000BF61
:102F900005FB03F600EB860C01EB86065CF824C00B
:102FA0000CFB07FC46F824C0641C64B29C42EFDBB7
:102FB0006D1C6DB29542E8DBF0BDF0B50025059FB4
:102FC00017E0002411E000BF05FB07F600EB860CBC
:102FD00001EB860E5CF824C05EF824E002EB860666
:102FE000F44446F824C0641C64B2BC42ECDB6D1CA3
:102FF0006DB29D42E5DBF0BDF0B50025059F17E001
:10300000002411E005FB07F600EB860C01EB860EB1
:103010005CF824C05EF824E002EB8606ACEB0E0CF4
:1030200046F824C0641C64B2BC42EBDB6D1C6DB27C
:103030009D42E5DBF0BD2DE9F04F814609A88A46A7
:10304000B0E822400020DDF834B08A4221D020E7E9
:1030500000241BE0002116E000FB02FC01FB05F848
:1030600000FB0BF609EB8C0C0EEB860603EB8808D5
:103070005CF821C056F8247058F82480491C0CFBD9
:10308000087746F824709142E6DB641CAC42E1DB31
:10309000401C5045DCDBFCE631480068017B427B8C
:1030A00041EA0221827BC07B41EA024141EA0060A1
:1030B000400070472A4800680179427941EA0221BC
:1030C0008279C07941EA024141EA006070472749AC
:1030D00031F91000704700B5FFF7DEFF40084000EF
:1030E00000BD2DE9F8430C460546FFF7F4FF0090BC
:1030F000FFF7D2FF814604216846FFF7FCFE05EB8F
:10310000400C0025009F29462B46012606FA03F2B3
:103110003A4208D012EA090F04D03CF8112024F8F2
:1031200015206D1C491C5B1C1E2BEFDB0C4909682C
:1031300091F8F017C9070AD000220C4905E093B2B4
:1031400031F8133024F81230521C8242F7DBBDE80C
:10315000F8830649403131F910007047F00A100039
:1031600028021000CE021000308301003CFE010056
:10317000A0E72DE9FC430C460646FFF7ACFF0190A3
:10318000FFF798FF0090FFF795FF8146042101A803
:10319000FFF7B1FE054604216846FFF7ACFE00EBE1
:1031A000450106EB41070025DDF8006029462B4666
:1031B0004FF0010C0CFA03F2324208D012EA090F68
:1031C00004D037F8112024F815206D1C491C5B1C15
:1031D000202BEFDBF749096891F8F017C9070AD0EF
:1031E0000022F54905E093B231F8133024F812308B
:1031F000521C8242F7DBBDE8FC8300B5FFF74CFFB1
:1032000040F0010000BD55E7EC4A520102EB81019C
:1032100001F108510860A0E70178012918D00229BE
:103220009BD1E7494160491C8160E6494161E5491C
:103230002C318161E249891CC160491C0161491F2F
:10324000C161E0496C310162DE498D31416284E740
:10325000DB4910394160491C8160DA49BD31416167
:10326000D849E9318161D6490E39C160491C0161F3
:10327000491FC161D4490162D3492131E6E7F0B564
:1032800007460598884201DD1846F0BDB84201DACC
:103290001046F0BD9E1AC01B4643CD1B00D1012530
:1032A000C44C96FBF5F02468104400B294F8F14742
:1032B0000E2CEED1A446C54CA4F800C04FEA264C13
:1032C000A4F802C0A6802E14E68025816781A18122
:1032D000E28123826082F0BD01EB8010801010B586
:1032E00001EB41014900182391FBF3F403FB141394
:1032F00000EB400000F5F8303F2401689C40A143FA
:103300009A400A430270110A4170110C817010BD7D
:103310002DE9F04F8B4682460026FFF76EFF81466F
:10332000FFF7C8FE07464FF0180C00254FF00108C4
:1033300008FA05F111EA090F13D0002408FA04F085
:1033400038420AD0BBF1010F10D01AF806202146EE
:103350002846FFF7C1FF761CB6B2641CA4B2202C2D
:10336000ECD36D1CADB26545E2DB92E52146284603
:10337000FFF7E2FC0AF80600EDE7914915390880ED
:10338000EBE68F481538B0F90000E6E62DE9FF4F6F
:103390000027864681B04FF0FF093E46BC46481CD8
:1033A00052D0501C50D0881E012800DC0120C4B22D
:1033B000804801F1020805682B7D981E404501DD1B
:1033C000881C00E0981E00F0FF0B901E012800DC16
:1033D0000120C0B20090687D02F10208851E4545BB
:1033E00001DD901C00E0801E00F0FF0A18E0009D47
:1033F00012E000BF05FB034080B21EF800008444C9
:103400001FFA8CFCB84200D90746814500D9814695
:10341000761C6D1CF6B2EDB25545EBD9641CE4B2D6
:103420005C45E4D953430EEB0100185CBCEB000192
:1034300001D5C1F10001A6F1010691FBF6F1411A97
:1034400000D5494204980170A7EB0900C0B205B04D
:103450001FE530B5574A0346594814681538B4F883
:10346000B52694F84647B0F9000004F00F04641C38
:1034700002FB040562439D4207DAA2EB60029A1A3E
:1034800092B292FBF0F0084409E0141A9C4208DD65
:1034900002EB6002D21A92B292FBF0F0081AC0B2AC
:1034A00030BD084630BD2DE9FC4F8B4682460026D4
:1034B000DFF81CC13F4CDFF81C91DFF81C8117E0DE
:1034C00001250FE0007D002205FB00618FB2391A53
:1034D00038F9170019F80110FFF7BBFF6D1C0CF845
:1034E0000700EDB22068417DA942EBD2761CF6B20E
:1034F0002068007DB042E3D820684FFA8AF24FFA84
:103500008BF1007D6B46604416460D46FFF73EFF8B
:10351000074601AB324629462E48FFF737FF0146E2
:10352000206890F8542407EB9210884207D39DF846
:1035300000009DF8041000EB9210884202D2012096
:10354000BDE8FC8F0020FBE71F4A533222F8101021
:1035500003E61D49533131F91000FEE5164A22F801
:103560001010FAE5144A403A22F81010F5E5F0B5CB
:103570001049074600200E68022396F815E015E072
:10358000347D0122A11E0EE003FB0425ADB205F13E
:10359000010C1FFA8CFC7D5D17F80CC0654501D14C
:1035A000401C80B2521C9142EEDC5B1C9E45E7DC65
:1035B000F0BD0000280210007CFE0100700B01200D
:1035C000F7FF010040F8010069F9010000DB01206C
:1035D000A0AD0120E0A90120F00A10002DE9F04380
:1035E0004FF00008FFF709FE4FEA500CFFF762FDAD
:1035F000074600264FF0010909FA06F1394214D0B6
:103600000024254609FA05F010EA0C0F0AD03146CD
:103610002846FFF791FBA04203D108F101011FFAF0
:1036200081F804466D1C182DECDB761C202EE3DBA4
:103630004046BDE8F0832DE9F14F4FF00008FFF759
:10364000DCFD4FEA500CFFF735FD074600264FF032
:10365000010A00BF0AFA06F1394221D0009800257C
:10366000DFF890B42C4600EB060900BF0AFA04F01C
:1036700010EA0C0F11D031462046FFF75DFBDBF856
:103680000010621C097D5143A84201F8090003D1D2
:1036900008F101011FFA81F80546641C182CE5DBCE
:1036A000761C202ED6DB4046BDE8F88F2DE9F05F72
:1036B00083464FF000084FF4787114F094FCFFF744
:1036C0009CFD4FEA500CFFF7F5FC074600244FF035
:1036D000010A00BF0AFA04F111EA0C0F1ED00025FE
:1036E0002E4604F1010900BF0AFA06F0384212D052
:1036F00031462046FFF720FBFE490BEB0602A842AD
:103700000968097D01FB09F1885403D108F1010121
:103710001FFA81F80546761C202EE5DB641C182C68
:10372000D8DB4046BDE8F09F01464FF404624FF4F9
:10373000F83014F0D9BB30B5EF4A0021ED4B05E06D
:1037400032F8114020F81140491C89B21C68257DCF
:10375000647D65438D42F3D830BD30B5E64A002123
:10376000E44B05E030F8114022F81140491C89B2C1
:103770001C68257D647D65438D42F3D830BD2DE9FD
:10378000F04381460026FF27481C38D0501C36D015
:10379000881E012800DC0120C4B2901E022800DC33
:1037A000022000F0FF0CD34801F102080068057DFB
:1037B000AB1E434501DD891C00E0A91E01F0FF0896
:1037C000417D931C481E984201DD911C00E0491E7A
:1037D000C9B212E063460CE003FB054080B219F861
:1037E0000000B04200D90646874200D907465B1C5C
:1037F000DBB28B42F0D9641CE4B24445EAD9F01B39
:10380000C0B216E72DE9F84F4FF0FF3B0024BB484C
:10381000CDF800B0FFF70FFFB64EDFF8E09230684A
:10382000007D00EB400109EB8100817B027C1144AB
:103830004908C1734846FFF79AFE05460027DFF89E
:10384000C0A2B04622E0012619E0007DAD4A06FB89
:1038500000711FFA81FCACEB000032F91C30A64A63
:1038600080B219F80C1032F9100000285ED082B234
:103870001846FFF7EEFD761C0AF80C00F6B2D8F8F1
:103880000000417DB142E0D27F1CFFB2D8F8003089
:10389000197DB942D7D8197D01EB41020AEB8201AB
:1038A0008A7B0E7C32444FEA5202CA734FF0000208
:1038B0001E7D1CE001215F7D15E000BF01FB06209D
:1038C00080B21AF8008019F80000B8EB000000D5AB
:1038D000404240B2A04204DD044648B24FFA82FBA7
:1038E0000090491CC9B28F42E8D2521CD2B2964213
:1038F000E0D88348FFF73BFE7E4C216891F88114A5
:103900002944814212D3A84212D359467C48009AD6
:10391000FFF735FF054659467848009AFFF72FFF15
:103920002168401B91F88214884201DD0120BBE62A
:103930000020B9E6704931F910000EE4821002EB64
:1039400042020A4400EB40004000182190FBF1F3D2
:1039500001FB1301106820F07F40C84000F03F00D9
:1039600059E4831003EB430310B51A4400EB400005
:103970004000182390FBF3F403FB14033F2410686A
:103980009C40A043994001431170080A5070080CF4
:10399000907010BD2DE9F14F82B04FF0000B7821EF
:1039A000029814F042FBFFF728FC4FEA5008FFF79B
:1039B00081FBDC46814666464FF0010A0AFA06F1B1
:1039C00011EA090F25D000240AFA0CF00127254638
:1039D000CDF800000AFA05F010EA080F14D03146BD
:1039E0002846FFF7A9F9A04208D00299009A51F899
:1039F00027101143029A42F8271003E00BF101014E
:103A00001FFA81FB04467F1C6D1C182DE2DB0CF1B4
:103A1000010C761C202ED1DB5846BDE8FE8F2DE927
:103A2000F04F8346334800242246D0F800A00121FD
:103A30009AF81450A5F1010621E003200123DFF8D4
:103A4000C8E003FA01F99AF8157015E05EF820C095
:103A50001CEA090F0FD0A0F1010300FB051C03FBBA
:103A600005183BF91CC03BF91830BCEB030300D52B
:103A70005B421C44521C401C8742E7DC491C8E42BE
:103A8000DBDC02B9012294FBF2F06EE42DE9FF4F7A
:103A900085B0002103910291019100911549012BFC
:103AA0000C6894F8725205F00F0700D10027667D6C
:103AB00094F87532C7F1100BB34200D21E460023B2
:103AC000049301238FE000BF4FF00009C846032490
:103AD0002DE00D4951F824C0012199401CEA010F45
:103AE00004FB053130F911C0A4F1010101FB0531DE
:103AF0000CE0000028021000BCF90100E0A9012040
:103B0000A0AD0120F00A1000EC23100030F91110D4
:103B1000ACEB010106D0002900DA4942DDF818C0FB
:103B2000A1EB0C01002900DA49428944641CB4422B
:103B3000CFDB31469EF815A01FE0FE4C54F821C0A3
:103B400001249C401CEA040F01FB053430F914C029
:103B5000A1F1010404FB053430F91440ACEB04047A
:103B600006D0002C00DA6442DDF818C0A4EB0C0487
:103B7000002C00DA6442A044491C8A45DDDC04992B
:103B8000012910D10199B1EB090101D5C1F1000161
:103B9000039C214403910099B1EB080100D54942EF
:103BA000029C21440291CDE900899EF87612994247
:103BB00016D11168039D79430BFB0511CC1701EB5E
:103BC0001471091111609168029D79430BFB051175
:103BD000CC1701EB1471091191600021039102913E
:103BE00001215B1C0491D449D1F800E09EF81450E7
:103BF000691E99423FF768AF5068039978430BFB01
:103C00000100C11700EB117000115060D068029BD9
:103C100078430BFB0300C11700EB11700011D0605B
:103C200009B032E730B5044600200222A1F10101BB
:103C30000BE000BF04EB420534F9123035F9025CA9
:103C40005B1B00D55B421844521C8A42F2DB30BD3C
:103C500070B5B94A002001461268B84C537D0BE09C
:103C600034F91150B2F84F64B54203DBB2F8516435
:103C7000B54200DD0120491C8B42F1DC70BD70B5FE
:103C8000AD4C00252068417DAC480AF01BF9064682
:103C90002068017DAA480AF015F92168B1F84D1491
:103CA000814201DBB14200DA0125284670BD2DE9D1
:103CB000F14FA149002318460C6894F84814267D5A
:103CC000C1F3C001B4F858B4B4F85AA4A6EB010982
:103CD00025E0657D0322DFF85CE2DFF86882A5F16C
:103CE000010518E05EF822C0012707FA01F71CEA77
:103CF000070F0ED102FB061738F917C0A2F1010712
:103D000007FB061738F91770BCEB070700D57F4291
:103D10003B44521CD2B29542E4DC491CC9B28945ED
:103D2000D7DC00999B450B6002D2534500D201209D
:103D3000BAE47CB50D460446FFF7CDF90090FFF7D5
:103D4000B9F9019000980421400800906846FFF7F7
:103D5000D2F80646042101A8FFF7CDF830448200CE
:103D60002146284614F0C0F87CBD0B46724930B499
:103D70000A6804460020517D157D01F1010192F889
:103D8000F02701FB05F1150709D40CE033F91050B9
:103D900034F91020954201DA23F81020401C8842A3
:103DA000F4D330BC7047D2070ED0674A674C1288F4
:103DB0002280674C05E082B234F8122023F81020EC
:103DC000401C8842F7D3ECE74A00214630BC184635
:103DD00014F08AB870B50446602114F026F900206A
:103DE000554B20806080196891F8941701F001010B
:103DF00040EA41116180A060FFF7FFF9E060FFF742
:103E000059F9544D206168886083186800F2467043
:103E1000C27A817A02F03F0241EA0221A18341780D
:103E2000E17590F8491021750178A17581782176A6
:103E3000017BA1774449407B143100F0F000097800
:103E400001F00F010843E077FFF745F9E062FFF763
:103E500031F92063E888A0866087186890F8B61169
:103E600084F8421090F8921784F8431090F8931752
:103E700084F8441090F8911784F84510B0F85E1754
:103E8000E186A18790F8601784F8381090F86117E0
:103E900084F8391090F8621784F83E1090F8631790
:103EA00084F83F1090F8661784F84B1090F848108B
:103EB000C9070AD090F8490000F00F0084F85C00B0
:103EC000608840F48060608070BD012084F85C00F0
:103ED00070BD10B50446FCF7E5F9012C0BD116486E
:103EE000006890F81001800705D5FCF70CFD38B18B
:103EF000FCF702FD04E0FCF706FD08B9FCF7F5FC51
:103F0000BDE81040FCF7CCB90020E2E70A4B10B541
:103F10001A68947F640704D5D28A0468A2EB04026D
:103F200002601A68947FA40703D5128B0C68121BD9
:103F30000A6011E0EC231000280210001008012094
:103F40004C08012080D30120E2FF010000DB0120AA
:103F5000BCF90100042510000268002A00DA0022E2
:103F600002601C68E48AA24200DD224602600A6800
:103F7000002A00DA00220A601C68248BA24200DDBD
:103F800022460A601B689B7FDB0702D003680B6038
:103F9000026010BDF0B5F74D002301242D6895F89F
:103FA000CE5000BF04FA03F635420AD031F913604F
:103FB00030F91370F61B32F91370BE4201DD012097
:103FC000F0BD5B1C062BEDDB0020F0BDF0B500253D
:103FD0002C46059E0AE000BF31F9147030F914C078
:103FE000A7EB0C07974200DD6D1C641C9C42F3D3C9
:103FF000B54201D30120F0BD0020F0BDF0B500278F
:104000003C465B1EDDF814C01BE000BF31F81450C5
:1040100030F8146000EB440EAD1B01EB4406BEF813
:1040200002E076882DB2A6EB0E0636B2002D00DC3B
:104030000025002E00DC00263544954200DD7F1C63
:10404000641C9C42E2D3674501D30120F0BD0020EF
:10405000F0BD2DE9F047C74EDDE9089A00252C4652
:10406000366811E0377D30F9148094FBF7FC07FBCC
:104070001C4731F914C07FB2ACEB080C944502DD4B
:10408000574500DB6D1C641C9C42EBD34D4502D3AD
:104090000120BDE8F0870020FBE72DE9F04FB54C8B
:1040A000DFF8D4C29B462468DDE90A759CF800C09D
:1040B0000023DDF824E094F89061BCF1010F01D1F8
:1040C000012D01D000242FE00121DFF8B092DFF8AC
:1040D000B0A294F815C015E0002010E0257D01FB8A
:1040E000050539F915703AF9155005EB02084745F1
:1040F00003DAA5EB0B05AF4200DC5B1C401CB042B1
:10410000ECD9491C8C45E7DA10E000BF31F91450B6
:1041100030F9146005EB020C664503DAA5EB0B05DC
:10412000AE4200DC5B1C641CBC42EFDB734501D972
:104130000120AAE40020A8E42DE9F04F8A46DDE939
:104140000997012547F6F8714E429346AC46002484
:1041500017E000BF30F814803AF81420A2EB0802F0
:1041600012B2914200DD1146964200DA1646002A4C
:1041700002DA4FF0000502E001DD4FF0000C04F11F
:104180000104BC42E6DB55EA0C0206D0012D01D049
:104190002DB108E0BCF1010F05D1002112E0BCF106
:1041A000010F00D13146002905DD03EB0902B1EB17
:1041B000420FF2DC06E005DA03EB09025242B1EBF2
:1041C000420FEADB00252C462A4610E030F8126048
:1041D0003AF812C00E44ACEB060636B29E4205DA3F
:1041E000C9F1000C664501DD3544641C521CBA421D
:1041F000ECDB95FBF4F20A44002105E030F81130C5
:1042000013442BF81130491CB942F7DB3DE42DE98A
:10421000FF4F8246DDE90DB7012447F6FF70C54325
:104220008E462646002216E03EF812C03AF81210DA
:10423000ACEB010109B2884200DD08468D4200DA8C
:104240000D46002902DA4FF0000402E001DD4FF0D4
:10425000000602F10102BA42E6DB54EA060105D08B
:10426000012C01D024B106E0012E04D1002011E080
:10427000012E00D12846002805DD03EB0B01B0EB31
:10428000410FF3DC06E005DA03EB0B01490049427C
:104290008142EBDC00221446164615469146114633
:1042A00019E000BF3EF811803AF811C0A8EB0C0CE1
:1042B000ACEB000C0FFA8CFC9C450BDACBF1000840
:1042C000C44507DD01FB014401FB0C550A4466446B
:1042D00009F10109491CB942E4DB04FB09F102FBC5
:1042E000121C05FB09F102FB1618744305FB124171
:1042F00091FBFCF5002215E008FB02F191FBFCF1BB
:104300002944994201DD194604E0CBF10004A142A1
:1043100000DA21463AF8124001442144029C24F874
:104320001210521CBA42E7DBBDE8FF8F30B564249F
:1043300007E000BF30F91350554395FBF4F521F821
:1043400013505B1EF6D230BDF0B506460020044681
:104350000546521C059F09E036F911C09C4504DD55
:10436000A44502DD64460D460120491C9142F3DB61
:104370003D60F0BD280210005A021000F00A100043
:1043800060A2012030B50268002513460AE000BF94
:1043900050F82540944201DD224602E09C4200DABA
:1043A00023466D1C8D42F3DBD01800EBD07040101B
:1043B00030BD30B57C4B1C68637D247D5B1C634342
:1043C00007E000BF32F8134030F81350641B21F8A7
:1043D00013405B1EF6D230BD70B5734B1C68247D54
:1043E000611A10E0012409E02D7D04FB0515641C11
:1043F00030F9156096FBF2F620F815601D686E7DA9
:10440000A642F1DA491C1C68247D8C42EADC70BDAE
:104410006649012008604FF47071654813F0E3BDF0
:104420002DE9F041064615460F46302801D1FFF729
:10443000EFFF5E4C20682844401CB0F5707F01D22D
:10444000206801E001202060594908700E542DB108
:104450000844401C2A46394613F046FD206828448B
:10446000401C2060BDE8F08170B54F48006890F8AE
:104470000513CA074F491DD090F8062302F00F021A
:10448000531C0A2B01D90A2200E0521C00F2073506
:1044900000234C8805E000BF35F81360B4420CD00F
:1044A0005B1C9342F8DBB0F84E274A80B0F8192322
:1044B0000A8002E0B0F84E274A80B0F85C07C88056
:1044C000088170BD03004FF0000006D00B785B1E22
:1044D00013F0FF030B7001D101200A70704730B553
:1044E00004460020034605E034F913508D4200DDF8
:1044F000401C5B1C9342F7DB30BD30B50446002006
:10450000034605E034F913508D4200DA401C5B1C71
:104510009342F7DB30BD30B5234B044600201B68C7
:10452000024693F8463703F00F03072B02D947F6EC
:10453000FF730DE05B1CC3EB03331BB208E000BF4D
:1045400034F912509D4200D00DB9401C80B2521C6B
:104550008A42F5DB30BD184818490078087070476A
:10456000012804D1154814490078401C0870704790
:10457000F0B50D4E3468657D247D6D1C65430FE0FC
:1045800037683F7D94FBF7FC07FB1C477FB2BA42BC
:1045900005DCBB4203DB30F8147021F81470641C96
:1045A000AC42EDDBF0BD0000280210002C02100030
:1045B000AC00012004251000DFFF010060021000A4
:1045C00010B501462022FC4813F0D3FCBDE8104092
:1045D0004FF400610120FBF75FBF70B59AB006464B
:1045E0000D4614466846FFF7F5FBF44800780128AD
:1045F00008D0F3480078072801D0062802D1684681
:1046000003F007FAE00702D00120ADF800006006D1
:1046100008D5EC4900200870BDF8000040F4806027
:10462000ADF80000200605D5BDF8000040F480502C
:10463000ADF80000600705D5BDF8000040F00600A9
:10464000ADF80000ADF81A60ADF83A50ADF834504E
:10465000AFF29300D84D03244FF4006602906846F1
:10466000FDF7B8F818AB002231460120FBF764FFD4
:1046700031460120FBF73FFF2878002804D0FEF7E1
:10468000AAF8641E002CEADC1AB070BD2DE9F041D6
:10469000CD4A0025294612682C46430504D592F8D8
:1046A0006D1240244FEA111110F4D17F05D092F819
:1046B0006D1244F004044FEA111110F0050F05D0FB
:1046C00092F86C3244F001044FEA1315C00604D589
:1046D00092F86C0244F0020405098D4200DA0D469E
:1046E0006D1C002C0AD00026B84F05E0F9887888A8
:1046F0002246FFF772FF761CAE42F7DBBDE8F08181
:104700002DE9F35FDFF8C0920D46D9F80000447D33
:10471000017D90F86C02641C00F00F074C437F1C75
:104720004FF48851AA4813F080FC0026DFF8A082DD
:10473000DFF898A2DFF880B21BE000BFBAF80610DD
:1047400001220098FFF749FFA249DBF8040003F0BB
:104750004FF8A04A0020414608E000BF51F8203041
:1047600032F910C0634441F82030401CA042F5DB10
:10477000761CBE42E2DBD9F800004B4690F86C0292
:1047800000F00F018E48491C0078072804D0062845
:1047900002D0002042462AE00020424607E000BF47
:1047A00052F8206096FBF1F625F81060401C1E6858
:1047B000367D06EB46068642F2D8D9F80030587DA1
:1047C0001B7D401E584306E052F8203093FBF1F366
:1047D00025F81030401CA042F6DBBDE8FC9F00BF6E
:1047E00052F8203093FBF1F325F81030401CA04222
:1047F000F6DBF2E72DE9FC47FEF76DFC0090FEF7D3
:10480000B7FC019004216846FEF775FB04460421BD
:1048100001A8FEF770FB6C4E204444003068A100F4
:1048200090F86D0200F00F077F1C694813F0FDFB44
:104830000025DFF884A1DFF89891B04621E06348B5
:104840004022C1884088FFF7C8FED8F80010DAF887
:10485000146091F89417C90705D032463046DAF84B
:10486000101002F008FD0020494607E051F8202012
:1048700036F910301A4441F82020401CA042F5DBE4
:104880006D1CBD42DBDBD8F80000514E454690F868
:104890006D024B4600F00F02521C002107E000BFE2
:1048A00053F8210090FBF2F026F81100491CA142B8
:1048B000F6DB49493046FEF714FC48493046FEF71E
:1048C00058FC28684FF0000690F8C10240061ED53B
:1048D00043480024068013E0407D42494200604383
:1048E00001EB40003C4913F0FFFA28683E49007D87
:1048F0004200604301EB4000384913F0F5FA641CB4
:10490000286890F8BE12C1F30111A142E4DC2868C6
:1049100090F86912890710D5344C2660417D2E48E5
:10492000FFF780F92168084420602868017D2B4842
:10493000FFF778F9216808442060BDE8FC872DE97D
:10494000FC47FEF7C8FB0090FEF712FC0190042123
:104950006846FEF7D0FA0446042101A8FEF7CBFA18
:10496000194E204444003068A10090F86D0200F018
:104970000F077F1C164813F058FB0025DFF838A0FE
:10498000DFF84C80B1463EE010488022C188408864
:10499000FFF723FED9F80010DAF8186091F89417A1
:1049A000C90705D032463046DAF8101002F063FC31
:1049B0000020414624E00000B84B10007B031000AB
:1049C000940210004102100028021000042510007B
:1049D000EC121000F00A10006C040120A804012061
:1049E0003202100008090120BC090120D403100084
:1049F00051F8202036F910301A4441F82020401C8C
:104A0000A042F5DB6D1CBD42BEDBD9F80000754D40
:104A1000434690F86D0200F00F00401C002106E0B4
:104A200053F8212092FBF0F225F81120491CA142F5
:104A3000F6DB6D492846FEF754FB6C492846FEF725
:104A400098FB6B490120087077E770B50446002099
:104A5000FBF713FE0320FBF710FE664D286890F865
:104A60006912C90701D124F4006490F8B811C9078C
:104A700001D124F0620490F80513490701D424F011
:104A8000040490F8CE1009B924F0100490F81A0428
:104A9000C00701D124F4805457490020401C8842AB
:104AA000FCD3200502D52046FFF7F0FDE00743D0F8
:104AB000524853494088FFF723FE286890F869025E
:104AC00080070AD54E48FEF7AAFF4E4901234E4AF9
:104AD000086001464A48FEF7D9FF28684B4A90F81B
:104AE0004C1051B14A490978962906D14849491CC8
:104AF0000978A52901D10021117090F84814CB073D
:104B00001AD01278C2B18A0713D490F8CC20520779
:104B10000FD490F8692412060BD490F87024120672
:104B200007D40A0605D4490603D490F85704C007F1
:104B300002D0204602F08BF8600501D5FFF75AFE3F
:104B4000E00401D5FFF7FBFE32490120087003F0B5
:104B500074FC0020FBF7ACFDBDE870400320FBF7C0
:104B6000A7BD2DE9F0412C4801242C4E04700025EE
:104B700035602B496006C1F8FC01C867294F052044
:104B800038724FF44870FBF793FB244844380560B3
:104B9000FF21397034600460B0E52049002030B452
:104BA000443908601F4908310A791D4B4FF00074E1
:104BB000FC331C60C2F1FB020978D2B2491CB2FB83
:104BC000F1F1134A14321170134A1070104A552033
:104BD0001232107014480170211330BC0120FBF711
:104BE0008ABC0000EC12100048B4012084B40120FB
:104BF0006C0210002802100020A1070004251000FC
:104C000060A2012078021000642410005F021000EE
:104C1000E0FF010040021000A6021000480500223B
:104C200084E000E02E000020A9021000F0B5FB494E
:104C300000204D68FA490A68537D117D5B1C01FB19
:104C400003F41CE035F91130002B02DC40F02000A9
:104C500014E040F6FF76B34202DB40F010000DE0B6
:104C6000B2F8B576B2F8446007EB060C9C4505DA5D
:104C7000BF1B9F4202DD0EB140F04000491C8C4238
:104C8000E0DCF0BD10B501462022E44813F071F9D4
:104C90008021BDE810400120FBF7FEBB30B599B084
:104CA00004466846FFF796F8012C07D10120ADF8BD
:104CB000000000208DF816008DF81400BDF80200E9
:104CC000AFF23F0140F48670D44D0291ADF802007E
:104CD00003246846FCF77EFD18AB002280210120EA
:104CE000FBF72AFC80210120FBF705FC287800282F
:104CF00004D0FDF770FD641E002CEADC19B030BD55
:104D00002DE9FF5F00200090FEF777FA0446FEF7DA
:104D10007AFA07464FEA540B4FF4F061C14813F09A
:104D200062F9BE484FF018098021203013F07DF958
:104D3000002002900120FFF7B1FFB848D0F804A08E
:104D4000B7480068047D01200025039091E0012010
:104D500000FA05F111EA0B0F6FD00026012000FACE
:104D600006F818EA070F77D0AC48203050F8250035
:104D700010EA080F6FD131462846FDF7DDFF01909C
:104D8000A7483AF914100368B3F8B526914256DCE7
:104D9000DFF890C23CF914C0BCEB0200A1EB0202A8
:104DA00000D54042002A00DA524290421FDC0198AE
:104DB0003146401EC0B2024601902846FEF78CFAEA
:104DC000984830F914103AF91400081A01D5C0F1C6
:104DD0000000009A104400909148006890F846271F
:104DE000007D02F00F0201FB021109B214E08D4AAE
:104DF000BCEB010000D54042DDF800C060440090EB
:104E000022F8141093F846173AF9140001F00F0134
:104E100000FB010001B2187D201A80B2FEF794FB5E
:104E20008149019821F814007C48203050F8251061
:104E300041EA080140F825100DE019E00CE0019866
:104E40003146401CC2B22846FEF746FA75483AF889
:104E5000141020F81410641C761C202EFFF67EAF70
:104E60006E48203050F82500B84201D00020039051
:104E70006D1C4D45FFF66BAF039838B9FCF761FF29
:104E80000298401C02904028FFF654AF64484FF04F
:104E9000010A00250068067D1DE0012000FA05F2E8
:104EA00012EA0B0F16D000240120A04038420ED089
:104EB0005D48214610F81600804602462846FEF757
:104EC0000BFAB8F13F0F01D34FF0000A761C641CB7
:104ED000202CE9DB6D1C4D45DFDBBAF1000F02D160
:104EE0000320FDF79BFCFCF72CFF0120FFF7D6FE0B
:104EF000FFF79CFE04464A480168087D4A7D91F808
:104F000046175043009A01F00F01B2FBF0F001FB8D
:104F1000000000B2FEF731FA04B02046BDE8F09F71
:104F20002DE9F05F3E4A116891F81007C4073F4829
:104F3000037803F0F00514D0057000264B7D0C7D3E
:104F4000DFF8D8A05B1CB046914604FB03F783460C
:104F50000120FFF7A3FE2046DAF80420D9F800105C
:104F60000DE091F8BF1601F00F0129430170D5E75C
:104F700032F91030B1F8B3C66345CFDB401C87422D
:104F8000F6DC0F2E0AD2761CF6B245EA060108F1CD
:104F900001088BF80010B8F1100FD9DBBDE8F05F05
:104FA0000220FDF73BBC70B501244FF404614FF4BF
:104FB000F83013F03AF8FCF7C4FEFFF7B1FFFFF743
:104FC0009FFE44EA0065164C18482268401D01788F
:104FD00092F8FB2701F0F00102F00F02114301707B
:104FE0001348FEF7D7FC284603F001FC206890F830
:104FF000A001C00702D0012000F00AFD206890F84F
:105000001A04C00704D0BDE87040022000F000BDC3
:10501000BDE87040422003F0EABB0000D84B10000E
:105020002802100080D3012000DB0120F6FF0100E0
:10503000EC231000024618215FF0010000FA01F392
:10504000134201D1491EF9D5491C884010437047CD
:105050002DE9F04F0020FF4D04460246FE49D5F8E9
:1050600014906E680B68012140F6FF7B01FA02F78D
:1050700037421BD039F914A0BAF1000F02DC40F01E
:10508000200012E0DA4502DB40F010000DE0B3F83A
:10509000B7E6B3F8C2760EEB0708D04503DBAEEBFC
:1050A000070CD44501DD40F04000641C521C202A4E
:1050B000DCD30024AF68D5F81860224601FA02F567
:1050C0003D421AD036F91450002D02DC40F0200089
:1050D00012E05D4502DB40F010000DE0B3F8C4863D
:1050E000B3F8BBC6C146E044A84503DBACEB090CF2
:1050F000AC4501DD40F04000641C521C202ADDD389
:10510000BDE8F08F10B501462022D44812F031FFDF
:105110008021BDE810400120FBF7BEB930B599B041
:1051200004466846FEF756FE2078012802D0022881
:1051300007D102E04FF4806001E04FF48050ADF8F9
:10514000000000208DF844008DF84300C1484168FC
:1051500049000B9180680C90BDF80200AFF25B0132
:1051600040F48670BD4D0291ADF8020003246846FC
:10517000FCF730FB18AB002280210120FBF7DCF9A3
:1051800080210120FBF7B7F92878002804D0FDF72B
:1051900022FB641E002CEADC19B030BD2DE9FE4F65
:1051A0000446AF480090DFF8BCB22121206A12F01B
:1051B0001AFF3021606A12F016FF2046FDF734F91D
:1051C0002046FCF72CFE0420019003253C2100988A
:1051D00012F009FF3C21584612F005FFDFF87482F7
:1051E000DFF874A24FF000092046FFF797FFE807A9
:1051F0003BD000200746064602900120D8F8041054
:10520000B04008422AD03046216AFEF797FBD8F812
:10521000141031F91720DAF80010B1F8C6168A42D6
:105220001BDA0121029101990844C1B23F2900D93A
:105230003F213046226AFEF794FBDAF80010D8F8D6
:10524000140091F8931730F9170001F00F0100FBDB
:10525000010001B2B8B2FEF785F97F1C761C202E42
:10526000CBD3029808B925F00105A8073BD500204B
:105270000746064602900120D8F80810B0400842C0
:105280002AD03046616AFEF759FBD8F8181031F978
:105290001720DAF80010B1F8C8168A421BDA01218B
:1052A000029101990844C1B23F2900D93F213046FB
:1052B000626AFEF756FBDAF80010D8F8180091F889
:1052C000931730F9170001F00F0100FB010001B244
:1052D000B8B2FEF743F97F1C761C202ECBD3029880
:1052E00008B925F002055DB12046FDF79DF820467E
:1052F000FCF795FD09F10109B9F1640FFFF674AFF0
:1053000003264FF000092046FFF708FFF00759D0A9
:1053100000200546074601900120D8F80410B84047
:10532000084248D03846216AFEF708FBD8F8141026
:10533000DAF800C031F91520BCF8C6369A4210DD03
:1053400078B101210191401EC1B23846226AFEF7B0
:1053500008FBD8F8140030F81510009820F8151044
:1053600028E0009931F91510C91AA2EB030300D502
:105370004942002B00DA5B42994211DC401CC1B269
:105380003846226AFEF7EDFADAF80010009891F834
:10539000931730F9150001F00F0100FB010005E043
:1053A0009CF8930700F00F0002FB002001B2A8B2A6
:1053B000FEF7D8F86D1C7F1C202FADD3019808B9DB
:1053C00026F00106B00761D500200546074601908A
:1053D0000120D8F80810B840084250D03846616A19
:1053E000FEF7ACFAD8F81810DAF800C031F9152039
:1053F000BCF8C8369A420FDD70B101210191401E00
:10540000C1B23846626AFEF7ACFAD8F8180030F834
:1054100015102BF8151031E03BF91510C91AA2EB45
:10542000030300D54942002B00DA5B4299421BDCA2
:10543000401CC1B23846626AFEF793FADAF80010EF
:105440003BF9150091F8931701F00F0100FB0100E3
:1054500010E00000D002100028021000784C10006C
:105460008C080120C80801209CF8930700F00F0069
:1054700002FB002001B2A8B2FEF770F86D1C7F1C81
:10548000202FA5D3019808B926F00206002E0BD0D4
:105490002046FCF7C9FF2046FCF7C1FC09F10109D1
:1054A000B9F1640FFFF62FAFBDE8FE8F2DE9F04193
:1054B00006460020F16908702121306A12F093FD40
:1054C0003021706A12F08FFD3046FCF7A8FC3046A0
:1054D000FCF7AAFFFE4D00273046FFF71FFED5E977
:1054E00004320024204605E032F91010A14200DD0C
:1054F0000C46401C9842F7DB0020EB68AA6905E0E7
:1055000032F91010A14200DD0C46401C9842F7DB36
:10551000002C0BDCF06901780F2904D8491C0170BC
:105520003046FCF781FF7F1C202FD5DB40F6FE7054
:10553000844208DDF1690878401E08703046BDE8F5
:10554000F041FCF771BFBDE8F0812DE9F0434168FF
:10555000DF4DD0F814C091F800808168D5F8047050
:1055600091F8009000210A460C46012303FA04F644
:105570003E4204D01CF804608E4200D93146641CBF
:10558000202CF3D38669D5F808C0002403FA04F769
:1055900017EA0C0F03D0375D974200D93A46641CD6
:1055A000202CF3D3C36801EB0804FF2619700369AC
:1055B0001A7002EB09039C420DD21B1B1944FF29F0
:1055C0001BD9C1680E70296841F08001296000690B
:1055D0000270BDE8F083A3420FD2E31A1A44FF2AF7
:1055E00002D803691A7005E0026916702A6842F051
:1055F00080022A60C0680170EBE7C3681970E6E7B3
:105600002DE9F041044600214569B148B14B012222
:105610004FEA010C476802FA01F63E420AD01F68C1
:105620006E5C97F8CB76BE4202D9F61B6E5401E051
:1056300005F801C0491C2029ECD3D4F818500021EA
:10564000876802FA01F63E420AD01F686E5C97F83E
:10565000CB76BE4202D9F61B6E5401E005F801C0BC
:10566000491C2029ECD32046FFF76FFF2046BDE8F8
:10567000F041FCF71BBC2DE9F14F2C210098D0E93B
:105680000565304612F0AFFC4021284612F0ABFC15
:105690000098FFF75AFF0098FCF7C6FE0098FCF749
:1056A00005FC03244FF0040A00270098FFF736FD9D
:1056B000A00750D086494FF0000C8946D1F814B0AD
:1056C000624660465FF00101D9F8048001FA00F3F8
:1056D00013EA080F10D07F4B3BF912801B68B3F818
:1056E000B936984507DA335C4FF0010C5344FF2B71
:1056F00000DDFF233354521C401C2028E4D3BCF1AE
:10570000000F01D124F001040023CE46D9F81890EF
:10571000DFF8C0C11A4618468B4600BFDEF8088085
:105720000BFA00F111EA080F0FD0DCF8008039F90C
:105730001210B8F8BD86414506DA295C01235144B0
:10574000FF2900DDFF212954521C401C2028E5D3ED
:105750000BB924F002045CB10098FFF7F6FE009844
:10576000FCF762FE0098FCF7A1FB7F1C642F9CDB1A
:10577000032400270098FFF7D1FCE00725D0544A06
:105780000023DFF850B1D2F814C0194618469146EC
:105790004FF0010AD9F804800AFA00F212EA080F61
:1057A0000DD0DBF800203CF91180B2F8B926904505
:1057B00004DD325C12B10123521E3254491C401CDC
:1057C0002028E7D30BB924F00104A00725D5404ACF
:1057D0000023DFF800B1D2F818C0194618469146E8
:1057E0004FF0010AD9F808800AFA00F212EA080F0D
:1057F0000DD0DBF800203CF91180B2F8BD269045B1
:1058000004DD2A5C12B10123521E2A54491C401C9B
:105810002028E7D30BB924F00204002C0BD0009809
:10582000FFF793FE0098FCF7FFFD0098FCF73EFBA6
:105830007F1C642F9EDBBDE8F88F70B4254B0021E0
:105840000C461E6896F8102792070BD5426896F80A
:10585000CA6601211578B54203D9A5EB0605157076
:1058600000E014701D6895F8102752070BD5826868
:1058700095F8CA5641F002011378AB4202D95B1B7E
:10588000137000E01470002901D070BC5DE670BC9C
:1058900070472DE9F0470F4E0446002530682F462B
:1058A00090F81017890703D560680125077008E094
:1058B0002178012901D0022903D1616890F8C0063E
:1058C0000870306890F8101749070AD504E0000006
:1058D000D002100028021000A06845F002050770F1
:1058E00008E02178012901D0022903D1A16890F8AC
:1058F000C1060870002D6FD02C21606912F073FB77
:105900004021A06912F06FFBE06921210770206A35
:1059100012F069FB3021606A12F065FBE168FF203C
:105920000870216908702046FCF7C0FA2046FCF791
:1059300076FA2046FCF778FD4FF01009DFF8D881A1
:10594000CA4600272046FFF7E9FBE80726D0D8E93A
:1059500004C30020014605E033F91120824200DD36
:105960001046491C6145F7DB3168B1F8B726824221
:1059700006DA61684FF001090878401E08700DE0F2
:10598000B1F8CC16814207DB616808784844FF28EB
:1059900000DDFF20087001E025F00105A8072AD5E9
:1059A00000200146D8F80CC0D8F8183006E000BF37
:1059B00033F91120824200DD1046491C6145F7DBB6
:1059C0003168B1F8BB26824207DAA0684FF0010ABD
:1059D0000178491E01700EE018E0B1F8CC16814242
:1059E00007DBA16808785044FF2800DDFF2008701D
:1059F00001E025F00205002D08D02046FFF7A5FDA7
:105A00002046FCF711FD7F1C202F9BDBBDE8F087B3
:105A1000F0B5424D8BB0012129708DF80000684629
:105A2000FDF7FAFB3C4C00262660FDF754FB606056
:105A3000FDF79EFBA0606068042140086060201DA7
:105A4000FDF759FA2061042104F10800FDF753FA2B
:105A5000E0606846FFF762FB9DF8001030480129BE
:105A600002D0022905D101E0406900E0806960614F
:105A7000A061D4E9040101EB40016161E16801EB3F
:105A80004000A16901EB4000A0616846FFF701FFFB
:105A90006846FFF7D2FE234F386890F8100780065B
:105AA00005D56846FFF7E7FD6846FFF7A9FD3868AA
:105AB00090F81007000702D56846FFF7F7FC386832
:105AC00090F81007C00602D56846FFF767FB6846E6
:105AD000FCF7AAFC6846FFF721FBFFF7B9FA21683B
:105AE0000143216010483A68037892F8FB2763F37A
:105AF000030202709DF80000012802D0022807D19D
:105B000002E041F00E0001E041F0020002F06FFE01
:105B10002E700BB0F0BD0000D00210005E0210002D
:105B2000784C100028021000FBFF010010B5014660
:105B30002022A34812F01DFA8021BDE81040012068
:105B4000FAF7AABCF0B59F4D06460C4628684FF000
:105B5000FF3199B090F8C30200F00F00401C814063
:105B6000CF436846FEF736F90120ADF80000ADF8E6
:105B70000240286800F2FB2001788DF8171044F0ED
:105B80000501ADF802100397ADF81A60AFF263019A
:105B9000029141788DF818108078894D8DF81E009B
:105BA00003246846FBF716FE18AB00228021012073
:105BB000FAF7C2FC80210120FAF79DFC2878002822
:105BC00004D0FCF708FE641E002CEADC19B0F0BD1E
:105BD0002DE9FC5FDFF8ECB14FF0000AD146DBF8AD
:105BE0000000564600F2FF20017890F8018080788E
:105BF00001904FF00850D0F88C0100B90126002028
:105C00008CB2009038E000BFDBF8000090F802038F
:105C100000EB80004700002524E020460099FFF7B4
:105C200091FF674840680BF0E6FC0146DBF8000096
:105C300090F8FA2212F00F0000D1012012094A4315
:105C4000B2FBF0F01FFA80F9012E09D1BAF5707F8E
:105C500006D25D4A0AF1010022F81A901FFA80FA72
:105C60006D1CADB2BD42D8D94A462146302002F063
:105C700001FE0198204484B24445C5DDBDE8FC9F87
:105C80002DE9FF5F4FF6FF764FF0000A93460F466F
:105C9000804634465546DFF82C911BE038F8150055
:105CA0005146FFF74FFF464840680BF0A4FCD9F877
:105CB000001091F8FA2212F00F0100D1012112090F
:105CC0004243B2FBF1F080B2A04202D238F8156034
:105CD00004466D1CBD42E1DBABF800600398048014
:105CE000BDE8FF9F2DE9F041364E054688463068F5
:105CF00088B090F8062302F00F01C2F30214491C89
:105D0000641C0A2900DD0A21022C00DD022400F2B5
:105D1000073006AB05AAFFF7B3FF326892F8050318
:105D200000061CD5BDF814600121ADF8006002F535
:105D3000477200204FF4803C6F4607E0135633440F
:105D4000634502D227F81130491C401CA042F5DB04
:105D5000002904DD06AB05AA3846FFF791FFBDF820
:105D600014002880BDF81810A8F8001008B0BDE88D
:105D7000F0817CB50020FAF780FC144C01A968463C
:105D80006588FFF7AFFF0F480068B0F81913BDF83A
:105D90000400814201D9218000E02080BDF800008C
:105DA00060800020FAF784FC094901200870094945
:105DB0000870BDF800202946092002F03EFD7CBD98
:105DC000984C10002802100000DB01200425100070
:105DD000400210009F021000FDF76CB910B5FDF7EE
:105DE0005BF94008400010BD7CB54FF4F83040F638
:105DF000FB7112F0F8F8FCF79FF8FCF766F8FBF778
:105E0000A0FFFF4C0020207020636063A063E0636C
:105E100020646064A064E06420656065A065E0655E
:105E20006060E06120626062A062E062FFF7D6FF1E
:105E30000090FDF73FF9019004216846FDF75BF8FB
:105E40000546042101A8FDF756F8014600EB450080
:105E5000C4E90305C4E905517CBD2DE9F0411746AD
:105E600004460D46002609E0E00703D031463846D7
:105E700002F01BFC761C6D084FEA340454EA05005E
:105E8000F2D1BDE8F08130B5034600204FF0FF327B
:105E90005FF0010505FA00F40C4202D0521C9A4250
:105EA00003D0401C2028F5D3002030BD70B50E462D
:105EB000012505FA06F2D24C12286DD2DFE800F077
:105EC0006C485109126C6C1B242D363F5A5E626C73
:105ED0006C6B3046216EFFF7D6FF8540606B054343
:105EE000656359E03046616EFFF7CDFF8540E06C99
:105EF0000543E56450E03046216EFFF7C4FF85405E
:105F0000A06B0543A56347E03046216EFFF7BBFF5A
:105F10008540E06B0543E5633EE03046616EFFF788
:105F2000B2FF8540606D0543656535E03046216E02
:105F3000FFF7A9FF8540206C054325642CE030461F
:105F4000616EFFF7A0FF8540A06D0543A56523E0C6
:105F50003046216EFFF797FF8540206B0543256390
:105F60001AE03046616EFFF78EFF8540A06C054356
:105F7000A56411E0606C024362640DE0E06D0243D1
:105F8000E26509E03046616EFFF77DFF8540206DD8
:105F90000543256500E025706068401C606070BDA9
:105FA00010B501462022974811F0E3FF8021BDE89B
:105FB00010400120FAF770BA2DE9F04789460546EE
:105FC0004FF0FF34FDF776F88D4F00231946BE6879
:105FD0004FF0010C0CFA01F2024200D0641CAC42FA
:105FE00006D1B9F1010F0AD020EA02030E462021A2
:105FF000491C2029EED31846BE60BDE8F087134641
:10600000F4E72DE9F047894605464FF0FF34FFF7E6
:10601000E5FE7B4F02460020BB6801464FF0010CB5
:106020000CFA01F6164200D0641CAC4206D1B9F15C
:10603000010F08D022EA06000B461E21491C1E292A
:10604000EED9BB60D9E73046F6E72DE9F0419EB0C6
:10605000054688466846FDF7BDFE18A8FCF70EFA0F
:10606000FFF7BCFE664E40083066FDF723F80024BB
:10607000654F7066012D30D0FFF7B0FE0B90FDF735
:1060800019F80C902020ADF800003968022D01F5B8
:106090005A7188788DF84200C8788DF845000878E4
:1060A0008DF8380048788DF83E008888ADF83400C7
:1060B0000889ADF83A00C888ADF836004889A1F5DE
:1060C0005A71ADF83C0053D0032D2CD0042D2FD0A5
:1060D000052D36D0062D3DD04AE00120ADF8000058
:1060E0000C20ADF81A001F208DF8180040208DF804
:1060F000170095208DF81E008DF81F403C20ADF84C
:106100001C0003984008306604987066386890F860
:106110004D078DF86C4040F003008DF8600018A822
:10612000FCF7C4F924E0FCF7C5FF01210C9003E063
:10613000FCF7C0FF00210C904046FFF762FF0B9078
:1061400016E0FFF74BFE0B9001214046FFF734FFAE
:106150000C900DE001F2613188788DF84200C8782A
:106160008DF8450008788DF8380048788DF83E00A5
:10617000BDF802008DF8144020F030008DF8164074
:1061800040F008008DF844408DF84340ADF802001F
:10619000AFF2F3101B4D032402906846FBF71AFB85
:1061A0001CAB002280210120FAF7C6F980210120D2
:1061B000FAF7A1F9287828B10020641E002CECDC45
:1061C0001EB05EE60120FBE72DE9FC5F0021012007
:1061D000FFF73BFF00B30B484768FDF70EF801904F
:1061E000FDF711F80090042101A8FCF784FE064693
:1061F00004216846FCF77FFE84460020054605E042
:10620000EC021000B84C100028021000DFF8F0B4C7
:10621000DFF8F0A4009059E000211120FFF746FEBE
:10622000BDE8FC9F4FF00008C1465C462846DBF8FD
:106230006410FFF728FE014601208840616D084286
:1062400043D1012432E000BF04FB0C52DAF8000015
:1062500037F9121090F86703B1EB001F25DA08F147
:106260000108B9F1000F00D1A146711E8C421CD16A
:10627000B8F1010F19D1ACF101018D4204D1611EB9
:106280000120FFF713FE0EE007EB4201B1F90220F7
:10629000B2EB001F05DB35B131F9021CB1EB001F79
:1062A00001DA002000E002208046641CB442CBDB0F
:1062B000A6EB0901414508D829460220FFF7F6FD63
:1062C00001200099A840084300906D1C6545A9DB9A
:1062D00001253AE04FF0000844462CE0DBF84C3052
:1062E000DBF8542000201A4311D0D9462046DBF8B1
:1062F0006410FFF7C8FD014601208840D9F854100A
:10630000084203D1D9F84C10084000D0012005FB09
:106310000C4137F91120DAF8001091F86713B2EB4D
:10632000011F07DA30B901200099A040084201D1CD
:1063300008F10108641C6445D0DBB8F1000F03D0FC
:10634000691E0120FFF7B2FD6D1CB542C2DB67E795
:106350002DE9F041EA4C00200546EB4FDFF8A4831D
:10636000E0611FE029460520FFF76FFEF0B161698B
:106370000120FE6800EB410C36F91C10D8F8000033
:1063800090F87703B1EB001F03D929460E20FFF7E1
:106390008DFD36F91C00E169884202DD36F91C00EA
:1063A000E0616D1CA0698542DCD36AE5BDE8F0417F
:1063B000002111207AE52DE9F04100210620FFF7A8
:1063C00044FE28B1D0480025CE4ECD4CC76813E01E
:1063D000BDE8F0410021112068E5206931682844BA
:1063E00037F9100091F86513B0EB011F03DD294662
:1063F0000A20FFF75BFD6D1C60698542EDDB00251F
:106400000EE0E0683168284437F9100091F866130F
:10641000B0EB011F03DD29460B20FFF747FD6D1C84
:10642000A0698542EDDB2CE52DE9F041B44C00205C
:10643000064660623EE031460420FFF706FE18B1D2
:10644000B1480025C76831E0BDE8F04100211120C6
:106450002CE500BFFCF72EFE01462846FFF713FD92
:10646000014601208840E16C08421ED1A549E06840
:106470002844096807EB400030F9040C91F87813C0
:10648000B0EB011F07D931460820FFF70FFD294661
:106490000920FFF70BFDE068616A284407EB400024
:1064A00030F9040C884200DD60626D1CA0698542F1
:1064B000D0D3761C60698642BDD3E2E42DE9F04179
:1064C0008F4C00200546904FDFF8388220621BE099
:1064D00029460320FFF7B9FDD0B1FE68B6F90210D6
:1064E000D8F8000090F87603B1EB001F03D92946D5
:1064F0000720FFF7DBFCB6F90200216A884202DDC3
:10650000B6F9020020626D1C60698542E0D3B8E4F0
:10651000BDE8F04100211120C8E42DE9F04100213F
:106520000220FFF792FD50B17748764E744CC76851
:10653000306890F86003000720D500251BE0BDE817
:10654000F04100211120B1E420693168284437F975
:10655000100091F87413B0EB011F03D929460320F2
:10656000FFF7A4FC2069A16A284437F9100088428B
:1065700000DDA0626D1C60698542E5DB306890F843
:106580006003C0061BD5002516E0E068316828448A
:1065900037F9100091F87513B0EB011F03D92946A4
:1065A0000420FFF783FCE068E16A284437F9100013
:1065B000884200DDE0626D1CA0698542E5DB60E495
:1065C0002DE9F0410020FAF758F8FFF70DFC4D4C8B
:1065D000206890F86003010701D4C00601D5FFF7D9
:1065E0009CFF206890F86003800601D5FFF766FFE6
:1065F000206890F86003000601D5FFF715FF2068BA
:1066000090F86003C00701D0FFF7D5FE206890F82E
:106610006003400601D5FFF79BFE206890F86003F9
:10662000800701D5FFF7D0FD354C606800285AD0AF
:10663000D4E90D359D43A563206BD4E91216984328
:10664000A8432063276DB143B943A164616CE26D37
:106650009943A943E56BB243A9436164616DBA43B1
:106660008A43AB436363E26501220021FFF7F5FB38
:1066700002220021A06CFFF7F0FB03220021606BD7
:10668000FFF7EBFB04220021E06CFFF7E6FB07229B
:106690000021A06BFFF7E1FB08220021E06BFFF770
:1066A000DCFB09220021606DFFF7D7FB0A220021E5
:1066B000206CFFF7D2FB0B220021A06DFFF7CDFB72
:1066C0000C220021606CFFF7C8FB0D220021E06D59
:1066D000FFF7C3FB0E220021206DFFF7BEFB2078E1
:1066E000012803D006E00021084601E00021112026
:1066F00001F0DBFFBDE8F0410020F9F7D9BF000051
:10670000EC02100028021000B84C10002DE9F84FE0
:10671000DFF81CA401004FF00004DAF80000457D0A
:10672000027DB0F84B3490F85D6490F85C74B0F87A
:10673000499405FB02F59B46FE4800EB420080466B
:1067400001D1002637462A461946FDF7C8FE0090BB
:106750002A4649464046FDF7D0FE81462946404636
:10676000FDF7D9FEDAF800300246002193F857C44D
:10677000F1485546B2EB5C0F0AD94278521CD2B2AE
:106780004270B24205D9417001700120BDE8F88F16
:106790004170009A4A452EDD0278BA4203D202F1D6
:1067A000010202702FE00170417093F84804400725
:1067B00014D5E248FDF77BFA040010D1286890F860
:1067C0004814C9060BD5DD49B0F86704096888424A
:1067D00005D95846FCF7C6FA044600E001242868AB
:1067E00090F84804800608D5FDF70CF808B101249C
:1067F00005E0002407E0017005E0012C03D1FDF75E
:1068000027FA0128F5D02046C0E72DE9F84FC84CFB
:10681000C84B002521682E46AA460A7D03EB420B91
:1068200091F8703403F07F0800B9A8464F7D5846B0
:106830005743394607F046FB81463946584607F02C
:106840002EFB00902068017DBD4807F03BFB07460A
:106850002068417DBB4807F035FB01463846FCF710
:1068600065FB07B22068017DB54807F018FB834639
:106870002068417DB34807F012FB01465846FCF7FB
:106880004DFB216802B2B1F871344B4509DDB1F816
:1068900073340098834204DAB1F87504B84200DA20
:1068A0000126B1F87704B84208DDB1F879049042C6
:1068B00004DAB1F87B14494500DA012500229E482C
:1068C000012E04D0012D02D0027150465EE70179FD
:1068D000414502D2491C0171F7E702714FF0010AEC
:1068E000F3E72DE9F04F002287B09146009216465B
:1068F00093469246019200208D4A02909248D2F827
:1069000000C0410C04469CF8B9210D46120705D57C
:10691000BCF9D2118D4807F0C4FF31E09CF8153066
:106920000222059323E00123571E3FB204979CF8EF
:1069300014700397A7F1010E15E0039FDFF80C8296
:1069400002FB073738F917708F4208DCDDF810803A
:10695000CDF800800FFA83F83946CDF804808742DD
:1069600000DB38465B1C9E45E7DC059B521C9342CE
:10697000D9DC401ABCF8D21100B2814201DA012000
:10698000824601217248FCF7C3FC69480168087D12
:1069900000EB40026E4800EB8200827B037C1A44CD
:1069A0005208C273087D4A7D0392A2F101020123BD
:1069B000049221E00122A0F1010E19E003FB002C5A
:1069C000634F17F80C8067447F78B8EB070701D452
:1069D000BC4601E0C7F1000C91F8548408F00308AC
:1069E000C44504DD761C002F00DA7F42B944521CF6
:1069F0009645E3DC049A5B1C9A42DBDCBAF1010F9A
:106A00003CD1039F03467F1C4743DFF8288109E000
:106A100038F913209344A24200DD1446AA4200DA5A
:106A200015465B1CBB42F3DB039A42439BFBF2F02F
:106A300091F8B92100B21207002A91F85424C2F348
:106A400083020CDAB24219DA91F855244A4515DA74
:106A5000211A401B814211DAFCF7D4FE0DE0B2424C
:106A600003DA91F855244A4503DB211A401B814281
:106A700004DADDE90001FCF716FD0290029807B088
:106A8000BDE8F08F70B52A490025096891F8564491
:106A900000B90024FFF725FF020027494FF000004E
:106AA00008D0CA78A24202D2521CCA7003E0C87051
:106AB000012500E0C870284670BD2DE9F0410300B3
:106AC0001B484FF000070068427D047D90F8535446
:106AD000B0F84B14174802FB04F200EB440000D15D
:106AE0000025FDF7FCFC0026134C00280BDDFDF70C
:106AF000C6F840B1A078A84202D2401CA07003E0C2
:106B0000A670012700E0A6703846BDE8F0812DE9A7
:106B1000F041074E0746002530680E4C90F84804B7
:106B2000400604D50120FFF7C8FF012853D013E029
:106B300028021000F00A1000540310007C0210001C
:106B40004C080120100801200080FFFF60A20120F6
:106B5000E0A901205F021000EFB9306890F8480406
:106B6000000604D50120FFF78DFF012832D03068E0
:106B700090F87004000604D50120FFF746FE0128B6
:106B80002BD0306890F84804800704D50120FFF727
:106B9000BDFD012823D02078D0B16F4840F6050212
:106BA0000168114301606D48016841F400610160B2
:106BB0004FF480610120F9F76FFC306890F8100104
:106BC000C00604D54FF400710520F9F765FC0125D6
:106BD00028469AE703202070DFE70420FBE7022025
:106BE000F9E770B55E49002209684C7D0B7D651C94
:106BF0005D43194604E000BF30F91160491C32447E
:106C0000A942F9DB5C4392FBF4F000B270BD10B511
:106C1000534C544A2068417D007D414302EB4000C3
:106C2000FDF779FC2168002291F857344E49B0EB0A
:106C3000530F09D94878401C10F0FF00487004D069
:106C40004A700A70012010BD4A70002010BD2DE965
:106C5000F047464F0026B14638783546002873D0B5
:106C6000022801D003280DD101214148FCF750FB37
:106C70004048FCF760FDFCF784FB81463C48FCF78C
:106C800076FC06B2DFF8F08000243978002007296E
:106C900019D2DFE801F0180D071115180400FFF7ED
:106CA000B6FF10E00020FFF731FD01280CD01EE0F8
:106CB0000020FFF702FF06E00020FFF7E3FE02E0FE
:106CC0000020FFF7A2FD90B10125FDF744FCFEF77F
:106CD0006AF9B8F802002949FDF712FDFDF78AFDAF
:106CE000641C032CD1DB0020FBF798FD2AE0C120B7
:106CF00040EA052001F07BFD012D23D138780228E0
:106D000001D0032819D101211D48FCF701FB1C48C3
:106D1000FCF72DFC124900B2096891F88014314447
:106D200081420ADD00211248FCF7F2FA1148FCF713
:106D300014FD4846FCF721FB04E00020FDF710FCA1
:106D40000FF01AFD00203870BDE8F0474FF4F061F5
:106D5000084811F048B90000340210003802100051
:106D600028021000F00A1000540310005F02100007
:106D7000E0A901200A6410000425100060A201208F
:106D8000AC00012008B55B4E0127DFF86C815B4D3C
:106D90000024307868B10128FBD16B4600224EF206
:106DA0007D71F9F7C9FB0098C10717D03470012134
:106DB00091E001210020FCF727FA6B460022022116
:106DC0000120F9F7B9FB01210846FCF71DFA0098EC
:106DD0008007DED537704EF27F717CE0010716D553
:106DE0000020F9F74AFC0620F9F747FCFDF7B3FB52
:106DF000FEF7D9F8424843494088FDF781FC062058
:106E0000F9F756FC0020F9F753FC082163E0010470
:106E100004D50FF0B1FC4FF400415CE0C10606D58B
:106E20003948007808B9FEF7A4FF102153E0810625
:106E300001D520214FE0C10504D5FEF7C9FE4FF46E
:106E4000807148E0810502D54FF4007143E04106AE
:106E500003D5FFF7B5FB40213DE041053FD52B4869
:106E600004602B48D0F8009004604846FDF7EDFD23
:106E7000D8F80000C10501D526490F70A9F5B85210
:106E8000B73A05D1052001F0B2FCC8F800401FE078
:106E90005FEAC97106D040F0150001F0A8FCC8F8FF
:106EA000004016E019F0420F03D0286840F00600B9
:106EB0000CE05FEA495003D5286840F4806005E0A3
:106EC0005FEAC94005D5286840F4805001F08FFC86
:106ED0002C604FF480610120F9F70DFB59E7800425
:106EE000FCD5FDF73EFE00224FF400510120FBF7D8
:106EF000C5FE4EE759031000380210003C02100096
:106F00000425100060A201204E021000840310002E
:106F100034021000500210000E4900204860086042
:106F20000D49087070470D4810B5006890F8B6001C
:106F3000C0070DD00A480B4900780978084307D1EB
:106F40000320F9F79AFBBDE810400320F9F7B0BB26
:106F500010BD00005C0310009E021000280210000B
:106F6000470210004E021000F0B40C46014604988F
:106F7000C3F11006012801D0002014E02046F0BC27
:106F8000520010F0B1BF00BF34F9105031F9107049
:106F90005D4307FB0655EF1705EB177545F30F1516
:106FA00024F81050401C9042EEDBF0BC7047F0B467
:106FB0000C460146DDE90460F51A012801D00020E5
:106FC00010E02046F0BC520010F08EBF34F9107073
:106FD00031F910C05F430CFB057797FBF6F724F8F7
:106FE0001070401C9042F1DBDFE770B5534C246811
:106FF00094F8F04724074FF000040ED418E000BFC7
:1070000032F8145030F81460AD1B31F914602DB211
:10701000AE4201DA21F81450641C9C42F0DB70BDD2
:1070200032F8145030F81460AD1B21F81450641C71
:107030009C42F5DB70BD10B5044647F6FF70002298
:1070400006E000BF34F91230834200DA1846521CC1
:107050008A42F7DB10BD10B504463948002205E02E
:1070600034F91230834200DD1846521C8A42F7DBA5
:1070700010BD30B5044630F911300020491C06E03F
:1070800034F911509D4201DD2B460846491C9142BE
:10709000F6DB30BD2DE9F043284CDDE90797246885
:1070A00094F8906100242546012F01D0002637E096
:1070B0000023761E18E000BF31F9137030F913C0B9
:1070C00007EB0208C44505DDBCEB070700D57F428E
:1070D0003D4408E0A7EB0208C44504DABCEB07070F
:1070E00000D57F423C445B1CB342E5D31AE000BFAD
:1070F00031F9167030F916C007EB0208C44505DDFA
:10710000BCEB070700D57F423D4408E0A7EB02082F
:10711000C44504DABCEB070700D57F423C44761C2B
:107120009E42E5DBB9F1000F00D10024AC4202D24F
:107130000120BDE8F0830020FBE7000028021000DA
:107140000080FFFF3C483D4A0068516841400AD03A
:1071500050603B48006890F81001C00603D54021FC
:107160000520F9F799B97047704710B533480021E9
:10717000344C017034492068084210D00620F9F7D9
:107180007CFA0620F9F794FA30480078022802D1F8
:107190002068002803DABDE81040FFF7C4BE10BD28
:1071A000264900204860FFF7B7BE244C08B50025EB
:1071B0006570FFF7F5FF4FF6FF76607820B3012882
:1071C000FBD16B46002255210420F9F7B5F9009850
:1071D000C00706D0FFF7E4FF657031460420F9F7D9
:1071E0008AF90098400705D5FFF7BFFF042108463C
:1071F000F9F781F90098C006DFD5FFF7A3FF10214A
:107200000420F9F778F9D8E704210020FBF7FCFF08
:107210006B46002202210420F9F78EF90421012097
:10722000FBF7F2FF00988007C7D5FFF7B9FF0120F1
:1072300060703146E4E70000D404100064031000DD
:10724000280210008002100010000080940210003C
:10725000F748002141718171C171C170017170479E
:10726000F34901208870F3E7F14800218160417003
:107270000121817070472DE9FC4715468946064675
:10728000FBF729FF0090FBF773FF0190042168468C
:10729000FBF731FE0446042101A8FBF72CFE014652
:1072A000304606EB440305EB4407002208E000BF2C
:1072B00030F802CB33F8028B521CC44427F802CBBF
:1072C000A242F5DB01EB440206EB840006EB42032D
:1072D00005EB4206002207E030F8027B33F802CBD0
:1072E000521C674426F8027B8A42F5DB4846294651
:1072F000002204E030F8023B21F8023B521CA2427B
:10730000F8DB09EB440005EB8402002105E000BF37
:1073100030F8023B22F8023B491CA142F8DBBDE8F1
:10732000FC87C44910B5096800200A0712D5C24875
:10733000C24A006890F89407C307906906D04900D4
:1073400004D41169BE4AFFF796FF02E0BC49FCF77E
:10735000F0FC012010BD2DE9FC5FB74DB44C0127B6
:10736000286821784FF00008B0F8A16159B9A278D7
:107370008021CDE90012427D7F23B249B248FFF758
:1073800016FE84F80280B1480078062805D0072848
:1073900002D0A7480078B8B3BCE02868AA4AB0F881
:1073A0001611407D0EB2CDE900603346A549104666
:1073B000FCF7C2FE2868324690F8FE1001F0030187
:1073C0000091437D9F49A048FCF700FE002701285B
:1073D00004D0C4F8088084F800809BE0207800285E
:1073E00011D1A068401CA060296891F81511814254
:1073F00009D2012060702070074600F0FCFA0121DC
:107400000220F9F749F885E0FFE72C68A84694F8D0
:10741000A00100904007002894F8B8014FEA0070DE
:107420000BDA002801DA8A4D00E0874D607DAD1C43
:10743000801EDFF82092C0B209E0002801DA844DF6
:1074400000E0814DDFF80C92607DA9F102098246CF
:10745000814890F800B0BBF1010F01D1B4F8826609
:107460003C217B4810F0BFFD94F8B80100073ED5E1
:107470007A49B4F9D631B4F9D8010978012905D18E
:1074800094F85A12CA18084413B200B294F8BA1108
:107490006F4A49070029617DCDE900016D496A48BD
:1074A000A1F1020102DAFCF7B2FE01E0FCF744FEB2
:1074B000D8F8000090F8A011090702D566490978AC
:1074C00051B190F8FE006349C0F38100009053462B
:1074D00032B2891E5E4819E090F8FE005D49C0F3A3
:1074E00081000090534632B2891E59481EE0009830
:1074F000000702D5BBF1000F0FD094F8FE005346F1
:10750000C0F38100009032B249462846FCF75EFD88
:10751000474908703846BDE8FC9F94F8FE00534682
:10752000C0F38100009032B249462846FCF766FD60
:10753000EEE7404910B5096800204A071CD53E48CF
:107540003E4A006890F89407C307506906D0490086
:1075500004D41169424AFFF78EFE02E04049FCF76D
:10756000E8FB39493E48FBF7BCFD3E493C48FBF788
:10757000B8FDBDE81040EEE610BD2DE9FC418446A3
:1075800032482D49012600780968062808D00728C6
:1075900006D0B1F82021304B1B78012B03D004E03A
:1075A000B1F82321F7E7B1F8AE26062816D02E4F02
:1075B0002E4D1F4C022813D091F8FD0012B2C0F3DB
:1075C00001100090087D497D00FB01F307EB4001AD
:1075D0000CEB4000FCF7FAFC20701FE0002623E0D3
:1075E00091F88106C00718D0012B16D12078A0B9D8
:1075F00091F8FD3091F88706C3F38103CDE900309F
:10760000087D497D12B200FB01F307EB4001184FE2
:1076100007EB4000FCF71DFD20702078012803D106
:10762000286840F0010028603046BDE8FC81000079
:107630006C0310009003100028021000D04D1000C1
:1076400058B20120980701205C0701209402100025
:10765000D40701206E04012062021000F70310001D
:10766000640601201008012060A20120C002100061
:1076700080D301202DE9F041C44D0E460346296810
:107680001446DFF810C34F7D087D07F1010702465D
:1076900007FB04F700FB07F0BD4F274417F8017CF8
:1076A0008CF8037091F824100F0702D5C90600D595
:1076B000104442001946304610F016FC2868017D3F
:1076C000407D401C641E6043414306EB4100BDE821
:1076D000F0812DE9F047AD4E814688463068174667
:1076E000447D017D90F8240004F1010404FB01F4C1
:1076F000020702D5C00600D50C4401250AE0306817
:107700004946007D420004FB05F008EB400010F004
:10771000EBFB6D1CBD42F2D3BDE8F0872DE9F84FBD
:10772000DFF8689280460646D9F80000DFF864A2C8
:107730000F46447D007D641C44439AF80610504671
:107740008AF8071000254FF0010B4CE08279924B2C
:1077500002FB04F103EB410605FB04F108EB4101D8
:1077600000910BFA02F1C27811438AF803103146F6
:107770000098FCF7FAFAD9F8001091F824000207F3
:107780001ED5C0061CD5781E854208D1087D420052
:10779000009800EB440106EB440010F0A5FB9AF8BA
:1077A000060068B9D9F80000017D90F849004A0048
:1077B00000097949604301EB4000314610F094FB29
:1077C0009AF806105046491CC9B28AF80610D9F832
:1077D000002092F84920B1EB121F03D300218171E0
:1077E0008AF805B06D1CBD42B0D33046BDE8F88FB5
:1077F00070B5064669480C460078072801D006286F
:1078000005D167480078012801D0084670BD654859
:10781000654D00682A7FC30405D511463046FFF741
:107820007DFF044610E080040AD55B493046FFF72F
:1078300021FF04462A7F58493046FFF74AFF03E0FC
:1078400001223046FFF716FF204670BD70B5534841
:1078500000240078042801D0FFF7FAFC514E524D65
:107860003078C00706D051496868FFF7C1FFFFF7BD
:1078700084FE0446308840040DD544480068017DEC
:1078800090F8060300F00F00401C41434A004848AE
:10789000A96810F029FB204670BD70B53B4C4548E7
:1078A0002168057891F8C810CA072DD08A072BD512
:1078B000414A1678C1F38202012101FA02F216420E
:1078C0003E4B4FF0000202D01970017001E01A70B7
:1078D00002703B490978012900D11A70007885426D
:1078E00012D001280ED0CD2000F081FF206890F842
:1078F0001001C00608D5BDE870404FF48071052026
:10790000F8F7CABDCC20EFE770BD70B5FFF7C5FF33
:107910002548244C007820B1FAF75DFF0020206054
:1079200070BD1E4D28780128F8D00620F8F7A5FE76
:10793000FFF78CFFFFF7FDFDFFF7F3FC0620F8F7DC
:10794000B7FE2048216801602878022806D0072861
:1079500011D006280FD0022804D00FE00D4800787F
:10796000012803D0002909DB082108E000F043F8D2
:107970000121022004E04FF4007100E00421032003
:10798000F8F78AFDCAE700207047000028021000BF
:10799000408301006C03100040B5012094021000E8
:1079A0007B03100090031000D04D1000F00A10006F
:1079B00064050120570210004B0000205602100001
:1079C0005802100080021000F74B10B51878F74CE1
:1079D00000F08002A4F124000179645C14431C705F
:1079E000491CC9B20171042901D10021017110BDE6
:1079F00080B2F9F7CCB8F9F7F0B810B501462022FB
:107A0000EB4810F0B6FA0221BDE810400846F8F73E
:107A100043BD0121C1607047F0B599B00446684686
:107A2000FCF7D8F9E149E3482439E34B8C6102883B
:107A30001A80E24AE24BE34D52880280E00774D09C
:107A4000487A042802D01878042856D0DE480078F6
:107A5000012852D0187803284FD0BDF8000040F01C
:107A6000010000BFADF800002A6892F8C002C0070C
:107A70000FD092F8060300F00F00401C042808D82D
:107A8000BDF8000040F40070ADF8000044F4804000
:107A9000886192F84800C0070ED0187807280BD0EC
:107AA000062809D0BDF8020020F48060ADF802007D
:107AB000886940F40050886192F82400060707D5D1
:107AC000C00605D5BDF8000040F48070ADF8000098
:107AD00092F87200BD4F5FEAC07C4FF0010604D0FF
:107AE00097F800C0BCF1000F0CD092F81BC15FEA00
:107AF000CC7C2AD0C00731D027E0BDF8000040F48C
:107B00008040AFE71878042852D0002C50DB563262
:107B1000907F8DF81700507F8DF81E00D07F8DF874
:107B2000220012F80E0C563A33E016E08DF85C6035
:107B3000886920F4005088612DE0886940F48060F5
:107B400002E0886940F480508861C878012839D003
:107B50001878072833D0062831D033E03878002849
:107B6000F3D11878072803D0062801D002281FD1A6
:107B7000002C1DDB02F1FF02907F8DF81700507F73
:107B80008DF81E00D07F8DF8220012F8B70CA2F1FC
:107B9000FF02C007CAD192F824000207CDD5C00663
:107BA000CBD5BDF8000020F48070ADF80000C4E72C
:107BB00092F848004007C8D5002CC2DAC5E76846ED
:107BC000FFF727FF600711D51878022806D0032891
:107BD00006D0042804D0062808D113E0002C1EDAB1
:107BE000BDF8000040F48060ADF80000200728D503
:107BF0001878022818D0032818D0042816D0062890
:107C00001FD111E0296891F81A0108B18DF84200DE
:107C100091F8220100F00F008DF84400DEE7BDF876
:107C2000000040F40060DFE7002C04DABDF800003B
:107C300040F4805003E0BDF8000040F40050ADF87F
:107C40000000AFF2492002906846F9F7C3FD19B071
:107C5000F0BD38B5002469460620F8F75CFC0098B2
:107C600018B9F9F7AEF8002800DD0124204638BD28
:107C7000534810B503784D4952482439022B8A796C
:107C8000006813D0062B1BD0072B1CD0012A1DD057
:107C9000022A1ED090F83D4090F82520120727D5E3
:107CA0004A7A042A1BD0042B16D018E090F84140E1
:107CB000022AF1D190F83F20A242EDDD1446EBE715
:107CC00090F81341E8E790F81441E5E790F83E405A
:107CD000E2E790F83F40DFE790F843200A7291F91D
:107CE0000820002A02DD521E0A7201E090F842408C
:107CF0004B7204B91424FFF7ACFF012800D16400D3
:107D0000204610BD30B52F49054600200A6892F87C
:107D1000B610C90729D02A490B7824492439022BE7
:107D200024D0072B22D0062B20D092F8BD30284C2F
:107D300024781CB192F84844A4074FD5CC68641C41
:107D4000CC609C4211DD0020C86092F8B81105F0AB
:107D50000100C90701D040F0040092F81A14C907C5
:107D600001D040F0080040F0004030BD194C2478AC
:107D7000012C10D0072B10D0062B0ED0164B1B78E1
:107D8000012B0DD092F8BE300C78032CCFD2641C9E
:107D90000C70CB60CBE71023F6E792F8BF30F3E727
:107DA00092F87F36F0E70000200000209C031000CE
:107DB000D04D1000A4021000A202100004251000F3
:107DC00094021000280210004E0210005A02100007
:107DD0004702100042021000620210005A42CA60BC
:107DE00030BD02460020F84B0146062A02D0072A81
:107DF00009D00BE0F5480278012A03D0062018705C
:107E0000042003E00170072018700120F04A11706F
:107E1000F04A1170F0490969084070472DE9F04FA8
:107E2000EE49002504460B78ED49A94628460E7810
:107E3000022C01D100231E46E749DFF8A8B3DFF882
:107E400094E30A69DFF880839246D7074FF0000277
:107E50000AD0E54F012E0ED06BB93B78012B0AD02A
:107E6000E24B1B78012B06D0042C0BD0E04B032CEB
:107E70001B680AD041E03A700420CA6188F800000B
:107E80000F204FE00A62CA613CE0DA4E3678012EDC
:107E90000ED0D94E3678012E0AD09BF80060012E04
:107EA00006D0D64F93F810613F78F60708D101E06D
:107EB0000A6222E093F8816676071ED5012F1CD155
:107EC000CE79012E19D193F881C693F912615FEA38
:107ED0004C7C03D5012F01D193F9B2660F6A06EBF2
:107EE00086067F1C0F62B7EB460F06D3C44D0A62AD
:107EF0008EF800200120287009E0032C02D0022C0B
:107F000005D00FE0032088F800001F200AE00220BF
:107F100088F8000093F810010125000601D51E2005
:107F200000E0132098F80030A34201D08BF8002025
:107F3000A74B00EA0A00002D1D708EF8009000D1BA
:107F40000A70BDE8F08F2DE9F041A94F9E4E012443
:107F5000386890F81001C106307800D504469E4D6F
:107F600000210428696108D0032806D0022804D023
:107F7000062805D0072803D007E0FFF74FFF01E0F0
:107F8000FFF72FFF6969084368612869FFF7BAFEA8
:107F9000696908436861307884420AD0386890F88B
:107FA0001001C00605D5BDE8F04140210520F8F7D5
:107FB00073BABDE8F0812DE9FC418D4E306890F830
:107FC0002400000601D5FFF7FFFCFFF7BCFF8D4939
:107FD0000868002809DD814A127832B9401E08601D
:107FE00003D102210620F8F757FAFFF741FE804639
:107FF000FFF7FEFC784C40F217216069084259D027
:108000000020F8F73AFB6069FFF706FD02216B4696
:1080100000220846F8F790FA02210846F8F76BFAB2
:1080200069480078022803D0042801D0032835D1FC
:108030000DF00DFF90BB01A90520F8F76CFA01982F
:1080400060B307270024704D01E0052C0CD005EB30
:1080500084012046F8F75FFA55F8240020B1022C7D
:108060001CD1A868012819D1641C64B2BC42ECDBA5
:10807000F8F7B3FD4FF480410520F8F70DFA4FF4FF
:1080800000546B46002221460220F8F755FA21469B
:108090000220F8F730FA4046FFF7AAFC306890F863
:1080A0002400000601D5FFF78FFCFFF72EFC00200F
:1080B000F8F7FEFABDE8FC8110B501210220F8F7BF
:1080C0001AFABDE8104076E73F480178022901D14D
:1080D0000321017040490020C8714FF480610220E3
:1080E000F8F709BA3C490120C871C1020220F8F72B
:1080F00002BA354810B50178012913D00621017064
:10810000FFF7B2F834490020C861086230490870AE
:108110003748006890F81001C00603D540210520BB
:10812000F8F7BAF94021BDE810400220F8F7E3B9AA
:1081300029490020354A486188611060C861086299
:10814000C86023490870234908702849087070479F
:108150002DE9F041002604210220F8F7CCF92C4843
:108160001D4D04682869014660401DD020424FF62D
:10817000FF7707D031B9012639460220F8F7BBF95D
:10818000FFF7D6FF20002C610F4C0ED00321012EEB
:1081900015D02078022807D100200D4A2862E86116
:1081A00010700C4A1070217003E7F8F716FD0120DB
:1081B00020703946BDE8F0410220F8F79CB9C007AD
:1081C00028D00420207026E0940210006D031000D7
:1081D0004102100042021000780310004702100014
:1081E0004A0210009E0210004D0210006C031000A5
:1081F000280210008702100088021000620210009E
:108200006E031000D0041000F04D1000800210002A
:10821000D40410002170BDE8F041CCE670B50446EE
:108220008F48006890F81001C00603D54021052052
:10823000F8F732F98B4D200705D50020A8710821E9
:108240000220F8F758F9E00605D50120A8711021A1
:108250000220F8F750F9E00406D50220A871BDE825
:108260007040C102F8F747B970BD10B5F8F7B5FC1A
:108270007D49012008707B4900204871BDE810400D
:108280004FF6FF710220F8F736B938B5744C43F257
:108290005D11206890F81001C00601D543F65D51CC
:1082A0006B4600220220F8F747F90098400804D0F6
:1082B000022269465520FCF7B3F80098C00501D5A5
:1082C000FFF7D3FF009841F21801084201D0FFF7F1
:1082D000A5FF0098400701D5FFF73AFF0098400638
:1082E00022D56048002141705F490978072919D1DA
:1082F000216891F81011CA064FEA017108D58078FB
:10830000002902DB02280DD007E003280AD004E090
:10831000002907DA8078012804D040210220F8F7EC
:10832000EAF801E0FFF7E5FE206890F81001C006CA
:1083300009D50098000501D5FFF7D4FE0098400547
:1083400001D5FFF7C1FE0098C00701D0FFF7B4FECA
:1083500038BD46480078434910F01F0001F1240160
:1083600008D007280CD0421E0A704870421C8A7040
:10837000C870704700200870012048700222F6E79C
:1083800005200870062048700722F0E7364810B52F
:108390000122027033480021354B01618171416136
:1083A0008161C161016219703249334B498819807A
:1083B000324B1980C271FF2101724272FFF7C9FF6F
:1083C000FEF74EFFBDE8104050212D480FF02DBEA6
:1083D00008B502210020FAF717FF6B4600224FF480
:1083E00000710220F8F7A8F802210120FAF70CFF2B
:1083F000022269465620FCF713F80098800509D53B
:10840000FFF7C4FF1749012048714FF6FF710220A2
:10841000F8F771F808BD1349002048717047114CF6
:108420000020607106E0607920B10128FBD1FFF7E0
:108430002CFFF8E7FFF7CCFFF5E70A490020C861F9
:1084400008621049087010490870704710B5F8F7B5
:10845000C4FB0121BDE810400220F8F71DB8000060
:108460002802100078031000940210002000002061
:108470009F02100004251000A2021000A4021000A8
:108480005C000120410210004202100010B50446B9
:108490000220F8F7F2F82046F8F79CFCBDE81040FF
:1084A0000220F8F705B9F8F795BC1CB5002100913A
:1084B000019102789DF8001062F303018DF800101D
:1084C000427862F307118DF800104289BDF801105F
:1084D00062F30B01ADF801100289BDF8021062F3DE
:1084E0000F11ADF8021081798DF80410C1798DF863
:1084F00005100179CA099DF8061062F3C7118DF8BD
:108500000610027962F306018DF8061080788DF866
:1085100007006846FFF7BAFF1CBD1CB5002000909D
:108520000190EA4800684178827810208DF80000B8
:108530004006437A8DF80130E54B1B788DF8023008
:1085400043891B0A8DF8033040898DF80400E14807
:108550008DF805108DF806200068C007400E8DF8D4
:1085600007006846FFF792FF1CBD1CB50020009075
:10857000019011208DF80000D6480068C007400E19
:108580008DF807006846FFF781FF1CBD2DE9FC410F
:108590000646002000900190122015460C468DF8EA
:1085A00000004FF008571EE0200A8DF80100C4F3C8
:1085B0000B008DF80240315C30448DF80310417897
:1085C0008DF8041081788DF80510C0788DF80600BC
:1085D000D7F8E001C007400E8DF807006846FFF7A6
:1085E00055FF241D2D1F002DDEDCBDE8FC811CB5D0
:1085F0000022009201920F228DF800208DF80100D8
:10860000080A8DF805008DF806104020B1498DF854
:108610000700012008606846F8F7DCFB1CBD1CB5AC
:10862000AA4B1B6893F8F0379B061DD500230093D7
:108630000193DB238DF800308DF801008DF80210D6
:10864000100E8DF80300100C8DF80400100A8DF840
:108650000500A0488DF806200068C007400E8DF880
:1086600007006846FFF712FF1CBD1CB500230093EE
:108670000193DB238DF800308DF801008DF8021096
:10868000100E8DF80300100C8DF80400100A8DF800
:10869000050090488DF806200068C007400E8DF850
:1086A00007006846FFF7F2FE1CBD1CB500220092D1
:1086B00001920F228DF8002005228DF801208DF8FF
:1086C000020084488DF803100068C007400E8DF842
:1086D00007006846FFF7DAFE1CBD2DE9FC410446A1
:1086E0000025009519208DF8000040070195417A7A
:1086F0008DF80110764909788DF802104189090A30
:108700008DF803104089714F8DF80400714E386860
:1087100041788DF8051080788DF806003068C00724
:10872000400E8DF807006846FFF7B0FE00951A204E
:1087300001958DF80000386800F5FC6001788DF82F
:10874000011041788DF8021081788DF80310C078FF
:108750008DF804003068C007400E8DF807006846A9
:10876000FFF794FE00951B2001958DF800006068CE
:10877000000E8DF801006068000C8DF80200A088E2
:10878000000A8DF8030020798DF8040020788DF818
:108790000500207B8DF806003068C007400E8DF87C
:1087A00007006846FFF772FE00951C2001958DF8C2
:1087B0000000A068000E8DF80100A068000C8DF884
:1087C00002002089000A8DF80300207A8DF8040049
:1087D000207C8DF80500207D8DF806003068C007EC
:1087E000400E8DF807006846FFF750FEFDE61CB509
:1087F0003649096891F82911490603D400F00F01A0
:108800000C2919D100210091019116218DF8001039
:108810008DF80100010A8DF80210010C000E8DF890
:1088200004002C488DF803100068C007400E8DF836
:1088300007006846FFF72AFE1CBD1CB50023009305
:10884000019316238DF800308DF80100080A8DF889
:108850000200100A8DF804001E488DF803108DF8F0
:1088600005200068C007400E8DF807006846FFF736
:108870000DFE1CBD1CB5002300938DF80000080AF6
:108880008DF802000193100A8DF8050011488DF84B
:1088900003108DF806200068C007400E8DF8070011
:1088A0006846FFF7F3FD1CBD1CB500200090019049
:1088B00080208DF8000007480068C007400E8DF842
:1088C00007006846FFF7E2FD1CBD0000280210000B
:1088D0009D021000E0010022474900EB400210B564
:1088E00001EB820101248B794449032B4A6802D0B1
:1088F000042B04D006E0844014434C6002E0844022
:10890000A2434A603D480421001DFAF7F4FAC0B2C0
:1089100010BD2DE9F0410520F7F7AFFE0024364EDB
:10892000012700BF306807FA04F108421DD004EBAC
:10893000440206EB8205AA79032A03D0042A01D057
:10894000052A12D1884330602D48006890F8100144
:10895000C00603D52B480078072806D060B2FFF781
:10896000BBFF0146A81DFFF7A0FD641C0A2CD9D34C
:10897000BDE8F0410520F7F79BBE20490020486084
:1089800080211D480FF051BB1C4C08B500252570F7
:1089900001261BE02078C8B10128FBD100226B46DC
:1089A00006211046F7F7C8FD0098400704D525704A
:1089B00004210020F7F79FFD00988007EAD5FFF714
:1089C000A8FF02210020F7F796FDE3E70021084603
:1089D000FAF71AFC00226B4608211046F7F7ACFDA7
:1089E00000210120FAF710FC00980007D2D5FFF70C
:1089F000C4FF26700E21E5E784241000A0031000B8
:108A000028021000940210002DE9FE43FE49086878
:108A100090F8B720467D02F00F05FC4A344690F8E6
:108A200014C0761C1278C5F1100706FB0CF604FB87
:108A30000CF4012A05D190F87E2602F00F05C5F14D
:108A400010070023CDE900340122B9300292B0F9B9
:108A50000230B0F90020EE4CEE48884604EB4C01A1
:108A600000EB4C00FBF719FB00282AD1D8F80020B6
:108A7000E94B107D11E000BF34F910C033F910103C
:108A80000CFB05FC01FB07C14FEAE17C01EB1C710B
:108A900041F30F1124F81010401CB042ECDB92F8A7
:108AA000690280070DD5DA48FAF7B9FFDB490023E0
:108AB000DB4A086003B00146BDE8F043D448FAF74A
:108AC000E5BFBDE8FE832DE9FE4FCF4D102128689C
:108AD00090F8B7201709A1EB121690F8A021D20741
:108AE0007ED0CA4AB0F8C280B0F8C0901278012A8D
:108AF00008D190F87E26B0F88986B0F890961709CC
:108B0000A1EB1216C749C848FAF7EBFAC749C6489D
:108B1000FAF72FFB2968C348C44C91F8B821AA463C
:108B2000120742D5DFF808C3B1F9D631B1F9D8013F
:108B30009CF800C0B1F9DA51B1F9DC41BCF1010F88
:108B40000BD191F85AC26344604491F85BC21BB2E6
:108B50006544644400B22DB224B291F8BAC1497D93
:108B6000B44ACDE90001B449AE485FEA4C7C0DD56A
:108B7000FBF74DFBDAF800002B46B04A007DB04908
:108B8000CDE90040A948FBF742FB0CE0FBF7D4FA23
:108B9000DAF800002B46A94A007DA949CDE900403A
:108BA000A248FBF7C9FAA348A44CDAF80010002544
:108BB000D346497D0FFA88F3CDE900510FFA89F2C7
:108BC0009A4691469C490295FBF767FA8046DBF886
:108BD000000053464A46007D9949CDE9005000E027
:108BE0004EE020460295FBF758FA58EA000147D1BB
:108BF0000020DFF83082904A5C46DBF800100FE07E
:108C000032F9103038F910C07B430CFB06334FEAC1
:108C1000E37C03EB1C7343F30F1322F81030401C6A
:108C20004B7D8342ECDC0020DFF80082844A0FE0B9
:108C300032F9103038F910C07B430CFB06334FEA91
:108C4000E37C03EB1C7343F30F1322F81030401C3A
:108C50000B7D8342ECDC91F86902800710D5794ED8
:108C600075483560497DFAF7DDFF316808443060AA
:108C70002068017D7248FAF7D5FF316808443060FA
:108C8000BDE8FE8F2DE9FE435F48016891F81A2484
:108C9000D30777D0804691F8340410234FEA10159B
:108CA000A3EB10146848694E92071BD54A7DB1F9B1
:108CB0002E04CDE90002B1F92C344646644A6549D8
:108CC0006148FBF739FA3068027DB0F93214CDE91A
:108CD0000012B0F93034604A60495C48FBF72CFA66
:108CE0005B485D4ED8F800100027C1464A7D0297C8
:108CF000CDE90072B1F93734B1F935245549FBF7A4
:108D0000CCF98046D9F80000017D0297CDE90071C9
:108D1000B0F93734B0F9352450493046FBF7BDF986
:108D200058EA00012ED10020474E4A4AD9F80010D7
:108D30000FE000BF32F9103036F910706B4307FBBB
:108D40000433DF1703EB177343F30F1322F81030CC
:108D5000401C4B7D8342EDDC00203C4E3F4A0EE040
:108D600032F9103036F910706B4307FB0433DF170C
:108D700003EB177343F30F1322F81030401C0B7DE5
:108D80008342EDDC9DE62DE9F0411F4C0746284E5D
:108D9000206890F84804C00716D0314800780628AB
:108DA00012D03048007807280ED006280CD02E4864
:108DB000007848B92D48007830B9307820B9084695
:108DC000FDF7A5FE012866D0206890F8B600C00720
:108DD00061D0274D1FB12748007898B151E003209A
:108DE000F7F74BFC2878C00701D0FFF70DFE287875
:108DF000400743D5206890F8A801000701D53078D6
:108E000008B939E040E039E02802100062021000A1
:108E100060A2012080D30120F00A10007802100027
:108E20006424100010080120640601204C08012071
:108E3000F7031000D84C10006C040120144D1000F2
:108E4000A8040120D403100050B30120C8B30120AE
:108E50007012100048B40120AC12100084B401203C
:108E60005F021000940210005A0210005502100018
:108E70008002100030021000FFF725FE0320F7F7F4
:108E800017FCBDE8F041FDE628784007F9D503203E
:108E9000F7F7F3FBAEE7BDE8F0810000FE490020E4
:108EA0000870704700E010460A5C8242FBD17047B0
:108EB00070B500250E4603462C4606E019462046AE
:108EC000FFF7F0FF1855641CE4B2B442F6D3002259
:108ED0000AE0985C904203D19D546D1CEDB201E014
:108EE000185C9854521CD2B2B242F2D3284670BDDC
:108EF00038B1884202D20B4601461846884200D05B
:108F00001154084670472DE9FF4F99B00120049095
:108F1000E24819689A460068067D477D41B19AF893
:108F200002109AF800905046B14205D2491C04E064
:108F30004FF000094D4608E0314645789AF80300A5
:108F4000CEB2B84200D2471CFFB2002007A9085495
:108F5000401C2D28FAD3199905EB051001EB400CA4
:108F6000681C67E01998E34608EB081100EB410C18
:108F700009F101045AE000BF0CEB040015900068F1
:108F800010B31CF8040000B31598002310F8010C6E
:108F900000B103461BF8041021B107AA1846FFF7D9
:108FA000A7FF03461A9800280BEB04000ED015907B
:108FB00010F8011C21B107AA1846FFF799FF0346D4
:108FC00015984178D9B91FE0E41C2EE0189010F8EC
:108FD000011C59B115981BF8042010F8010C10431E
:108FE00004D007AA1846FFF783FF03461898417874
:108FF00051B115981BF804204078104304D007AAFB
:109000001846FFF775FF034613B10CF804300CE067
:1090100004982D2806D20CF804000498401CC0B215
:10902000049002E0401E0CF80400641CB442A3D972
:1090300008F101008046B84294D907A80499FFF7C7
:1090400037FF804641001B980EF0CDFF00204FF601
:10905000FF7202E04AF82020401C4045FAD33BE072
:10906000199905EB051001EB400022304C460590A4
:109070002FE00598011901204058A8B3487838B36B
:1090800007AA105C48701B991B9A0AEB800B31F8F9
:109090001010491C22F810109BF800102046F9F718
:1090A0003DFF8BF800009BF801102846F9F736FFCA
:1090B0008BF801009BF802102046F9F737FF8BF878
:1090C00002009BF803102846F9F730FF8BF80300E5
:1090D000641CB442CDD36D1CBD42C1D3A8F10100C4
:1090E0001DB0C0B2BDE8F08FFFE7E41CF0E72DE94A
:1090F000F043994655784FF0010C1BE005EB051342
:1091000000EB430622360023147897780CE000BF6A
:1091100006EB040898F90180884503D10CFA04F89D
:1091200048EA0303641CE4B2A742F1D249F82530AF
:109130006D1CEDB2D378AB42E0D2BDE8F083F0B560
:10914000554B0026554D1C78A0B0012C11D11E7036
:109150000B78002B5AD04B78002B57D02B688F7888
:109160001C7D641EA74251D05B7DCC785B1E9C4267
:109170004CD000234FEA0D0444F823605B1C202BE5
:10918000FAD34B7891F803C01BE000BF50F823706E
:10919000B7B17E0846EA47063E4354F8237037438A
:1091A00044F8237004EB8307D7F804E04EEA060E78
:1091B000C7F804E0D7F808E04EEA060EC7F808E062
:1091C0005B1C9C45E2D2002304EB8306766840F8E2
:1091D00023605B1C1E2BF7D3012A17D1087808B136
:1091E000401E0870487808B1401E48702A68887888
:1091F000127D521E904201DA401C88702A68C8789D
:10920000527D521E904201DA401CC87020B0F0BD61
:10921000F0B50025059E2C468F1E00EB410006D4BC
:1092200030F9045CCF1E02D430F9067C3D448F1C1B
:10923000974207DAB0F90440C91C914202DAB0F94A
:1092400006000444281B00D540424FF435714843C2
:10925000C11700EB91508012A54203DD316808442C
:109260003060F0BD196808441860F0BD2DE9FF4F6B
:10927000DFF828B007460E46DBF80000002585B071
:1092800090F88A002C46C10605484FF4803900EB5F
:10929000460A2FD500210BE0A80310002802100079
:1092A000504E100037F8112000EB4103491C5A8042
:1092B000B142F7D34188018030F81620AAF8022085
:1092C00000210DE04A1C00EB420330F8122033F875
:1092D00002CC5B88634403EB420227F81120491C4F
:1092E000B142EFD307A80023009032461946384612
:1092F000FBF72AF807994FF0000800291CDCDBF87F
:10930000000090F88A00C00604D5F748B0F90000C4
:10931000019001E0CDF80480701E37F911C0039070
:10932000814224DBDBF8000090F88A00C00608D5F3
:10933000BAF90200029006E007EB410030F9020C96
:10934000E6E7CDF80880DBF8000090F88A00000717
:1093500006D502A8009001AB721E3846FFF758FFF1
:10936000DDE90110814207DD05460C4607E007EB09
:109370004100B0F90200DDE701DA0D460446A0EB3A
:109380000102A2FB09064FEAE27303FB096102FB3B
:1093900008110CEB0402C5F1000302EB43024FEA93
:1093A000E2730EF07DFD079CA4FB0936E51705FB73
:1093B000096204FB08221B184A410899A3FB010516
:1093C000CC1702FB015103FB04114A4600230EF0A7
:1093D00067FD039AD3170EF063FD00B209B081E672
:1093E0002DE9FF4F044681B00020DFF800930F9D68
:1093F000064607460090D9F8000090F88A0000075A
:1094000019D5207808B1401E2070607808B1401E40
:109410006070D9F80020A078127D521E904201DAC7
:10942000401CA070D9F80010E078497D491E8842A0
:1094300001DA401CE070AC48442144380EF0D3FD02
:10944000002293469246607830E021782AE000BFFF
:10945000D9F80030D5F82C8093F814C0431CE646A8
:1094600003FB0C1C08EB4C0CDDF80080BCF900C0C1
:10947000C44502DD761CB6B26744944502DD6246FF
:109480008B46824695F81CC0BCF1010F09D10EFB3A
:1094900003FC974B0B441CF8038048F080080CF841
:1094A0000380491CA3788B42D2DA401CE1788142C8
:1094B000CBDA6078D9F800100FE000BF91F814C043
:1094C00000F1010808FB0CB2EB6A03EB42021388BF
:1094D000854A443A22F81030401CE2788242EDDAA4
:1094E0008148497D52464438039BFFF7BFFE0E99E1
:1094F00008607D48442144380EF075FDDFF8E881AE
:109500002078A8F144080AF10101D9F800200AE006
:1095100092F814C0EB6A01FB0C0C03EB4C031B88A4
:1095200028F81030401CA3788342F1DA6E48117D90
:109530005A464438029BFFF799FE049908602F6150
:10954000AE8105B0CEE52DE9F047DFF8A0A1089F78
:10955000DAF80080D8F8AD5098F88C40BD4202D3BC
:1095600004F00F0512E0D8F8B190B94501D82509EB
:109570000CE004F00F06A7EB050CC6EB141404FB7B
:109580000CF4A9EB0505B4FBF5F4351998F8F1874F
:10959000584CC5F11006B8F1240F0CD14FF0240837
:1095A000A4F800806780A080E180178827811F8849
:1095B0006781A581E6811768684307FB06000009FB
:1095C00010601868694300FB061000091860DAF89B
:1095D000000090F8F107242806D11088208218880E
:1095E0006082A08A401CA082BDE8F0872DE9FF4F71
:1095F0003E48964684B00D7891F80190CA7800688C
:10960000002489780290007D2346A0465FEA050B7E
:109610002AD1CC4626E000BF0CF101060196DEF807
:109620002C604FF0000A0125009609E0DDE9006793
:1096300007FB005706EB47066D1CB6F90070BA44ED
:10964000A942F3DADDE90065454306EB4505B5F9C6
:1096500000506D4395FBFAF505FB0C33641BA844E1
:109660000CF1010C6245D7DA451EA9422FD1CC4638
:109670002BE000BF0CF1010601964E1E0396DEF8AA
:109680002C604FF0000A5D46009609E0DDE90067B6
:1096900007FB005706EB47066D1CB6F90070BA448D
:1096A000039EAE42F2DA019D05FB0016009D05EB1C
:1096B0004605B5F900506D4395FBFAF505FB0C33F3
:1096C00005FB0044A8440CF1010C6245D2DAB9F163
:1096D000000F2ED15D462AE0DEF82C704FF0000A14
:1096E0000126009713E00000504E100028021000E1
:1096F000E0A9012000DB0120771C07FB0057DDF803
:1097000000C0761C0CEB4707B7F900C0E244B24238
:10971000F2DA009E471906EB4706B6F90060764379
:1097200096FBFAF606FB05449B1BB0446D1CA94250
:10973000D2DA029D6D7D01956D1EAA422CD15D4647
:1097400028E000BFDEF82C704FF0000A4E46A2F170
:10975000010B00970AE0771C07FB0057DDF800C0FB
:10976000761C0CEB4707B7F900C0E244B345F2DAC8
:10977000561C06FB0057009E06EB4706019FB6F9F4
:109780000060764396FBFAF606FB054406FB0733BA
:10979000B0446D1CA942D5DA07980460079843606D
:1097A0000798C0F8088008B09CE42DE9F04F89B014
:1097B0004FF00009DFF87CB48646CDF81090CDF864
:1097C0001490CDF81890DBF8000014460F46828EF6
:1097D000217F4D464E46C84609B9B0F861217878D8
:1097E0003EE000BF5EF821A03878039032E001200F
:1097F000884010EA0A0F2BD0DBF80000D4F82CC008
:10980000029B007D01935B1C009303FB00130CEB98
:109810004303B3F90030934209DDC446DDF8048008
:1098200001FB036608FB03C81D4409F10109237FFE
:10983000012B7ED0002B009B00FB03F0FE4B0B4462
:1098400010F803C07ED04CF0200C00BF00F803C01D
:10985000491C0391B87803998842C8DA0298401CE1
:109860000290F87802998842BCDADBF8000090F8A0
:10987000240080060BD504AB224639467046FFF71C
:10988000B5FE049805990644069888440544E948BD
:109890000022F3170168087DC98A401E00FB05FA03
:1098A000A1FB060C02FB06C201FB03214FEAEA7B87
:1098B00052465B460EF0F4FA0390DE4841464FEA0A
:1098C000E87C00680026427D038B521EA3FB010842
:1098D00006FB01816A4303FB0C114FEAE27A53460F
:1098E0000EF0DEFA02900398002800DA0020D14E34
:1098F00003903168C98A814200DA084603900298D1
:10990000002800DA002002903168098B814200DAD9
:10991000084602902561A4F80C900399618120818A
:10992000207F022811D0012816D000B356E000E0B5
:1099300008E0009B5843C04B0B4410F803C04CF0A8
:10994000800C83E74CF0400C80E7306890F82500ED
:10995000C00743D0002210E0306890F82510C907F6
:1099600012D090F88A004007F4D4012205E0306854
:1099700090F85A01400631D5022202A903A801F04D
:109980009BFF207F012829D1306890F88A10490771
:1099900024D508A9CDE90014B0F91820B0F91610A3
:1099A00007AB3846FFF71CFD306890F82500C0076C
:1099B00004D0012208A907A801F07EFF20690090C9
:1099C000DDE9021008AB07AAFFF7BDFD08A907A84B
:1099D000FAF79CFA0798E0800898A08002A903A8EB
:1099E000FAF794FA039800B26080029909B22180D4
:1099F000326892F88A20520701D4E080A180EDE419
:109A00002DE9F04F91468B4A8646002348784FF067
:109A1000010BCE78D2F800A01AE000BF5EF82070EB
:109A20000A78441C8D7810E00BFA02FC1CEA070F40
:109A30000AD09AF81480D9F82CC004FB08280CEB43
:109A4000480CBCF900C06344521C9542ECDA401C3F
:109A50008642E3DAC9F81430BDE8F08F2DE9FC4FF7
:109A60007648521E009002EBD27040F34F030FFA7B
:109A700081F9A9EB030005B209EB030007B20A1450
:109A8000D01A1A446B4B4FF0000A01B216B250467E
:109A90002A46DFF8ACE11C685EE000BF40F6FF7BC1
:109AA0000B4618E0002A14DB94F815C0944510DD2D
:109AB000002B0EDB94F814C09C450ADD02F101086E
:109AC00008FB0C38DDF800C03CF918C0DC4500DAB2
:109AD000E3465B1C1BB2B342E4DDB4F834C05B4622
:109AE000DC4500DB00239B46914500D1DA460B465E
:109AF0002EE0002A2ADB94F815C0944526DD002BC1
:109B000024DB94F814C09C4520DD02F1010808FB19
:109B10000C38DDF800C03CF918C0B4F83480E045DA
:109B200001DB4FF0000CCDF804C094F8F1C7BCF194
:109B30000F0F05D14FF00008AEF81A80AEF81C8068
:109B4000DDF804C0ACEB0B0C604400B25B1C1BB234
:109B5000B342CEDD521C12B2BA429FDD94F8F12717
:109B60000F2A0ED10F23AEF80030AEF80250AEF837
:109B70000470AEF80610AEF80860AEF80A00AEF851
:109B80000EA0BDE8FC8F70B50D462E491446064662
:109B90000A7828490020012A096801D191F87F003C
:109BA000227F042A01D0022A10D191F87D30E28967
:109BB000184482420AD991F8250041074FF003006A
:109BC00003D521490978012900D120772868A061AF
:109BD000012229463046FFF7B2FA2246294630468E
:109BE000FFF7E3FD2046BDE870400AF03FBE2DE9D7
:109BF000F041C0B01C4690466B46FFF778FA22460B
:109C000041466846FFF7FCFE104E114F094D307873
:109C100078B9286890F8B801800729D5387840B914
:109C2000207F022801D0012822D18022694620A865
:109C300010E01DE028021000E0A901200A641000D5
:109C400000DB012056021000B40410004E02100088
:109C50004F0210000EF08DF90122414620A8FFF7B7
:109C60006EFA414620A8626905F054F9012826D011
:109C7000286890F8B911C9071CD0F949097819B1B9
:109C800090F8C102400615D5387898B9307888B96F
:109C9000F448007870B9F448F4490078097808432A
:109CA00008D1F348007828B94146684605F0BEF867
:109CB000002804D0224641466846FFF764FF40B0C2
:109CC000BDE8F0812DE9FF4F86468B4600204FF618
:109CD000FF755378D67828E003EB03140EEB4401AC
:109CE00001F12209E34914789778D1F800A018E02F
:109CF00009EB040191F801C0DC4510D10E999AF8E6
:109D00001480D1F830C0591C01FB08410CEB410113
:109D10000988884200D208468D4200D90D46641C4D
:109D200024B2A742E4DA5B1C1BB29E42D4DA039948
:109D300008800D990D8004B08EE62DE9F04F9B460A
:109D400082465378DDF824E02CE000BFCA4D03EBD7
:109D500003100AEB4004AD68223405EB40052235C0
:109D60001078C44F4FF0010917E0261876788E421C
:109D700011D13E68DEF830C096F814805E1C06FBF8
:109D800008060CEB4606B6F900605E4503DD05EB00
:109D9000000C8CF80190401C00B296788642E4DA00
:109DA0005B1C1BB2D0789842D0DA55E62DE9F0471B
:109DB000B04F8146C8B038681D46884690F860604C
:109DC00047A8CDE90005144646AB4846FFF77AFFA1
:109DD000287F48B9A34800780028386802D090F856
:109DE000616001E090F86260BDF81811BDF81C01D7
:109DF0006422091A7143B1FBF2F19F4F0E184FF420
:109E00008861B8680EF0EFF8B3B222464146484682
:109E10000095FFF792FF2068029002AB2FAA012164
:109E2000B868FFF770F8064601281ED901240DF125
:109E3000BC0A0DF10809B84612E000BF3AF8140058
:109E4000E88109EB84072946384601F005FE2B46D8
:109E50003A462146D8F80800FFF7C9FE641CE4B270
:109E6000B442EBD948B0BDE8F0872B4622464146C4
:109E70004846FFF7BCFEF5E72DE9F84F7F4CDFF8C9
:109E8000F4818946DDE90ABA257811789778D8F8FF
:109E90000040012D09D0724D2D78012D02D0784D52
:109EA0002D782DB194F86E5008E094F8595005E0E3
:109EB000744D2D78012D18D094F85550DFF8B8C1A5
:109EC00003EB031600EB4600DCF808C022300CEB75
:109ED00046062236247D5B1CDBF830C05C430CEB6D
:109EE00044034FF0010B19B10CE094F87050E5E712
:109EF00044784C4505D1B3F90040544501DD86F85E
:109F000001B00121D8F800C094789CF814C0ACF1DD
:109F1000010C64455ED1471C14F807C0CC4507D13D
:109F200033F914C0D44503DD06F1010C04F80CB07C
:109F30009278521ED7B24DE0421854784C4547D122
:109F400033F91120524543DD03EB41042A4434F92F
:109F500002CC4FF0000ECDF800C0624503DAB4F930
:109F600002C0624534DB012910D0D8F800C09CF84B
:109F700014C0ACF1020C8C4512D134F904CC62450A
:109F800023DAB4F90240A24222DB1EE0B3F9022038
:109F9000B3F900402A44A24217DAB3F90640F2E7C7
:109FA000DDF800C0624505DAB4F904C0624501DAA3
:109FB0004FF0010E34F904CC624503DAB4F90240E3
:109FC000A24205DBBEF1000F02D1741884F801B083
:109FD000491CC9B2B942AFD9BDE8F88F2DE9FF4F8E
:109FE0009AB092F8018092F803A00020ADF84000EA
:109FF000ADF84400159021481E4E9946017830680E
:10A000001446012908D016490978012902D01C49B3
:10A01000097819B16E3006E0593004E01949097821
:10A02000012933D0553011A905784778CDE90019B9
:10A03000DDE91A0110ABFFF745FE3068124990F8D0
:10A04000580060B1BDF84020BDF844300988D21AEC
:10A0500042436420B2FBF0F0084406B21AE017E075
:10A06000F70310005A0210005102100052021000B3
:10A070006202100028021000A8031000560210000F
:10A080005502100054021000280410007030CAE776
:10A09000B1F90060607848B9CDE90096DDE91A01B0
:10A0A0004FF0010800232246FFF7E6FEFE49E07864
:10A0B0000968497D491E88420AD1CDE90096401EB3
:10A0C00000F0FF0ACBB2DDE91A012246FFF7D4FE09
:10A0D0004046EEE01A9A00EB001102EB410202F159
:10A0E000220BF24A00F1020C00F10308926802EB25
:10A0F000410122310991EC49D9F83030421E0968FA
:10A10000097D4A4303EB42020A9201FB00F203EB92
:10A1100042020892421C96464A4301FB0CFC01FB9A
:10A1200008F103EB41010D9103EB420203EB4C0CF0
:10A130002178B8E00BEB010393F801801B9B984555
:10A140007ED132F911300693B34279DD00231393A7
:10A15000069BDDF820802B44019338F91180CDF85F
:10A160005080434505DA3CF91180434501DA01236B
:10A170001393E9B3CC4B1B6819931B7D18935B1E9B
:10A180008B427BD002EB4108CDF81480019B38F95B
:10A19000028CCDF83880434507DADDF81480B8F931
:10A1A0000280434501DA01231393069BDDF82080EA
:10A1B0003B4408EB41080693CDF8488038F9028CFF
:10A1C000434507DA0CEB4108B8F90280434501DA50
:10A1D00001231393DDF84880069BB8F902804345BC
:10A1E00005DA0CEB410838F9028C434559DB00E0F5
:10A1F00044E0139B23BB199B5B7D9B1E83420CD0C9
:10A20000DDF85080019B434507DA98460D9B33F9F2
:10A210001130984501DA0123139301280CD0DDF8A1
:10A220002880019B38F91180434505DA3CF91180FB
:10A23000434501DA01231393012922D0189B00E042
:10A240001EE09B1E8B420CD0DDF83880019B4345FD
:10A2500007DADDF81480B8F90480434501DA0123F8
:10A260001393DDF81480019B38F9048C434505DA1B
:10A27000DDF81480B8F90280434512DB139B53B11B
:10A280000FE0B2F90230B2F900802B444345F5DA11
:10A29000B2F90680F0E7099B4FF001080B4483F800
:10A2A0000180491CC9B2A3788B42BFF443AF0EF0C2
:10A2B000FF0050457FF60EAF15981EB075E52DE9ED
:10A2C000FF4F7A4CC5B000264FF48861A0680DF0AE
:10A2D0008AFE45AD0FCDFFF781FE479909680091D1
:10A2E000E8BB6B462DAA0021A046A068FEF70BFE36
:10A2F0000546012838D90AF091FB01246A4F0DF177
:10A30000B409EA4622E000BF396839F8140091F830
:10A310005710884212D9012688F800604899C881F0
:10A320000AEB84008346489901F096FBE1B25A4655
:10A33000489BD8F80800FFF75AFC06E05C48007814
:10A3400018B90AEB840004F09DFD641CAC42DBDD0F
:10A35000386890F85000000604D4002000E003E0C4
:10A360000AF061FB002E03D145AC0FCCFFF73FFC98
:10A3700049B01AE52DE9F04F8A464B490025994628
:10A3800086460E6828462B4609EB0301491E1FD45A
:10A39000747D8C421CDD377D01F1010107FB01F169
:10A3A0000EEB410803EB430C4FF000010AEB4C0BA2
:10A3B00002EB0104641E08D4A74206DD3BF911C07C
:10A3C00038F91440604404FB0C55491C0329EFDBA9
:10A3D0005B1C032BD8DB00B9012095FBF0F0E4E413
:10A3E0002DE9FF4F82B00C464178DDF83CB001B159
:10A3F000491E2D4A01F0FF09C1781668737D5D1E64
:10A40000A94201DA491C00E02946CDB2017801B128
:10A41000491E01F0FF0A8178307D431E994201DA1E
:10A42000481C00E0401EC6B2B4F9120009F1010157
:10A4300001906BE01C4B4A1C1868007D00FB02F782
:10A44000484305990BEB470E01EB400000900AF1E1
:10A45000010058E0144909680B7D059902FB0307C8
:10A4600001EB4701049FB1F90210B94247DD0099A1
:10A47000B4F9008001EB40010027B1F900C00CFBEA
:10A480000877B1F902C0B4F902800CFB0877B1F982
:10A4900004C0B4F9048001EB43010CFB0877B1F967
:10A4A00000C0B4F9068005E028021000A8031000DF
:10A4B0004F0210000CFB0877B1F902C0B4F9088014
:10A4C00001EB43030CFB0877B1F904C0B4F90A802F
:10A4D000B3F900100CFB0877B4F90CC001FB0C7148
:10A4E000B3F90270B4F90EC0B3F9043007FB0C11D4
:10A4F000B4F9107003FB0711019B91FBF3F12EF8E7
:10A500001010401C00B2B042A4DB11B2A94291DB92
:10A510004F4617E0017D781C41430BEB410800904A
:10A520003B46524621460598FFF724FF28F81A00BB
:10A530003B46324621460598FFF71CFF28F81600D7
:10A54000009807B2FB48AF420068E3DD007D691C5C
:10A5500041430BEB4101009109F1010148430BEB31
:10A560004008574612E04B463A4621460598FFF709
:10A5700001FF28F817002B463A4621460598FFF7B9
:10A58000F9FE009921F817007F1C3FB2B742EADDBF
:10A5900006B00AE4F8B5E8491046069A09781D465F
:10A5A000022914D2E54CE3492E7F236809687EB165
:10A5B00091F83D6376070AD5012A08D10093B1F9D5
:10A5C0004623DF4BDF49FFF70BFF20682863F8BD08
:10A5D00091F85A61F706FAD5B60609D50093B1F994
:10A5E0005D21D74BD849FFF7FBFE2068E862F8BD34
:10A5F000012AFCD10093B1F95D21E2E72DE9F04F8A
:10A60000834600208DB0CB4B0890009001900290C3
:10A61000039004900590069007901C68064601463A
:10A62000024604F5D3600B90607DC84F04F2926936
:10A6300004F29568450700D0012505EBD00C9A4639
:10A6400000200AE019F80030C500AB40194318F8A3
:10A650000030AB401A43401C00B26045F2DB0020E2
:10A6600004AD01E0032802DA45F8201001E045F8C6
:10A670002020401C00B20428F4DBB4F8A4060A90A1
:10A68000D1462021B2480DF0D0FC94F88716DFF8AF
:10A69000C0A228E0002021E094F814C0421C134618
:10A6A00002FB0C1237F91220B24200DD1646DFF829
:10A6B000A4C2BCF900C062450FDD089A0AB90122A4
:10A6C000089294F88726A1EB020C01225AF82C80FC
:10A6D000824048EA02084AF82C8018B2627D824221
:10A6E000DADC491C09B2227D8A42D3DCABF8246053
:10A6F0000024E846964951F8340001EBC40149684A
:10A70000084348F8240055F824201040002748F852
:10A7100024003E4651E000BF58F824C04FF0010E1F
:10A720000EFA06FA1CEA0A0F3ED00B9BDDF828C091
:10A73000DB5D09930EFA07F313EA0C0F04D0099BB3
:10A74000C3F100031BB20993937F128B9B074FEA5F
:10A7500040030DD5B2FBF3F3B2FBF0F2401E00FB59
:10A76000023006FB120209980244ABF8022009E00D
:10A77000B2FBF3FCB2FBF0F0099B634406FB003034
:10A78000ABF80200D9F80000C18A027D90F8870674
:10A79000B1FBF2F1401C4843614300EB4100ABF8D0
:10A7A000000058460AF062F855F8240010EA0A0F33
:10A7B00001D07F1CFFB2761C36B2D9F80020507D44
:10A7C000B042A9DC641C24B2042C93DB08980DB0C1
:10A7D00005E6F0B4584C2678564C256816B1B5F805
:10A7E000534001E0B5F851401E7F64431EB195F817
:10A7F0005050EE0702D0F0BCFFF7D8BAAD0705D530
:10A80000554D2D68A54201DAF0BC58E5F0BCFFF7C4
:10A81000EEB92DE9F047814646488A460023016893
:10A82000184601250E7D4F7D1EE000BF00EB001491
:10A8300009EB44042234194612E000BF52F820808C
:10A8400005FA01FC18EA0C0F08D004EB010898F88F
:10A8500001C0BCF1000F01D188F801A0491CC9B2A8
:10A86000B142EBD3401CC0B2B842DFD3BDE8F087A1
:10A870002DE9F041304ADFF8BC80012412783AB962
:10A88000D8F8002092F82420920724D5012922D15B
:10A8900081780278891A01D5C1F1000101F1010125
:10A8A000CDB2C1784078081A00D54042401CC7B2EA
:10A8B00039462846F8F732FBC6B239462846F8F73B
:10A8C00035FBC0B2012E06D1D8F8001091F88510E2
:10A8D000814200D800242046BDE8F0812DE9F04FE8
:10A8E0008A46144983469E464FF001095078D6782F
:10A8F0000C6839E000EB00130BEB430322331178B3
:10A9000095782DE05F1897F801C0D44526D194F8CA
:10A910001480471C07FB0817DEF82CC00CEB470718
:10A92000B4F867C1B7F90070BC4517DA4FF00009F9
:10A9300018E00000280210005502100074021000F8
:10A9400000DB0120A28301008E8301000A64100055
:10A95000984E10002804100030041000491C09B261
:10A960008D42CFDA401C00B28642C3DA484636E553
:10A9700030B5FE4AB2F90030FD4AB2F90020FD4C74
:10A98000246834F9A95FB4F9024029B9FA49B1F948
:10A990000030FA49B1F90020A04201DD104630BD77
:10A9A000A84201DA184630BD201AD11A4843611B6B
:10A9B00090FBF1F0101A00B230BD2DE9FF4F83B0CB
:10A9C0004FF0FF36DDE9105489460746019693465D
:10A9D0004FF0640AB04610460699F8F7A7FA01B29C
:10A9E0004FEA6900009188427DDAE2480068B0F8D9
:10A9F0008D204A4577DD129931B1012918D00229FD
:10AA000027D0032970D13DE0A11E05D4027D611E2F
:10AA100001FB025137F91160427DA11C8A424DDDD4
:10AA2000007D04F1030404FB005037F9100044E0FA
:10AA3000A91E07D4027D611C01FB025107EB4101F5
:10AA400031F9046C007DA91C884237DD04F1010452
:10AA500015E0A91E0BD4427DA11C8A4207DD027DB0
:10AA6000E11C01FB025107EB410131F9046C007D4F
:10AA7000A91C884222DDA11E20D4A4F1010404FBFC
:10AA8000005016E0A91E09D4A11E07D4027D611E44
:10AA900001FB025107EB410131F9046C017DAA1C55
:10AAA00091420BDD427DA01C824207DDE41C04FBC9
:10AAB000015007EB4000B0F904008046701C36D00E
:10AAC00018F1010033D058460699F8F727FA009993
:10AAD00002B2A9EB0100069B01B2ABEB03006423B9
:10AAE0005843009C01E042E021E009EB040354429A
:10AAF00003EB440390FBF3F0002800DA40424143AB
:10AB000091FBFAF1A9EB010109B25A4512D1069A5B
:10AB100064235A43069BF31A03FB002393FBFAF2C8
:10AB200064240BFB04F312B2A9EB0B0412E00198AE
:10AB300007B054E464230BFB03F2A8EB0B0303FB05
:10AB4000002393FBFAF2069B6424069D634312B232
:10AB5000A9EB050404FB003494FBFAF3484390FB93
:10AB6000FAF01BB21A440844C2EB400006B2304669
:10AB7000DEE72DE9FE4F99467E4B571C0646D3F87B
:10AB800000C04FF0FF3004469CF81430054607FB28
:10AB9000031B5FEA090836F91BA009D0B8F1010FC1
:10ABA00018D0B8F1020F21D0B9F1030F52D133E020
:10ABB000B2F1010803D402FB031536F915509CF8D5
:10ABC0001580B84544DD02F1020404FB031336F995
:10ABD00013403DE04F1E03D406EB4B0535F9025CF4
:10ABE0004F1CBB4234DD06EB4B032FE0B1F10108F3
:10ABF0000AD49CF81580B84506DD951C05FB0315A5
:10AC000006EB450535F9025C4F1CBB4220DD571EA3
:10AC10001ED402FB031317E0B1F1010808D4B2F10E
:10AC2000010805D402FB031506EB450535F9025C66
:10AC300001F1010843450BDD9CF81580B84507DD9F
:10AC400002F1020404FB031306EB4303B3F90240D1
:10AC50006B1C01D1631C0ED09CF88A309B0607D573
:10AC60008DE806022B46224651463046FFF7A5FEE8
:10AC7000691C03D003E047F6FF710AE02546611C1A
:10AC800000D12C466219C2EB4A0109B2884200DDAC
:10AC900001463848006890F8F107022808D1384882
:10ACA00020F8395000EBC900A0F802A08480C180D0
:10ACB0000846BDE8FE8F2DE9FF4F1E462D4B4FF095
:10ACC000000A1178186883B0554654465FEA010EB1
:10ACD00006D15178B9B1417DD778491E8F4212D043
:10ACE000017D97788B46491E8F4204D192F801C0AE
:10ACF000BCF1000F07D08F420BD1417D92F803C009
:10AD0000491E8C4505D1B0F8AB00801CA6F8270081
:10AD1000B6E0517892F803C0F06A24E04B1C0BFBBC
:10AD200003F200EB42020192039A01EB011302EBE2
:10AD3000430202F122090BB27246009310E000BFF9
:10AD400009EB020393F80180049B984507D1019B0E
:10AD500033F91230534502DD009C9A4615B2521C5D
:10AD60009742EDDA491C8C45D8DA0BE02804100034
:10AD70002A041000280210002004100022041000F1
:10AD800000DB0120012322462946FFF7F2FE074699
:10AD9000002322462946F06AFFF7EBFE8046022395
:10ADA00022462946F06AFFF7E4FE83460323224643
:10ADB0002946F06AFFF7DDFEDFF884A48146DAF861
:10ADC000000090F88A1049061DD5ADB1017D491EDD
:10ADD000A94211D01CB1407D401EA04201D1B8460D
:10ADE0000AE041463846F8F799F802B24946584613
:10ADF000F8F7A4F80FFA80F80027601ED446641C08
:10AE0000DAF800901FE008EB0700F3E7002819DBF1
:10AE100099F81510814215DD99F814A0431CF26AC7
:10AE20000AFB03F102EB410B691E6A1C08E00029D2
:10AE300005DB8A4503DD3BF811303B441FB2491C5A
:10AE40009142F4DD401CA042E0DDFA2008FB00F84E
:10AE500098FBF7F004B2A6F8274001212046FFF73F
:10AE600087FDF8490C80DCF8001091F8F1170229F1
:10AE700003D1F5490C844F848884B18C814201DD73
:10AE8000012055E6002053E62DE9F04F8246DDE92A
:10AE900009B500209E462860894653782CE000BF03
:10AEA000E74903EB0314DBF82C70096803F1010C8C
:10AEB0000AEB44040E7D223406FB0CF607EB460633
:10AEC000117814E0671897F80180C8450DD136F95C
:10AED00011802F6847442F6036F91170874204DDD6
:10AEE000AEF802103846AEF80030491CC9B2977867
:10AEF0008F42E7D20CF0FF03D1789942D0D236E5E9
:10AF00002DE9FF4F83B01878109C92461E46A07022
:10AF1000987820705878E070D87860704FF000080A
:10AF20005F784CE0039907EB071001EB400101F15A
:10AF30002209049901EB400000F1220B1298C26A29
:10AF4000BF480068017D781C4143019002EB41003D
:10AF5000009035782EE000BF09EB0500417851459F
:10AF600026D1009830F91510119881421CDD08F1A6
:10AF700001001FFA80F821782846F7F7CFFF2070EC
:10AF800061783846F7F7CAFF6070A1782846F7F76E
:10AF9000CDFFA070E1783846F7F7C8FFE0700BEB03
:10AFA000050080F801A003E00BEB050000214170D3
:10AFB0006D1C2DB2B078A842CEDA019807B2F078B5
:10AFC000B842AFDA0FFA88F0B2E59D490278096815
:10AFD00022B10A7D8378521E934208D1427822B171
:10AFE000C278487D401E824201D101207047002076
:10AFF0007047017869B19249837809680A7D521EC9
:10B00000934206D0427822B1C278487D401E8242E7
:10B0100001D1012070470020704730B50546A1B02E
:10B02000874800238DF8803002680C46107D401E52
:10B030008DF882008DF88130507D6B46401E8DF872
:10B04000830020AA2846FEF752F8002220A968466D
:10B05000FEF775F86A4621462846FFF7DAFB21B06D
:10B0600030BD2DE9F74F76480C46154601684FF084
:10B070000009B1F93AA0217809B1491E217061781F
:10B0800009B1491E61700268A178127D521E914279
:10B0900001DA491CA17083460068E178407D401EBA
:10B0A000814201DA491CE170A0782870E07868706C
:10B0B0002078A8706078E87067782FE0267807F12C
:10B0C000010826E00098C16ADBF80000027D08FB59
:10B0D000026001EB4000B0F90000504517DB09F1B8
:10B0E000010000F0FF0929783046F7F717FF2870B4
:10B0F00069783846F7F712FF6870A9783046F7F795
:10B1000015FFA870E9783846F7F710FFE870761C4D
:10B11000F6B2A078B042D5D208F0FF07E078B84286
:10B12000CCD24846C5E52DE9FE4F0A780192521E61
:10B13000D2B202928A78424B521C02F0FF0A4A783D
:10B140000092CE78D3F8009035E000BF4FF0000EAB
:10B1500074467546029B25E099F8148002F1010CB3
:10B160000CFB083CC76A07EB4C08B8F900B04FF07D
:10B17000020808EB4C0C6744B7F90070ABEB07070B
:10B18000002F02DA4FF0010402E001DD4FF002046B
:10B190002DB1A54203D00EF1010505F0FF0E5B1C99
:10B1A0002546DBB25345D7D9BEF1010F01D90020A6
:10B1B0007FE5521CD2B29642C8D2009A019B521E21
:10B1C000D2B2761C06F0FF0A009241E04FF0000E6A
:10B1D000F0467446009A2AE099F81470551CAB4664
:10B1E00005FB0735C66A02F1020C0CFB073706EBBC
:10B1F000450506EB4707B5F90050B7F900703385F0
:10B20000C66A7285C26A9585EA1B002A02DA4FF087
:10B21000010802E001DD4FF002082CB1444503D0E3
:10B220000EF1010202F0FF0E44460BF0FF02524500
:10B23000D2D9BEF1010F09D9002180F83410B6E748
:10B24000280210000E25100000DB01205B1CDBB281
:10B250008A789A42BAD201202BE52DE9F14FE8B065
:10B260000024FF48DFF8FC835E940068C8F80400FF
:10B27000FD4D00F58860C8F808002968A246A1467F
:10B28000B1F994105B9126464FF488610CF0ABFE47
:10B29000286890F85010CA0701D1890701D54FF0EE
:10B2A000010AF249097821B190F85B01C0F340002E
:10B2B00003E090F85A01C0F3C0006490002014909D
:10B2C00014AB41AA0121D8F80400FDF71CFEE8499F
:10B2D000074601240873AB4666E23C2103A80CF044
:10B2E000A4FEE4480E900F90E1B241A88DF8321010
:10B2F00030F81400ADF81A005EAA03A8CDE90002E8
:10B3000014A800EB8402129263ABD8F80400FFF794
:10B31000BBFD0546DBF8000090F8F1071D280DD1B4
:10B32000D4481D21018004EB440120F8115000EBAA
:10B330004100BDF81A20428063218180ADF8305071
:10B34000052203A86399FEF789FBADF846000021AA
:10B35000ADF833108DF84010BDF98E01BDF98C2188
:10B36000ADF84400ADF8422088F8001050B14AB161
:10B37000DBF800100B7D5B1E984203D0497D491E0F
:10B380008A4208D1012160919DF8411041F00101EC
:10B390008DF8411001E000216091B7490978012939
:10B3A0001ED1DBF8001091F88726904218DB0A7D49
:10B3B000521E904214DCB14AB14BB1F984061080A0
:10B3C0001B78012B03D191F88E3618441080B1F808
:10B3D000842691F88606AB49A2EB00000880E2E1E2
:10B3E000A948007880077DD5A0480078002879D149
:10B3F000DBF80000A54A90F8A83012889342A04AD2
:10B40000127801D212B16DE0022A6BD25E9B5B9A78
:10B41000934267DA01228DF8282090F8A4105D91FC
:10B4200097490978012905D190F8CE225D991144F8
:10B4300089B25D91609901293CD010F8A51F407830
:10B4400008445890924803A9129BB0F900205AA8CA
:10B45000CDE900020291D8E90101E2B2FFF750FD07
:10B460008C4980B2ADF81A0008555D99884239D9E7
:10B470005899884236D88649B1F900108D4231DD9D
:10B4800001281AD02ED9DBF8000090F88A1089071D
:10B4900018D58149B0F8A20009684043884211DB01
:10B4A000E1B203AB5AAAD8F80800FFF704FC012860
:10B4B00008D017E090F8A700C3E77848B0F900007B
:10B4C00085420FDD0220ADF82A00ADF82C000020E7
:10B4D0008DF829004FF00109E1B203AB5AAAD8F860
:10B4E000080098E060991298FFF7C2F901287DD111
:10B4F0006448B0F90000854279DD41A931F81410A3
:10B5000059916749B1F90010814213DA5AAACDE97D
:10B51000002003A90291D8F80410E2B2129B084659
:10B52000FFF7EEFC41A921F8140012995A9A0A601B
:10B53000ADF81A00DBF80000018FA9421ADD90F87F
:10B5400024005D46400615D5012F13D166AA03A835
:10B550001299FFF786FD296891F83C10814209D2C3
:10B5600066A8FFF746FD28B966A903A8FFF7DBFD2B
:10B570008DF84000DBF8000090F87C5040480078DF
:10B5800050B11298FFF721FD0128DBF800003BD0F5
:10B5900090F8CF02284485B241A830F81400A842A0
:10B5A00024D903A800904FF001094E46E3B2454666
:10B5B000129A0E98D8F8041000F06AFA41A8DBF845
:10B5C000001030F8142091F87E0082421FD2284BE0
:10B5D00002208DF82800BDF82E209A82B1F8801044
:10B5E00050468A4200D20020599901E05EE015E001
:10B5F00003290FD300280DD00090E1B203AB129ABB
:10B600006868FEF7C7FFC8E090F8D002C2E70420E0
:10B610008DF82800D0E0FEF7EAFAC4E0DBF800106D
:10B6200091F85A21D20741D01E4A1268F2B31E4A3D
:10B630001278DABB00228DF8282091F85A014007D1
:10B6400005D5E1B214AAD8F80400FFF7E6FC47F6E6
:10B65000FF7058900548007848B3DBF8000027E0F9
:10B6600070021000A8031000280210005A021000F7
:10B670000E25100000DB01206202100020041000E3
:10B680005502100028041000A8021000BA03100090
:10B690002A041000E0A90120300410002C0410003E
:10B6A0001E0410009C010022430210007BE002E017
:10B6B00090F892510AE060980128574800780AD023
:10B6C0000128DBF8000010D090F86451534800784E
:10B6D00001280DD012E00128DBF8000002D090F81C
:10B6E0006651F3E790F86551F0E790F86351EDE7A4
:10B6F000DBF8000090F8D102284485B24848B0F940
:10B7000000104848B0F90000814213DA5AAACDE986
:10B71000002003A90291D8F80410E2B2129B084657
:10B72000FFF7EEFB41A921F8140012995A9A0A601A
:10B73000ADF81A0041A830F81400A84233D958993E
:10B74000884230D868990220E3B2087003A80090BC
:10B750004546129A0E98D8F8041000F099F96498AA
:10B760000090E1B203AB129A6868FEF713FFDBF8B2
:10B77000000090F85A0180070DD52748007801286D
:10B7800009D1E1B203AB129A6868FFF7A7F8012864
:10B7900001D125490870649870B1E1B203AB129AE7
:10B7A0006868FFF716F8641CBC427FF696AD1F4828
:10B7B0000078012805D017E0E1B203AB129A68685F
:10B7C00029E70420ADF81A00ADF8180018486421E4
:10B7D00008910088401CADF8300002208DF8280048
:10B7E00003A8FEF70BFF0643124880F800901248AA
:10B7F0000670DBF8000090F8F107182803D10F4815
:10B80000418D491C418569B0BDE8F08F0C4800218D
:10B8100001730180704700004B02100055021000B8
:10B820001E0410002E0410001C0410006202100000
:10B8300020041000490210004A02100000DB012021
:10B840000E251000F0B5B2F900400568AC4202DDEB
:10B85000B3F900102EE002EB410434F9026CAE4261
:10B8600004DA03EB410131F9021C23E00024491EF4
:10B870000BE000BF32F91470AF4205DC02EB440666
:10B88000B6F90270AF4202DA641C8C42F2DB32F984
:10B89000146003EB440133F91430B1F9021002EBE8
:10B8A0004402AD1BC91AB2F902206943921B91FBF5
:10B8B000F2F119440160F0BDF0B50E462D4909685A
:10B8C00091F82A315C0701F29A4303D52A4C247877
:10B8D000012C26D072B3012A35D0022A3CD0042A8A
:10B8E00047D191F893C491F892441A4691F899146B
:10B8F00003EB4C0303EB410707EB44050CEB04019E
:10B900003E2936DCBCF1010F02DD6146FFF79AFFEC
:10B91000012C2EDD2B463A4621463046BDE8F0404C
:10B9200090E791F894C491F8954403EB4C0591F895
:10B930008F1419E091F894C491F8954403EB4C05E9
:10B9400091F8961410E091F894C491F8954403EBA3
:10B950004C0591F8971407E091F894C491F8954438
:10B9600091F8981403EB4C0503EB410202EB4C07F2
:10B97000C4E7F0BD280210003D0410004FF47A72B5
:10B98000504390FBF1F1744810B5814201DAC011C7
:10B9900010BD42F6A640814201DD5A2010BD6F4A1B
:10B9A000002000BF32F910308B4205DC02EB40036F
:10B9B000B3F902308B4202DA401C4528F2D332F947
:10B9C000104000EB800302EB4000091BB0F90200BD
:10B9D000553B001B01EB810191FBF0F0184410BDB9
:10B9E00030B50D460446FFF7C9FF00EBD07040109C
:10B9F000002D02D00DDD34B130BD002C03D005DDAB
:10BA00004FF02D0030BD4FF0000030BD4FF05A0018
:10BA100030BD002C03D005DD00F15A0030BD6FF0C1
:10BA2000590030BDA0F15A0030BD10B58C1A00D5B8
:10BA30006442002800DA404204EB400011440A1836
:10BA4000081A521040104FF47A71484390FBF2F0FC
:10BA5000C0F57A70588410BD30B582780378CD89EE
:10BA6000D21AC3784078521C1B1A5B1C05FB02F0EB
:10BA7000D4185D4340006A00B0FBF4F0B2FBF4F26E
:10BA8000904202D9C8830A8430BDCA83088430BD7D
:10BA90002DE9FF4F0027164682B03A463C46BC4689
:10BAA000BB46BA46707896F8039025E0039900EB00
:10BAB000001301EB4301223101913178009196F896
:10BAC000028016E0019B0B445D78059B9D420FD1DF
:10BAD000A9EB000303F1010E009B0EFB0EAACD1A89
:10BAE0006D1C05FB05BB05FB0ECC7F1C2A44744472
:10BAF000491C8845E6DA401C8145D7DA4FF47A7054
:10BB0000504390FBF7F101FB04F54FF47A734FF4C7
:10BB10007A70604390FBF7F0514391FBF3F260437E
:10BB200090FBF3F195FBF3F5ACEB0505ABEB0207EE
:10BB3000AAEB01046800391BFFF752FF0F99224658
:10BB40004877394628460F9BFFF76FFF0F9906B0DD
:10BB50003046BDE8F04F7FE75AD3FFFF488301002E
:10BB6000FC4900200870FC490870FC4908707047C7
:10BB700010B5FB4A00206FF0004100BF42F82010D2
:10BB8000401C1428FADB3C21F6480CF02CFA40212A
:10BB9000F5480CF028FAF5490020486188610870E2
:10BBA00010BD70B5F249002001220870F149FA4B2E
:10BBB000FA4D0A70F049FA4E0870F0490870F049E1
:10BBC0000870F0490870F0490870F0490A70F049AF
:10BBD0000870E6490871486288628870C861086226
:10BBE000CA70EC4A126832F8794F1C80938A2B8015
:10BBF000B2F817503580EB4EB2F8E6203280EA4EAC
:10BC00003480EA4C2380EA4B1D80EA4B1A80EA4AD2
:10BC100010800861FFF7A4FFBDE87040A8E72DE998
:10BC2000FF4FDC4881B09A460068427D90F814B01E
:10BC3000521C62E0D7494FF0010ECDF800E00968D0
:10BC400047F6FF70C543097D0024019B514303EB78
:10BC50004107029B264603EB410C039B03EB410982
:10BC60005B4615E03CF8131037F81380A1EB080190
:10BC700009B2884200DD08468D4200DA0D460029EF
:10BC800002DA4FF0000E03E002DD4FF000010091F8
:10BC90005B1EE7D2009B5EEA030108D0BEF1010FF4
:10BCA00003D0BEF1000F04D006E0012B04D1002028
:10BCB00002E0012B00D1284659460EE03CF8113035
:10BCC00037F811505B1B1B1A1BB2534505DACAF13A
:10BCD0000005AB4201DD1C44761C491EEED2002E4D
:10BCE00001DD94FBF6F42118584604E037F81030D3
:10BCF0000B4429F81030401EF8D2521E9AD105B0DC
:10BD0000BDE8F08F2DE9FF4FA24881B000680E9D7D
:10BD1000437D007D5B1C009085E000BF9D4947F698
:10BD2000FF70C6430968019A4FF0010C097DE04697
:10BD3000594302EB4104029A02EB410B039A02EBD6
:10BD4000410E009A14E000BF3BF8121034F8127054
:10BD5000C91B09B2884200DD08468E4200DA0E4651
:10BD6000002902DA4FF0000C02E001DD4FF000087C
:10BD7000521EE9D25CEA080109D0BCF1010F03D0E0
:10BD8000BCF1000F05D008E0B8F1010F05D100208B
:10BD900003E0B8F1010F00D130460022164692466A
:10BDA00091469046009917E03BF8117034F811C0A5
:10BDB000A7EB0C073F1ADDF810C03FB267450BDA5E
:10BDC000CCF1000C674507DD01FB016601FB07991B
:10BDD0000A44BA4408F10108491EE5D206FB08F1FD
:10BDE00002FB121709FB08F102FB1A1C06FB0AF6FC
:10BDF00009FB126191FBF7F8009A12E00CFB02F1CB
:10BE000091FBF7F14144A94201DD294603E06E426E
:10BE1000B14200DA314634F81260014431442EF860
:10BE20001210521EEAD25B1E7FF478AF67E72DE94D
:10BE3000F00F9B46574B614E1D68367895F8904140
:10BE4000022E02D0032E03D003E095F8914100E0CA
:10BE50000024C2F11007BBF1010F08D0DFF8609198
:10BE6000042E08D0002E74D001269A4667E0BDE863
:10BE7000F00FF7F77ABF01259A463FE0002336E03E
:10BE800005FB043431F914C030F914800CFB02FCBA
:10BE900008FB07CC4CF30F1C21F814C0D6F800C0E7
:10BEA0009CF88C81984503DC9CF88DC19C4503DA95
:10BEB00039F814C021F814C0DAF8006096F88EC181
:10BEC0000CF1010CAC4505DC96F88FC10CF1010CAE
:10BED000AC450BDA96F88CC19C4507DA96F88D6173
:10BEE0009E4203DD39F8146021F814605B1CDAF817
:10BEF00000405646247D9C42C2DC6D1CDAF80030BE
:10BF00005B7D5B1CAB42B9DCBDE8F00F70470025E0
:10BF100012E000BFDAF800301B7D06FB03536D1CF6
:10BF200031F913C030F913800CFB02FC08FB07CC7D
:10BF30004CF30F1C21F813C0A542EBD9761CDAF89C
:10BF4000005053466D7D6D1CB542E0DC01224D462C
:10BF500046E04BE04B0210001C04100043021000AE
:10BF6000B84E1000F40A0120300B0120B403100079
:10BF70004702100040021000480210004902100061
:10BF80004A02100045021000460210008402100010
:10BF9000A00210002802100020041000220410004B
:10BFA0002404100026041000280410002A041000A5
:10BFB0002C0410002E0410001E0410005A02100061
:10BFC00060A20120204606E002FB0606401C35F870
:10BFD000167021F816701E68367D8642F4DC521CFD
:10BFE0001868407D401C9042ECDC8DE7FE4C2478C4
:10BFF000012C04D06B7D2C7D5B1C634341E001254B
:10C000009A4626E000241EE0F84EC4F11F0806EB15
:10C0100085064FF0010C56F8046C05FB03430CFA3F
:10C0200008FC16EA0C0F1ED0BBF1010F18D031F935
:10C03000136030F913C056430CFB076646F30F1626
:10C0400021F81360641CDAF800301B7DA342DBDAB0
:10C050006D1CDAF80040647D641CAC42D2DC53E70E
:10C0600030F81360ECE739F81360E9E731F9134071
:10C0700030F91350544305FB074444F30F1421F8DF
:10C0800013405B1EF2D23FE72DE9FF4FDFF86083DC
:10C0900083460C46D8F800009946002590F82410F5
:10C0A00083B0CB06017D4FF0010A04EB41004FEA5B
:10C0B00041020FD50327464659460BF015FF30685D
:10C0C000417D007D491C414342000BEB410104EBE3
:10C0D000800001E0022759460BF006FF01264FF0D1
:10C0E000300B00BFD8F800204FF03003107D92F8DD
:10C0F000BA21CDE900B000FB06F1520704EB410084
:10C10000002A0246214602DAF8F781F801E0F8F742
:10C1100013F8761CBE42E5DB0021404634E000BF48
:10C1200092F8242003EB0106D206002A34F91120EC
:10C1300034F91660A2EB060252DA002A01DAC2F1E3
:10C14000000203EB43030B4424F81320036834F983
:10C1500011201B7D01EB430634F91660921B00D5BC
:10C16000524201EB830312B224F8132003681B7DB3
:10C1700003EB43030B4434F913604E4500DD6D1CA3
:10C180004A4500DD6D1C491C0268137D8B42C7DCEB
:10C19000DAB202EB820245F2AA5124F812100168C9
:10C1A000097D01EB810104EB41014D800268914959
:10C1B000127D02EB820204EB4202A2F80490D8F84E
:10C1C00000008989007D00EB800004EB4000C18005
:10C1D0000598854201DD4FF0000A504607B08FE513
:10C1E000002A00DA524201EB430312B224F8132072
:10C1F000C6E7F0B57E4B00221C68237D94F8875675
:10C20000B4F8A97603EB050C5E1B00EB4C0501EBC3
:10C210004C0110460DE000BF31F910E035F910C0B7
:10C22000BE44F44500DD521C05EB430501EB430120
:10C23000401CB042F0DB94F8AB166E48914207D236
:10C24000816A09B10120F0BD012181620020F0BDA9
:10C250000021FAE72DE9FF5F16466748644A8B46DE
:10C26000077810680025012490F87C12A84617B1C1
:10C270004FEA111101E001F00F0101EB81014FEADA
:10C28000410790F86912924689071FD5B0F9739259
:10C290005B485A4A01680098F7F7F8FB5948574934
:10C2A00002680B68D1F804C0D21A4368A3EB0C03F0
:10C2B0001A448368D1F808C0C068C968A3EB0C03AE
:10C2C0001A44401A8118494500DD0024DAF80000BC
:10C2D000D14690F88006000713D54B48007880B906
:10C2E0004A48007868B94A480078012809D1494885
:10C2F000007830B959460098FFF77BFF08B1002459
:10C3000000E00CB94FF005083A480021C0F8108051
:10C310000279AAB13170426A521C4262D9F80030E7
:10C3200093F87D3203F00F0303EB8303B2EB430F6B
:10C3300002DD41620171012504B02846BDE8F09F8D
:10C34000012314B141623370F6E7426A541C44621F
:10C35000BA4209DD03714162D9F8002092F87D22CA
:10C36000120701D1017101253170E5E72DE9F84F80
:10C370001F48294900688979B0F98D40B0F990309B
:10C38000012906D190F8BA11890702D5B0F9032224
:10C3900001E0B0F9792090F8F1171C2903D11F4969
:10C3A00063258A82CD8214490978009111B1B0F9D0
:10C3B000931101E0B0F95F11194D2D78012D10D1C5
:10C3C000184D2D686DB190F85A51B0F99240B0F9FE
:10C3D0009521AD0705D5144D2D78012D01D1B0F96A
:10C3E0009721094D2D7821E0CC021000382610004D
:10C3F00028021000B40310005A0210007424100028
:10C400007802100064241000550210004E02100043
:10C410006202100047021000AC02100000DB012095
:10C420004B0210009C0100221C041000012D38D08A
:10C43000022D07D3B0F8D31209B1B0F9D3221446B4
:10C4400023461946FC4DA146FF4F2C80FB4D2B8007
:10C45000FB4D2A80FB4D298090F88F6090F87B502F
:10C46000A41B0FFA84FC90F8CA4090F85C61A7F80E
:10C4700000C0E6461C1BDFF8D4C324B2A346ACF8C8
:10C480000040F34C551B2DB22580DFF8C8C38E1B2E
:10C49000F14C36B2ACF800602478AA46012C0FD0DB
:10C4A00063E090F8CC522C442B4490F8CD5224B247
:10C4B0002A4490F8D2521BB2294412B209B2C1E701
:10C4C00090F8C940642504FB02F8B8FBF5F8424433
:10C4D000DFF86C83A8F8002004FB09F8B8FBF5F836
:10C4E00008EB0902DFF85083A8F8002004FB03F2F0
:10C4F000B2FBF5F2DFF844831A44A8F80020009A52
:10C50000002A05D090F86931CE4A03FB01F302E01E
:10C51000CC4A04FB01F3B3FBF5F31944118004FB8F
:10C520000AF2B2FBF5F3CA4903EB0A020A8004FBE4
:10C530000BF2B2FBF5F3C54903EB0B020A8004FBD7
:10C540000EF1B1FBF5F202EB0E01398006D090F846
:10C55000691101FB06F1B1FBF5F103E004FB06F400
:10C56000B4FBF5F13144ACF80010BC4909788907F7
:10C570000AD4B349B04A09881180B04A1180B4493D
:10C58000B24A09883980118090F85A01C00702D058
:10C59000B348006830B9A8480188AA4801803888A3
:10C5A000ACF80000AA48BCF90020B0F90010B7F9B7
:10C5B0000000F6F7C3FCAB490880BDE8F88FAA4A33
:10C5C00010B51268537D127D5B1C534307E000BF1A
:10C5D00030F912408C4201DD012010BD521C9A42FC
:10C5E000F6DB002010BDF0B59F4B1B685D7D1C7D08
:10C5F0006D1C654323460DE093FBF4F604FB1636F1
:10C6000030F9137076B28F4203DD964201DB0120D0
:10C61000F0BD5B1CAB42EFDB0020F0BDF0B5924CEF
:10C620002468657D267D6D1C7543344614E000BF8B
:10C6300094FBF6F706FB17477FB2BA420BDCBB420E
:10C6400009DB30F914708F4203DCC1F1000C67453F
:10C6500001DA0120F0BD641CAC42E9DB0020F0BD32
:10C66000814A10B51268537D127D5B1C534306E06E
:10C6700030F912408C4201DD012010BD521C9A425B
:10C68000F6DB002010BD2DE9F05F814677480E46AD
:10C6900015460068002482464FF408610BF0A3FCA5
:10C6A000002028607048834601680A7D497D491C46
:10C6B000012718E0DBF8000001EB01130AEB430C43
:10C6C000007D401C0DE000BF36F91230521C4B4576
:10C6D00007DD0CF80070D5F80080641C4344A4B258
:10C6E0002B60401EF0D1491EE4D1204626E670B5ED
:10C6F0005D4B1B685C7D1B7D641C5C43002506E074
:10C7000030F91360964201DA21F813505B1CA34202
:10C71000F6DB70BD2DE9F04F534A82468B46106818
:10C72000477D057D6F432DE0D2F800C007EB05097A
:10C730000AEB49019CF8153000201C4688465B1C1A
:10C740000CE000BFB1F90060002E1BDD08B186428D
:10C7500000DA30469CF81460A1EB46015B1EF1D173
:10C7600000280FDD0BEB4901641C09E0B8F800302C
:10C770001B1A0B8013681B7DA8EB4308A1EB430138
:10C78000641EF3D16D1ECFD2BDE8F08F2DE9F043CA
:10C79000354E3468627D02F1010994F83C2352065B
:10C7A00017D594F84423642A03D194F83A33642BC0
:10C7B0000FD094F83A33642B02D31A44C83A02E0FB
:10C7C000642A05D9643A002A02DDC2F1640300E05C
:10C7D0006423227D66E0376897F83C4364061FD5E2
:10C7E00097F83B5395420CDD97F84473541C643F13
:10C7F000674397FBF5F46D1E1C4495423FD12346D9
:10C800003DE03C7DA2EB050C641B97F83A530CF11C
:10C81000010C643D05FB0CF595FBF4F41C442EE083
:10C8200097F844533C7D642D22D9C5F164055543E6
:10C8300095FBF4F422E00000220410002404100010
:10C8400020041000260410002A0410002C041000FC
:10C85000280410002E04100056021000A802100038
:10C860009C0100221E04100028021000700210001B
:10C87000643D05FB02F797FBF4F42C1B64344D4632
:10C880004FF064080CE037683F7D05FB072C30F95A
:10C890001C70002F04DD674397FBF8F721F81C702C
:10C8A0006D1EF0D1521E96D2BDE8F0832DE9F04FF7
:10C8B000FB4AB0B08B4682460021FA4D20AB10688F
:10C8C00019E000BF90F85C7390F85B63641EBF1BB7
:10C8D0004F43BF0197FBF4F404EB861424B223F812
:10C8E0001140A41123F8114090F8F167232E01D1D3
:10C8F00025F81140491C90F85A438C42E2DCE1B221
:10C9000021E000BF90F85E7390F85D43A7EB040C44
:10C9100090F85A73A1EB07080CFB08FCF61B4FEAD2
:10C920008C1C761E9CFBF6F606EB841424B223F8CE
:10C930001140A41123F8114090F8F167232E01D182
:10C9400025F81140491C067D8E42DBDC9146427D74
:10C95000F1B2521C6C4664253AE00846D9F800C092
:10C960001DE000BF44F8205033F91060642E08DD4C
:10C97000C6F16406571E7E439CF8157096FBF7F6C9
:10C980000AE0643EA2F1010806FB08F79CF8158056
:10C9900097FBF8F8A6EB0806643644F82060401EC2
:10C9A000E0D29CF8140050430AEB400C0BEB40071C
:10C9B00008460BE03CF91060002E07DD54F820809B
:10C9C00006FB08F696FBF5F627F81060401EF1D23C
:10C9D000521EC2D130B0D7E62DE9F043B04C8946A3
:10C9E0002268517D157D491C2BE0226892F8453361
:10C9F000642B07D9C3F164034E1E7343567D93FB2A
:10CA0000F6F306E0643B4E1E577D5E4396FBF7F659
:10CA10009B1B127D64334A4300EB420709EB42063D
:10CA20002A464FF064080AE037F912C0BCF1000F43
:10CA300005DD0CFB03FC9CFBF8FC26F812C0521E23
:10CA4000F2D2491ED1D12FE72DE9F04F944C824606
:10CA5000521E20688B46437D007D03F1010943434C
:10CA6000861838E019180AEB41050BEB41074946D7
:10CA70002EE03278642A0CD9C2F16402A1F1010CD3
:10CA800002FB0CF2D4F800C09CF815C092FBFCF23B
:10CA90000CE0D4F80080643AA1F1010C98F81580FC
:10CAA00002FB0CFC9CFBF8FCA2EB0C02B5F900C0ED
:10CAB0006432BCF1000F05DD0CFB02FC64229CFB20
:10CAC000F2F23A802268127DA5EB4205A7EB4207FD
:10CAD000491ECED1761E401EC4D255E6F0B5704E2A
:10CAE000521E3468237D647D03FB04F500EB45078B
:10CAF000224401EB4505641C27E018461CE0117830
:10CB0000642905D9C1F16401414391FBF3F106E0C9
:10CB1000643901FB00FC9CFBF3FCA1EB0C0137F931
:10CB200010C06431BCF1000F06DD0CFB01FC642178
:10CB30009CFBF1F125F81010401EE0D23068521E27
:10CB4000007DA7EB4007A5EB4005641ED5D1F0BDE5
:10CB50002DE9F047524E8946002732683D463C4653
:10CB6000137D517D9846491C4246B2460DE00E4663
:10CB700009E000BF06FB032C30F91CC0BC4502DDF8
:10CB80006746D5B2F4B2761EF4D1521EEFD244E01D
:10CB9000002637460B46DAF800C00CE09CF814205B
:10CBA00003FB028230F91220164436B2002A00DA62
:10CBB00052423A4417B25B1EF0D197FBF1F396FB59
:10CBC000F1F21BB29A1A12B2002A00DA52429CF811
:10CBD0005F63B24221DD0A461DE0A84507D1A242AB
:10CBE00019D0661CB24216D0661EB24213D0A242C1
:10CBF00002D16E1CB0450ED0A24202D16E1EB045CD
:10CC000009D0DAF80060367D02FB068630F816702F
:10CC1000FF1A29F81670521EDFD1B8F10108B7D2F9
:10CC2000BDE8F0877CB504461F49F6F75AFA1F495C
:10CC30002046F6F79EFA1A4C1D4D206890F83414E1
:10CC400001F00F0690F81A1489073BD5427DB0F920
:10CC50002E14CDE90012B0F92C34164A16491248A8
:10CC6000F7F76AFA2068027DB0F93214CDE90012B4
:10CC7000B0F93034114A12490C48F7F75DFA2878B8
:10CC8000009020680B493346427D0846FAF76CF95C
:10CC900028780090206809493346027D084620E044
:10CCA0002802100000DB012050B30120C8B301208E
:10CCB0006C0210007012100048B40120AC12100079
:10CCC00084B4012029780091427D3346F849F9481F
:10CCD000FAF74AF92878009020683346F649027D31
:10CCE000F648FAF741F9002028702068F44AF5491F
:10CCF000437DEF48FAF779F92068F249F24A037D5B
:10CD0000407D01EB4001EC48FAF76FF9EF480078FD
:10CD100040070FD52068017D407D08444100E94867
:10CD20000AF04BF8EA498880BDE87C4010210520D4
:10CD3000F3F7B2BB7CBD2DE9F0478946DDE908A7D2
:10CD4000C7F1100C1D461CE039F9151056460C466B
:10CD50000AE000BF03FB065830F91880884500DA66
:10CD60004146A04500DD4446761EF3D2611A09B261
:10CD700032F9154079430CFB041141F30F1122F8ED
:10CD800015106D1EE0D247F6FF71184605E000BF92
:10CD900032F910408C4200DA2146401EF8D204E0FD
:10CDA00032F81300401A22F813005B1EF8D237E75E
:10CDB00070B5049C0DE000BF31F8145030F81460D9
:10CDC000AD1B32F914602DB2AE4200DB354623F8BC
:10CDD0001450641EF0D270BD2DE9F04F894607460D
:10CDE000DDE9091E0020064609B1BA4D01E0B94D42
:10CDF00040350021A2F1010236E000BF05EB410CF5
:10CE000035F81140BCF802C007EB4108A4EB0C0454
:10CE10000FFA84FC37F81140B8F80280A4EB08043C
:10CE20000FFA84FA09EB410439F811806488A8EB01
:10CE300004040FFA84FBBCEB0A0401D5C4F100041E
:10CE40000FFA84F8BCEB0B0400D5644224B2984579
:10CE500003DDA8EB030C664436B29C4202DDE41A03
:10CE6000204400B2491C09B29142C7DBAEF8006011
:10CE70008AE42DE9FF5F044697484FF000084FF021
:10CE8000010AD0F800B0ADF80880ADF80C809349E5
:10CE90002046F6F726F992492046F6F76AF9914CB2
:10CEA000206890F8C112490654D590F8BE1201F0DE
:10CEB0000F02C1F30111CDE90012437D8A4A87496F
:10CEC0008A48FFF738FF206890F8BE1201F00F0281
:10CED000C1F30111CDE90012037D854A80498548DF
:10CEE000FFF729FF206890F8BF22642A0CD07E4902
:10CEF000437D0846F7F71AFA20687D49037D90F8CC
:10CF0000BF220846F7F712FA20687B4D407DB5F93D
:10CF1000001042004843754901EB40006F490AF098
:10CF2000E3FF2068B5F90010007D420048437149D5
:10CF300001EB40006A490AF0D7FF2888401C00B284
:10CF40002880216891F8BE12C1F30111814201D1FC
:10CF5000A5F800800320F3F790FB2068674EDFF808
:10CF6000A09190F8B811090761D599F80020B0F99F
:10CF7000D631B0F9D811B0F9DA71B0F9DC51012A23
:10CF80000BD190F85A221344114490F85B221BB243
:10CF900017442A4409B23FB215B290F8BA21407D35
:10CFA0005207CDE90010002A564A57494B480CDA7F
:10CFB000F7F72DF920683B46544A007D5449CDE9E6
:10CFC00000504748F7F723F90BE0F7F7B5F820686A
:10CFD0003B464E4A007D4E49CDE900504048F7F7A8
:10CFE000ABF83078009020685B464A49427D45485E
:10CFF000F9F7BAFF30780090206847495B46027D18
:10D00000424800BFF9F7B0FF86F800802068434E21
:10D01000454690F8B9118A0701D53278BAB190F82F
:10D020008026520702D53278012A10D087E0317865
:10D030000091427D5B4637492848F9F795FF3078E3
:10D04000009020685B463449027D2548DAE74907AD
:10D050006BD590F8BA11427D49070029B0F9EF115C
:10D06000CDE90012B0F9ED312D4A27491B480FDAFE
:10D07000F7F7CDF82068027DB0F9F311CDE9001281
:10D08000B0F9F131274A22491548F7F7C0F856E0C0
:10D09000F7F752F82068027DB0F9F311CDE90012DC
:10D0A000B0F9F1311F4A1A490D48F7F745F846E043
:10D0B0007012100050B30120AC121000C8B3012050
:10D0C00048B40120C4B4012084B40120C00410007D
:10D0D000242510003CFE010004041000100801206B
:10D0E0004C080120280210007C0A012008090120B8
:10D0F000B80A0120BC09012032021000E50310002B
:10D10000F7031000D84C10006C040120144D1000DF
:10D11000A8040120740B0120B00B01206202100052
:10D12000544D1000904D1000FFE73C22F849F9489B
:10D130000AF0DAFE4022F849F8480AF0D5FE2068E5
:10D1400090F8B911890701D5317831B190F880167E
:10D1500049077BD53178012978D190F8C112490669
:10D1600003D599F8001001297ED0ED4900274FF032
:10D1700001080978012916D090F88016490717D5BB
:10D180003178A9B1CDE90085437DB0F8AC26E549F9
:10D19000E048F9F77FFFCDE9008507462068037D69
:10D1A000B0F8AC2614E0CDF80080CDF804800CE097
:10D1B000CDE90085437DB0F8F521DA49D548F9F786
:10D1C00069FFCDE9008507462068037DB0F8F521A9
:10D1D000D549D248F9F75EFFDFF850B3012801D0F6
:10D1E000012F31D1206890F8BA1189067ED502AAA4
:10D1F000CDE90082B0F86432427DCD49C948FFF7DD
:10D20000EBFD804603A8CDE900502068C949B0F87D
:10D210006432027DC448FFF7DFFD216891F8BA212E
:10D22000920675D5BDF90830BDF90C70B1F86622CB
:10D230003B441344404483426ADC91F88006400733
:10D2400002D53078012863D0ABF80850206890F8F8
:10D25000C112490603D599F8001001297AD0437DFF
:10D26000B04AB549B24800E074E0F9F7BEFE206864
:10D27000AD4AB249037DAF48F9F7B7FE0320F3F793
:10D2800017FA206890F81011C9063DD5AC49097805
:10D29000890739D0407DA6494200AA480AF024FEF9
:10D2A0002068017D407D4A00A64901EB4000A1496C
:10D2B0000AF01AFE2068A049407D4200A2480AF008
:10D2C00013FE2068017D407D4A009F4901EB40002C
:10D2D0009A490AF009FE2068017D407D084441001A
:10D2E000984809F06AFD994D688000E010E02068D8
:10D2F000017D407D08444100934809F05EFD28808F
:10D3000010210520F3F7C8F804B05046BDE8F09F9F
:10D31000BBF80810491C89B2ABF808102268B2F8B3
:10D320005E22914292D9ABF808504FF0000A88492A
:10D330008848F6F71AFD3C227D497A480AF0D4FD68
:10D3400040227C4978480AF0CFFD42F21800FBF7F2
:10D350004EFA7BE7407D0090774B7F4A71497448D5
:10D36000FFF726FD2068754B7C4A007D00906E49D2
:10D370007048FFF71DFD81E7F0B5794E00231D468B
:10D3800036681C46777D05E030F914C0944500DD11
:10D390005B1C641CA742F7DC0020347D06E000BF64
:10D3A00031F91060964200DD6D1C401C8442F7DCB0
:10D3B0002B4301D00120F0BD0020F0BDF0B5684E38
:10D3C00000231D4636681C46777D09E030F914C0FD
:10D3D000944503DCC2F1000EF44500DA5B1C641CCA
:10D3E000A742F3DC0020347D09E000BF31F9106072
:10D3F000964202DC5742BE4200DA6D1C401C844259
:10D40000F4DC2B4301D00120F0BD0020F0BD2DE95C
:10D41000F74F82B00024534F009486463A88264640
:10D4200047F6FF702146EAB34D4A0023156895F888
:10D4300015C00EE03EF9132037F813801444A2EB18
:10D44000080212B2904200DD1046914200DA114605
:10D450005B1C9C45EEDC0023DFF80CC12F7D0FE048
:10D46000039A3CF8138032F913201444A2EB08020B
:10D4700012B2904200DD1046914200DA11465B1C68
:10D480009F42EDDCDFF8A4A0384F0022DAF8143018
:10D49000B9469B4647F82340ABEB020707F1140857
:10D4A000142300E026E098FBF3FC03FB1C881E37E6
:10D4B00059F828C097FBF3F803FB1877521C59F86A
:10D4C00027300A2AACEB03031E44E5DBD5F88B2298
:10D4D000B24202DA01238AF80030049A0023B2B182
:10D4E000CAF818300BF10100CAF81400142801DB47
:10D4F000CAF814303C2271461A480AF0F5FC402262
:10D50000194803990AF0F0FC009805B0B0E42FE048
:10D5100010080120544D10004C080120904D1000BF
:10D520005A0210006C040120A8040120B40310006A
:10D53000740B0120B00B0120E80401202405012018
:10D54000C004100040251000BC2510002425100048
:10D5500060A2012080D301207C0A0120B80A0120AA
:10D5600028021000F40A0120300B0120B84E1000F0
:10D570009AF800605246012EB4D195F891729669DE
:10D58000B74215DD081AB5F88F1288420CDC93619A
:10D590008AF800300020494641F82040401C1428F9
:10D5A000FADB012000909DE7761CCAF8186099E725
:10D5B00093618AF8003095E72DE9FF4FFF48002579
:10D5C00081B000689B4691462C4682464FF4086124
:10D5D0000AF009FDFA480021C9F80010016800238B
:10D5E0000E7D012141E000BFDFF8D8C301FA03F24C
:10D5F000DCF800C012EA0C0F34D003EB03170AEB7F
:10D600004702233200920022DFF8BCE323E000BF90
:10D61000DEF8008001FA02F717EA080F19D0029F1E
:10D62000DDF8048037F9167047450BDDDDF800C0E2
:10D630006D1CADB20CF80210D9F800C0BC44C9F89A
:10D6400000C006E0BCF886C0CCF1000CBC4500DD93
:10D650003C44761C521CD0F800C09CF814709742D1
:10D66000D6DC01E03A7D16445B1C07687A7D9A425D
:10D67000BADC002C00DA64422846CBF8004044E7CC
:10D680002DE9F0410546D1480C460178D048007894
:10D6900001434FF0FF300CD0C94E316891F8B921E9
:10D6A000D20706D0CB4A12782AB191F8C12252068D
:10D6B00001D420603CE0C84A1278002AF9D1C74A58
:10D6C000C74B12781B781A43F3D1C64A1278002A46
:10D6D000EFD1497DC44800F0E2FB07463068017D88
:10D6E000C24800F0DCFB804630682B46427DB0F833
:10D6F000C101384401B2BC4800F0F3FB3068234656
:10D70000B0F8C111027D01EB080001B2B74800F08A
:10D71000E8FB206840EA50002060286840EA50009A
:10D720002860206840EA40002060286840EA400005
:10D730002860BDE8F0812DE9F041A14DAB4B0026FA
:10D740002868AB4C90F88726B0F8A61633F912700B
:10D750008F420CDB077D03EB470333F9023C8B421E
:10D7600005DBB0F98416A348FEF73DFF08B126702B
:10D77000DFE7286890F8A8162078814202D9401C7B
:10D780002070D6E79C4840F20542016811430160D1
:10D790009A48016841F4801101602670BDE8F041AB
:10D7A000511F0120F2F778BE70B5854C2068B0F8A3
:10D7B000931190F85C218E1AB0F885228B498A4823
:10D7C000FFF7DAFD05462068002231B2007D401ED9
:10D7D000C3B28848FEF722FF0DB9012803D088495B
:10D7E0000020487070BD2068012290F8871284489C
:10D7F000401CF5F78BFA0128F4D17F48016841F00D
:10D80000050101607D48016841F080710160BDE85B
:10D8100070404FF480610120F2F73EBE2DE9F043E5
:10D8200089466749002480460F68204623463E7D8E
:10D8300017E00025012297F815C00AE002FB063127
:10D8400038F91110A94200DD0D46A14200DD0C4659
:10D85000521C9445F2DAB5F5C87F01DD401C00B2D8
:10D860005B1C9E42E5DCA9F80040BDE8F08330B5C2
:10D87000534A0020014612685C4B40F24C44127D32
:10D8800007E000BF33F91150A54201DD401CC0B2D2
:10D89000491C8A42F6DC30BDF8B500260124ADF8FB
:10D8A0000060FFF7E4FF054669465248FFF7B6FF00
:10D8B00001464348006890F8F12752481E2A07D1D4
:10D8C0001E23038045808180BDF80030C38006811F
:10D8D0001C2D0BD3BDF90030B3F5487F06DA0429BF
:10D8E00004DA1E2A01D1642101810024464D2878E2
:10D8F00054EA000102D0012C09D004E0D320FAF749
:10D9000076FF012C08D0012028702046F8BD0128A0
:10D9100002D1D320FAF76BFF2E70F6E72DE9F34F13
:10D920002D4883B0002700784FF0010810B1374927
:10D9300081F800803648002690F800900670032099
:10D94000F2F79BFEFEF712FD1D4C324DDFF8C8A02A
:10D950002068DFF8C8B090F83C03800614D5304842
:10D96000BAF90020B0F90010BBF90000F5F7E6FAAB
:10D9700003B22C4A2C4900930398FEF7C3F92949B6
:10D980004B4608462A6803E04B4626492A68039816
:10D99000FEF74DFA4B4601AA23492248FEF75AFCEE
:10D9A00005469DF80400DFF85890F8B3206890F819
:10D9B0003C03C00748D0BAF9002038E070021000DC
:10D9C00028021000900210008C0210004F0210007C
:10D9D0004E021000F70310005A021000510210000E
:10D9E0005202100062021000E80401202405012008
:10D9F000CD0210000A64100034021000380210003A
:10DA0000B403100000DB01205D0210004B02100087
:10DA1000400210000404100026041000220410002C
:10DA20002004100080D3012060A2012028E0D84803
:10DA3000B0F90010BBF90000F5F780FAD54A03B23F
:10DA4000D5491046FEF7EBF8D44DD34AD1482968A2
:10DA5000F6F7AFFC0320F2F72BFE206890F83C03AA
:10DA6000800703D529680846FEF754FE206890F821
:10DA70003C03C10619D529680846FEF717FF1AE0CE
:10DA80000320F2F715FE012D0ED1C548D9F810205C
:10DA9000016811430160C348016841F400710160ED
:10DAA000A9020120F2F7F8FCFAE0400703D5296843
:10DAB0000846FEF791FF206890F83C03000703D565
:10DAC00029680846FEF762FE226892F83D03800648
:10DAD00005D5296802F24A620846FEF7B5FF2268BA
:10DAE00092F83D03400605D5296802F22C620846EB
:10DAF000FEF7F4FF216891F8B801C20701D1800751
:10DB000008D5087DA8492A6801EB400102EB4000D6
:10DB1000F6F72BF9206890F83D03C00609D5A34815
:10DB2000007830B1A248007818B929680846FFF794
:10DB30000FF82068DFF87CB290F8A001C0070CD085
:10DB40000498FFF796F940B99BF8000000284BD0E5
:10DB5000206890F8C102400646D49748DFF85CA2DE
:10DB600000780028206807D090F86902C0061BD50D
:10DB70009BF80000B0B117E090F8C202C00703D0D4
:10DB8000FFF78AFE002863D08D48007830B18D48B9
:10DB90008AF80080067000F037F90CE003F036F8E0
:10DBA000074608E0FFF700FE00F02EF986498AF8E4
:10DBB000008081F800802068A24690F881068007E6
:10DBC00005D582480078012801D1FFF7B4FDDFF8C0
:10DBD00000B2804C032F01D03FB10AE0BBF9001026
:10DBE0007148FEF7ECFC20705AE07B480078012871
:10DBF00028D0DAF80000D44690F8C112890701D580
:10DC000076490E7090F82410C90705D02968B0F93C
:10DC100034200846FEF76BFDDCF8000070492A68E6
:10DC2000007DE24601EB400102EB4000F6F79DF873
:10DC3000BBF900106A48FEF7C2FC207005460128B7
:10DC400007D020E06748267006705E480670002006
:10DC50005BE4012764496548FFF712FD6B46644A9F
:10DC60005F49BBF90000FFF7A7FCA9F80600DAF846
:10DC70000000009AB0F888105E48914202DA80F8FD
:10DC8000008000E00670B9F8060000B145B95548BB
:10DC90002670002706705848017809B1491E0170A6
:10DCA000384632E4F8B507460320F2F7E6FC534D58
:10DCB000534E544C286890F83C1389060CD5B0F9A3
:10DCC0007930344A344938460093FEF71BF831491D
:10DCD00023780846326803E023782E4938463268B4
:10DCE000FEF7A5F800202070286890F83C13C907BB
:10DCF00006D0284AB0F9793027491046FDF78FFF42
:10DD0000264C254A23482168F6F753FB286890F8EB
:10DD10003C03800703D521680846FEF7FBFC286812
:10DD200090F83C03C10604D521680846FEF7BEFD05
:10DD300005E0400703D521680846FEF74DFE286838
:10DD400090F83C03000703D521680846FEF71EFD46
:10DD50002A6892F83D03800605D5216802F24A62DE
:10DD60000846FEF771FE2A6892F83D03400605D585
:10DD7000216802F22C620846FEF7B0FE18492068BE
:10DD8000F5F7F3FFBDE8F8400320F2F791BC00007F
:10DD90002004100080D3012060A201207002100036
:10DDA00034021000380210000A64100055021000FE
:10DDB00056021000F70310005A0210005002100023
:10DDC000CC021000E10310004B02100062021000B0
:10DDD0001E041000490210004E02100086021000BE
:10DDE00000DB01204A0210008C021000900210009B
:10DDF000C00310005402100043021000280210005B
:10DE00000404100040021000F848F94B012242714E
:10DE100000211970F74B1A70F74A11700181418186
:10DE200081810222C2810282F44A117081700171E3
:10DE3000C17081717047F24A0229136802D0032928
:10DE40000BD011E093F8BA11C9070DD0B3F8031243
:10DE50000180116891F805120CE0B3F8CA11018035
:10DE6000116891F8E81105E0B3F8C7110180116855
:10DE700091F8BB1181717047C2EB023310B503F604
:10DE8000AA73002207E000BF30F912409C4201DB78
:10DE9000012010BD521C8A42F6DB002010BD10B5D7
:10DEA000044647F6FF70002206E000BF34F9123046
:10DEB000834200DA1846521C8A42F7DB002800DA57
:10DEC000002010BD10B504460020024606E000BF49
:10DED00034F91230834200DD1846521C8A42F7DBC7
:10DEE00010BDF0B50746002005460446012618601F
:10DEF0000DE000BF37F914C0BCEB010C06D41D685F
:10DF000006FA04FC45EA0C051D600125641C9442D8
:10DF1000F0DB012D00D10120F0BD30B50446B0F991
:10DF200000300020012206E034F912509D4201DD4C
:10DF30002B461046521C8A42F6DB30BD2DE9FC5FB1
:10DF40001C461346AE4D30F9132000268946834601
:10DF500000920192B44602FB03F1DDF830A00120EB
:10DF6000D5F800E02FE01F1A10D47EB93BF9175006
:10DF7000BEF8CC81454508DBDDF80080454504DC72
:10DF800005FB07112A44009500E001261F184F45A4
:10DF900013DABCF1000F10D13BF91750BEF8CC8159
:10DFA000454508DBDDF80480454504DC05FB071129
:10DFB0002A44019501E04FF0010C012E05D0BCF17F
:10DFC000010F02D0401C5045CDDDA9F101004243B4
:10DFD00081FB0401D31709F063FF002800DA002059
:10DFE000611E884200DD084600B2BDE8FC9F70B5A6
:10DFF000834A03460020126892F82060D48A158B69
:10E000009E4204DA92F82160A41B9C4200DC0120AD
:10E0100092F822308B4204DA92F82320AA1A8A421C
:10E0200000DC012070BDF0B5754F059E05680C68D9
:10E030003F68F2B195420BDCAA1A00D5524292B267
:10E040007243C2F38F12AD1A012D12DA012510E0CE
:10E05000B7F818C0ACEB0202AA420ADCAA1A00D533
:10E06000524292B27243C2F38F121544AC4500DAA9
:10E070006546E3B19C420BDCE21A00D5524292B2F3
:10E080007243C2F38F12A41A012C10DA01240EE09D
:10E09000FF8AFA1AA2420ADCA21A00D5524292B2B0
:10E0A0007243C2F38F121444A74200DA3C46056063
:10E0B0000C60F0BD17B581B01446DDE90101FFF732
:10E0C00096FF00281AD102A901A8F5F71FFF4C48B6
:10E0D000006890F8B811C90609D500F5EF7001790C
:10E0E00000914388028802A901A8FFF79CFF0198CC
:10E0F000608002982080204606F0B8FB1FBD2DE905
:10E10000FF4F3F4C8B4681B020681E464FF0000AFF
:10E1100090F8B811890631D53A490A7E72B30025C4
:10E12000894626E0374920681A3119F805704A5D9A
:10E1300090F8C91101F00F010091C38A017D584682
:10E14000FFF7FCFE804620683A4690F8C91101F0BE
:10E150000F010091038B417D0198FFF7EFFE01460F
:10E160006FF063007081318132464046FFF7A2FFB5
:10E170006D1C99F81810A942D4DC2AE0017D58469C
:10E18000FFF7CBFE05462068417D0198FFF7C5FEED
:10E19000074620682A4690F8C91101F00F01009146
:10E1A000C38A017D5846FFF7C9FE054620683A46F6
:10E1B00090F8C91101F00F010091038B417D019886
:10E1C000FFF7BCFE75810146308132462846FFF7D5
:10E1D00071FF206890F8F107182803D10A49C88D0B
:10E1E000401CC88505B05046BDE8F08FE003100024
:10E1F0004E0210004F021000500210005302100097
:10E2000028021000D653100000DB01202DE9F04F4A
:10E21000ADF51D7D002520216FA8999509F005FF1A
:10E220003C2140A809F001FFA84620216FA809F071
:10E23000FCFE3C2140A809F0F8FEFE4C93A8217892
:10E24000FFF7F9FDFC48DFF8F4A3FD4A0068CAF8BF
:10E25000000000F58861116012AB7BAA01211295C4
:10E26000FAF751FE0546F748006890F8F117F648AE
:10E270000A2900D18581F4480E902078022808D020
:10E2800038B1022600274FF001090DF10C0B0124D3
:10E290001EE00A26F6E799A9CDE900B112A800EB25
:10E2A0008402E1B298ABDAF80000FCF7EDFD09FA60
:10E2B00004F010EA080F0AD140A8999950F82720D5
:10E2C0008A4204DA40F827106FA820F81740641C2F
:10E2D000AC42E0D96FA810F8171009FA01F07F1CC2
:10E2E00040EA0808B742D2D3012482E04FF0000888
:10E2F00040466FA907E000BF31F91020A24201D1CA
:10E300004FF00108401CB042F6D3BDF94C129AAA56
:10E3100012A800EB8403CDE90021C948CDF808B06C
:10E3200099460168E2B25746DAF80000FCF7E8FDCA
:10E3300000047BA9000C21F8140059D0B8F1010F9A
:10E3400056D1C1480E900F9002208DF8280005206C
:10E35000ADF81A0041F6583007900720ADF81800C4
:10E3600099A8CDE900B0E1B298AB4A463868FCF70D
:10E370008BFD8046ADF83000BDF86202ADF8440078
:10E38000BDF86002ADF8420003A94846FDF764FB02
:10E39000E1B24FAB4A463868FAF7A9FED9F8000057
:10E3A000099000220321CB20FAF739F903AA494644
:10E3B0004FA8FBF725FBA34F386890F82A01800788
:10E3C00006D5052203A89899FBF748FBADF846004F
:10E3D00003AA49464FA8FBF7E8F903A806F046FA56
:10E3E000386890F8F107062802D1974820F8148081
:10E3F000641CAC427FF67AAF924C206890F8F1171B
:10E40000062916D1007D904D420005EB40008F4952
:10E4100009F06AFD00208E4A216807E00B7D461C4A
:10E4200032F810707343401C25F813704B7D834203
:10E43000F4DC206890F8F107182803D18248818D18
:10E44000491C81850DF51D7DCEE6F0B500242546DD
:10E45000264610E030F91670974207DD1BB1D3F85D
:10E4600000C067441F60641CE4B203E0AC4200D902
:10E4700025460024761C8E42ECDBAC4200D82C46AC
:10E480002046F0BDF0B5441C4D1CD38966195C4391
:10E490005D4364006D00B4FBF6F4B5FBF6F5401C7B
:10E4A00003FB00F6491C47184B4376005900B6FBA6
:10E4B000F7F0B1FBF7F180B289B2AC4202D9D08358
:10E4C0001184F0BDD1831084F0BD2DE9FF4F5D4D67
:10E4D000604E91B028684FF000091E9F90F82510FB
:10E4E0009B464A0731684C4641F480514FF0020880
:10E4F00014D58DF81C80022F37D13160B0F8D026AA
:10E50000417D00231198FFF7A0FF28680023B0F891
:10E51000D026017D1298FFF798FF26E0022F24D124
:10E520004D4A1278012A01D190F87F403160B0F84D
:10E53000D026417D00231198FFF787FF8246286887
:10E540000023B0F8D026017D1298FFF77EFF2968DE
:10E550000AFB00F091F87D102144814203D2032090
:10E560008DF81C0001E08DF81C80BBF1010F47D035
:10E5700000200F9028680FABB0F8D026417D11988D
:10E58000FFF763FF044628680FABB0F8D026017D83
:10E590001298FFF75AFF014604FB01F0ADF80E0098
:10E5A00000F10100ADF80C000F982C4A4FEAD0039F
:10E5B00000F101004FEAD000CDE904031088022FDA
:10E5C00000F10100ADF8240001D08DF81C806A46EE
:10E5D0002046FFF757FF286890F82A01800702D5E8
:10E5E0000598ADF83A0011AC6B4607CCFFF787FDF4
:10E5F0008146306840F400503060484615B0F3E57D
:10E60000FFF704FEF9E72DE9F34F154815490068B7
:10E61000096840EA400041EA410141EA510140EA0B
:10E62000500041EA410140EA400041EA510A40EA13
:10E63000500719E05B02100070021000AC031000DC
:10E64000B00310002802100000DB01202405012087
:10E65000E804012068021000560210002004100097
:10E660008C02100090021000FE4800210468667DB4
:10E67000257D761C012083462EE000BF009B00FB19
:10E6800005F203EB420CDFF8E09300231A4649F849
:10E690002030431E0BFA03F303EA0A0E19E000BF11
:10E6A0000BFA02F919EA070F02D0BEF1000F0FD1E1
:10E6B0003CF91280019B98450ADDEB4BDFF8A883FB
:10E6C000491C53F8203089B243EA090348F8203046
:10E6D000521CAA42E4D3401CB042CFD394F8F107B5
:10E6E000182801D1E148018494F8E701884202D258
:10E6F0000120BDE8FC8F0020FBE72DE9F34F8146A8
:10E70000D848002681B007684FF0010A6FF0004436
:10E7100097F8BA013546000772D54FF4F061D44836
:10E7200009F061FC387DCF4942000120D04B07E061
:10E7300002EB000839F818C023F815C06D1C401C06
:10E7400097F814C0ACF1010C8445F1DC7A7D387D7A
:10E75000521E4243012098468B4606E0131839F8B2
:10E76000133028F815306D1C401C397D491E81423C
:10E77000F4DC0020024601460090EBB2BC48F4F7FE
:10E7800091FADBF8007097F8BA01000738D5B9495B
:10E79000002097F856B20978012903D197F857223B
:10E7A000ABEB020B05EBD57121F0010232F9081039
:10E7B000029A00918C18022297F815E011E03B7D37
:10E7C000012103FB02F55B1E08E000BF05EB010819
:10E7D00039F918C0A44500DD401C491C8B42F5DC0A
:10E7E000521C9645EBDC584501D94FF0000A97F8CA
:10E7F000F11718292AD19D49009ACA842FE0FFE712
:10E80000984902200D6895F815C013E02A7D012172
:10E8100002FB00F7521E0AE007EB010839F9183035
:10E82000B34200DD1E46A34200DA1C46491C8A4260
:10E83000F2DC401C8445E9DC0299301B884201DD92
:10E840004FF0000A95F8F117182906D0854800689E
:10E8500090F8F1070A2804D008E08449CC840885A0
:10E8600004E08248311B8184A0F826A05046BDE810
:10E87000FE8F30B5044600200246A1F101010DE0F3
:10E8800004EB420534F91230B5F902505B1B00D598
:10E890005B421BB2834200DD1846521C8A42EFDB0A
:10E8A00030BD2DE9F04F6F4A8B460021D2F800A011
:10E8B000DFF8C4C102239AF81520A2F101092AE069
:10E8C0009AF814400122A4F1010620E003FB04257C
:10E8D0002DB2A5EB040730F8158000EB45053FB2DB
:10E8E0006D88A8EB05050FFA85F83CF817500CEB7E
:10E8F00047077F88A5EB07052DB2B5EB080500D5C6
:10E900006D422DB2A94200DA2946521C12B296423B
:10E91000DCDC5B1C1BB29945D2DA594501DD0020D5
:10E9200062E4012060E4F0B54E4E3468657D247DDC
:10E930006D1C654300241C609C80DC803468247D51
:10E9400016E000BF30F91460002E10DA1F683E4454
:10E950001E6030F914608E4202DA9E88761C9E801A
:10E9600030F91460964202DADE88761CDE80641C80
:10E97000AC42E7DB1868002800DA40421860F0BDBE
:10E980002DE9F843374C0E46034621680027904690
:10E9900091F8C10245063948027803D53848007815
:10E9A000012804D0B1F80102012A07D00AE0B1F829
:10E9B000BA02012A06D1B1F8BC1201E0B1F808127E
:10E9C000084480B201B21846FDF7F9FD05462068FB
:10E9D0006B46427DB0F90A123046FFF782FA0646CE
:10E9E00020686B46027DB0F90A124046FFF779FABB
:10E9F00025B9012E02D1012800D10127216891F803
:10EA0000F117182908D119494A8B521C4A83AA00C8
:10EA100042EA460202438A833846BDE8F8832DE97C
:10EA2000F34FDFF850A087B00E4600279AF8004059
:10EA300014480C490497059702780868022AB0F830
:10EA4000F72128D0039290F8F9210292B0F8FA2128
:10EA500090F8BA11DFF830809346090731D590F865
:10EA6000B91113E0280210006C52100000DB0120E5
:10EA7000B02610004E021000BCF901005302100035
:10EA8000F70310005B02100050021000090718D4B1
:10EA9000B0F9581225E0B0F8FC31A2EB030292B2B3
:10EAA000039290F8F92190F8FE31A2EB0302D2B262
:10EAB0000292B0F8FA21B0F8FF31A2EB030292B251
:10EAC000C6E798F8001049B1B0F9D41190F8B9012F
:10EAD000000706D5FC48FFF7E4FE05E0B0F9D211C7
:10EAE000F4E7F948FFF709FE0546404698F800109C
:10EAF000DFF8D8834FF00009012903D1494680F897
:10EB000000901DB1F248017819B114E0F04801708D
:10EB100001E0012D0CD0A8F80C909AF8002049468D
:10EB20004046012A27D00289D2B10278BAB117E053
:10EB30009AF8001011B1A8F80C901DE0B8F80C205C
:10EB4000E44B521C92B2A8F80C201B6893F8E531F4
:10EB5000934211D2A8F80C90012101700CE00181C0
:10EB6000DD4888F80010B0F900100798FFF74BFD5A
:10EB70000125012800D10025D648006890F8B91178
:10EB8000090605D5012E03D19AF80010012902D0FB
:10EB9000012D09D002E0012D00D1002590F8BA1115
:10EBA00009075ED5F6BB90E090F8B801000609D5DC
:10EBB0002EB99AF80010012901D18AF80090384640
:10EBC00009B0ADE6C548C64AC6490378C648FFF74E
:10EBD000D7FE844601280CD1BE486B460068B0F8C9
:10EBE000BC01404201B2CBF1000002B20798FFF72E
:10EBF0009AFE022276B10099039881420ADBBDF8A1
:10EC000006100298814205D3BCF1010F02D1B7482A
:10EC1000007840B1B148A8F80E2041460278012A98
:10EC200014D01AE038E0AD49A8F8102040460A7820
:10EC300032B9C289521E12B2A8F80E20002A6BDA2D
:10EC40000120087000240227049065E00A8A521E01
:10EC500012B2A8F81020002A5EDA80F80090002492
:10EC60005AE0B0F8BC01DFF86CC2404201B2CBF10F
:10EC7000000002B26B460798FFF755FE2EB3DCF892
:10EC800000000099B0F8BE2191421EDBBDF80410CF
:10EC900090F8C001814218D38D4AA8F80A909AF8DA
:10ECA0000030127848461A4302D0A8F808000AE05B
:10ECB00088480122006890F8E31184480830F4F78E
:10ECC00025F8012803D1012401E0A8F808909AF85A
:10ECD000000001280CD17E4A854BA8F808901278D4
:10ECE0001B78324349461A4306D0A8F80A1001247B
:10ECF000012D11D06DB10FE076480122006890F827
:10ED0000E41172480A30F4F701F80128F0D1002428
:10ED1000EEE7012C00D101276E48006890F8BA1187
:10ED2000090706D59AF80010012902D10EB1012772
:10ED30003C4690F8B8114A076E4903D50A780AB1E3
:10ED4000012F03D06C4A1278012A01D100273C46DA
:10ED50008AF8004090F8F1276848142A02D0182A4F
:10ED60000AD02CE0048098F806204280644A127889
:10ED700082800978C18022E0182101800099B1F5D4
:10ED8000004F01DD47F6FF714180BDF8041081801E
:10ED9000C680BDF806100181049941818481C58136
:10EDA000059901824782848298F80620C282554ADA
:10EDB00012780283B8F8081064225143818498F8CD
:10EDC00006004546012801D018B107E034B90820F3
:10EDD00002E0012C02D10720F9F709FD9AF80000A2
:10EDE000A871ECE670B53B490020444A09683D4CE7
:10EDF0000AE000BF0B7D851C6B4334F8106002EB0A
:10EE00004303401C23F8026C4B7D8342F2DC00205C
:10EE1000334C07E04E7D34F8105006FB0303401CD2
:10EE200022F813500B7D8342F4DC70BD2DE9F04FC6
:10EE3000354C864600202768344C4B784FF001094A
:10EE4000CE78D4F800B01AE009FA03F25EF8235045
:10EE50000C7802EA070A91F802C00DE009FA04F200
:10EE60002A4208D0BAF1000F04D012EA0B0F01D0E9
:10EE7000012000E09543641CA445EFDA5B1C9E4230
:10EE8000E2DA4DE52DE9F043104F4278DFF880C01B
:10EE90003B784FF00109C57810E00178847809E0EB
:10EEA0005CF8228009FA01F618EA060F00D0012367
:10EEB000491CC9B28C42F3D2521CD2B29542ECD258
:10EEC0003B70BDE8F083000060A20120E003100069
:10EED0004F021000280210001E0410005302100000
:10EEE00024050120E80401200A64100056021000E5
:10EEF00047021000550210006202100000DB0120E2
:10EF00005B0210003C041000900210008C02100004
:10EF10006C5210002DE9F74F9646FC4A002082B053
:10EF200015680446834695F8B8214FF0010A920708
:10EF300048D5F74A1278E2BB4A7891F803C028E036
:10EF4000029B561C53F822902B7D7343F14E06EB27
:10EF5000430301930B788F7818E000BF0AFA03F699
:10EF6000009616EA090F10D0019E36F91360002EA4
:10EF70000ADBE94EDDF8008056F8226016EA080F39
:10EF800003D04FF0010B00E034445B1C9F42E5DAF4
:10EF9000521C9445D4DA0CB94FF0FF3464220EFBB6
:10EFA00002F1624291FBF2F1B5F8EB218A420CDDED
:10EFB00000E007E0B5F8E921724506DD0120BBF16C
:10EFC000010F02D1D54A82F800A005B0A8E42DE9CE
:10EFD000F04F0026CD4D91468A4683463446314651
:10EFE000304632462D68DFF8388314E01AF8027094
:10EFF00017F0110F04D008EB01163270012608E05B
:10F00000012E06D12FB908EB011672700026491C9B
:10F01000C9B2521CD2B26F7D9742E7D8012E04D1FB
:10F0200008EB0116491C7770C9B2002217E000BF37
:10F0300019F8026016F0110F00D014B1012C05D0A0
:10F040000BE008EB0014A270012406E02EB908EBD7
:10F050000014E2700024401CC0B2521CD2B22E7DBB
:10F060009642E5D8012C04D108EB0014401CE67050
:10F07000C0B200252C461CE0002216E008EB041666
:10F08000C5EBC50796F800C003F807C01F447678A3
:10F090007E7008EB02166D1C96F802C087F802C05D
:10F0A000F678521CFE70EDB2D2B28242E6D3641CF6
:10F0B000E4B28C42E0D3002415E000BFC4EBC402EC
:10F0C00002EB0305AA78EE7809E000BF19F8027098
:10F0D000FF0602D52F797F1C2F71521CD2B29642A7
:10F0E000F4D2641CE4B28442E8D3002413E000BFED
:10F0F000C4EBC4055A5D1D446E7808E01AF802702E
:10F10000FF0602D56F797F1C6F71521CD2B29642F6
:10F11000F4D2641CE4B28C42EAD348438BF80C006E
:10F12000AFE62DE9F04F99B01D4690460E460023FC
:10F13000DDE923215C1ECDE914430793089309936D
:10F140000A9311930B930593129313939B1EA1465D
:10F150000393CA46169400230EE000BF36F91370DD
:10F16000A74200DD3C46012804D1DDF888C0FF2716
:10F170000CF803705B1CDBB24345EFD3022A04D0CA
:10F180006248006800F226200BE0664800780128FB
:10F1900017D15E48006890F8C122520611D500F5DB
:10F1A00004700278B0F806C00A4461448378878806
:10F1B00089B2179141780C91C1780D9192B2018971
:10F1C00012E05248006800F21B200278B0F806C036
:10F1D0000A4461448378878889B2179141780C91F9
:10F1E000C1780D91018992B2009190F80AB004FBA8
:10F1F00003F0642190FBF1F11046F3F79BFE01460A
:10F200003846F3F78FFE07B20D984443642094FB11
:10F21000F0F15846F3F78EFE01460098F3F782FEB0
:10F2200000B20F9025980780B6F90000B84203DDC0
:10F23000287840F00100287001241AE12298DDF8B6
:10F240003CB00057012800D030B90C990BFB01F0FD
:10F25000ABEBE0100FFA80FB1AF1010008D036F991
:10F26000140036F91910884204DD0AF0FF000DE0A1
:10F27000601E0AE036F91A10884202DA09F0FF002F
:10F2800004E051464846F3F755FEC0B236F9141073
:10F2900036F81000081A00B2B94203DD295D41F0CA
:10F2A0000101295536F91410B94205DC06EB440179
:10F2B00031F9021CB94215DD584504DD01204FFA31
:10F2C00084F9149005E0CBF10001884201DA0020B6
:10F2D00014901698401C08D0169801282ED0401C77
:10F2E0002ED04BE04FF0FF30F2E7149840BB19F1FD
:10F2F000010019D036F91910179881423EDD15F832
:10F30000090040F0100105F8091035E0280210004E
:10F31000550210000A6410006C521000E003100047
:10F32000DA501000F7031000B6F900101798814268
:10F3300024DD287840F0100028701DE0149818B1E2
:10F340001498012838D019E036F91910179881421D
:10F3500014DD00BF15F8090040F0100105F8091090
:10F3600036F91A00B84207DD079828B115F80A00E7
:10F3700040F0200105F80A100120159022991498F8
:10F380001690085519F1010020D036F9141036F9FD
:10F390001900814201DD60B281461AF1010022D0DC
:10F3A00036F9141036F91A00814201DA60B2824649
:10F3B0001598012824D02BE036F9191017988142AE
:10F3C000DCDDA8F101008442C4D0D7E706EB44019C
:10F3D00036F9140031F9021C884201DD204600E0B4
:10F3E000601E40B2D8E706EB440136F9140031F94B
:10F3F000021C884201DD601E00E0204640B2D6E7D4
:10F4000007984FF0FF3A401CC0B2079000201590BB
:10F4100036F91400B84211DC06EB440131F9021C44
:10F42000B9420BDD079949B1059A891A012905D11D
:10F4300011A98C540599491C49B20591B84216DCB2
:10F4400006EB4400B0F90200B84210DD079870B135
:10F4500005990898081A012814D008460899884286
:10F4600005D1002903DD09A8084400F8014C641CFB
:10F47000E4B24445FFF4E2AE4FF0FF394E464F464A
:10F48000002441E0089909A844540898401C40B25F
:10F490000890ECE70398401C844233D0285DC007F5
:10F4A0000AD0701C0AD10021601EF3F743FD46B25A
:10F4B000A85D40F00100A855701C16D0285DC1065B
:10F4C00000D50027C00703D0A8F1010084420CD169
:10F4D0007F1C08D1611EF0B2002202E02A54401CB9
:10F4E000C0B28842FADD4E464F46611E0020F3F757
:10F4F00021FD285CC00705D0285D18B901202855DA
:10F5000060B20390641CE4B24445C3D30798022858
:10F510001AD30021FE4F11AA0E4609AC505678B1FD
:10F5200063566BB1D7F800C0181A9CF831C2604519
:10F5300006DA505C02E02E54401CC0B28342FADA74
:10F54000491CC9B20A29E9D30020202105E02A5C20
:10F55000920600D52954401CC0B24045F7D3079805
:10F5600019B08EE42DE9FF4F002081B0834682461A
:10F570000090E848DFF898930678D9F8000090F8F2
:10F58000CF160A092ED04D4609072BD0407D801E8C
:10F5900081B20298801CF7F75EFD296891F8CF26AA
:10F5A000097D120990FBF2F084B20398F7F753FD3E
:10F5B000296891F8CF2602F00F0290FBF2F085B295
:10F5C000AC4201D9204600E02846B1F8F72600B247
:10F5D000824201DA002600E0012691F8DA7691F8FD
:10F5E000DC0606E00EB300F2D26004884588077A94
:10F5F000807A00238046C64822460068417D0298F2
:10F60000FEF723FF8146C24800232A460068017D99
:10F610000398FEF71AFFBE49DFF8FCE2096891F88B
:10F62000F1C7BCF11F0F07D017E000F2D6600488C5
:10F6300045884779C079DCE71F23AEF80030AEF883
:10F640000260AEF80640AEF80890AEF80A70AEF868
:10F650000C50AEF80E00AEF81080B04AB94503D990
:10F66000404501D9002404E0B94501D8404517D9E7
:10F67000012401251570AA4BAA4AA3F80090108016
:10F68000D6B1012C2CD0B1F8DE06B1F9E0764042BB
:10F69000B1F8E26602B24B7D087D5B1C434333E068
:10F6A00000211170BCF11F0F04D1AEF814100099A5
:10F6B000AEF82610009888E4012C08D0B1F8EA06CC
:10F6C000B1F9EC76404202B2B1F8EE66E3E7B1F888
:10F6D000F006B1F9F276404202B2B1F8F466DAE728
:10F6E000B1F8E406B1F9E676404202B2B1F8E86654
:10F6F000D1E7019931F91010914204DA8B440AF1F3
:10F7000001011FFA81FA401C9842F2DBBBF10003B1
:10F7100001DACBF10003BB4203DDB24501D9012080
:10F7200000E00020BCF11F0FC5D1AEF812407146B9
:10F73000AEF81450002A00DA5242CA8242F20F7226
:10F740000A834B838F83CA83A1F820A04E848A84C6
:10F75000C8840A8D521CAEF8282036E410B5002467
:10F760000AE000BF30F91430002B00DA5B428B4214
:10F7700001DD012010BD641C9442F3DB002010BDAC
:10F780002DE9F047894680461C469246002601270F
:10F790004FF4C8716448089D08F025FC5C480021BE
:10F7A000D0F800C0604818E019F8012012F0110FDD
:10F7B00001D0012F04D002F011023A4305D00AE033
:10F7C00000EB06120027117005E000EB061201277E
:10F7D000761C5170F6B2491C49B29CF815208A4239
:10F7E000E2DC1FB900EB0612491E51700123002212
:10F7F000114618E01AF8016016F0110F01D0012B24
:10F8000004D006F011061E4305D00AE000EB0213F7
:10F810009970002305E000EB0213521CD970D2B29C
:10F820000123491C49B29CF814608E42E2DC1BB9EA
:10F8300000EB0212491ED17000231A461CE0002181
:10F8400016E000BF00EB021708EB031697F800C0A4
:10F8500086F800C07F78777000EB01175B1C97F883
:10F8600002C086F802C0FF78491CF770DBB2C9B24B
:10F87000A942E7D3521C52B2A242E0DBBDE8F087B6
:10F880002DE9FF4F22489B468DB0036891461C7DB1
:10F8900093F86A12254609070DD52449244A0968B8
:10F8A000126841EA510646EA4101009142EA5201DA
:10F8B00041EA4201029100263746324601215B7D32
:10F8C0000DE000BF19F802C01CF0110F06D05FEA6E
:10F8D0008C6C03D401FA02FC4CEA0606521C9342DB
:10F8E000F0DC00228A460AE01BF8021011F0110F2A
:10F8F00004D0890602D40AFA02F10F43521C944242
:10F90000F2DC81460B484FF488610068834613E0BF
:10F91000280210005302100000DB0120B404100084
:10F92000B6041000B8041000DA5010009002100065
:10F930008C0210007002100008F055FB002153E00B
:10F940000AFA01FE1EEA060F22D001EB01130BEBAF
:10F950004300233004900020534612E003FA00FCD9
:10F960001CEA070F0BD0DDF838C0DDF834803CF915
:10F9700014C0C44503DDDDF810C00CF80030641C71
:10F98000401CD2F800C09CF814C08445E6DC01E0BD
:10F99000187D0444D9F8002092F86A02000722D5A5
:10F9A000F94BDDF8008000201B780EEA080E16E007
:10F9B000012B11D1BEF1000F06D0DDF808800AFA44
:10F9C00000FC1CEA080F07D1DFF8C0C33CF8158023
:10F9D000DFF8BCC32CF815806D1CADB2401C92F84A
:10F9E00014C08445E4DC491CD9F800304A46587DEF
:10F9F0008842A5DC11B0BDE8F08F2DE9F047002763
:10FA0000E44D994605F11A067B1E2F76BC461C462E
:10FA1000377608E000EB0718B8F80580E04501D913
:10FA2000C4463B467F1C8F42F4D3002B23DB00EB04
:10FA3000031C4FF0010A9CF8007008E012F80780E0
:10FA40005FEAC86802D52F7085F818A07F1C9CF863
:10FA50000180B845F2DA9CF8027008E019F80780D6
:10FA60005FEAC86802D5377086F818A07F1C9CF83A
:10FA70000380B845F2DA4FF0000801292ED95F1C47
:10FA80002CD000270AE0BB4207D000EB071CBCF8D3
:10FA900005C0C44501D9E0463C467F1C8F42F2D3E5
:10FAA000002C1BDB00EB04114FF00203087805E08B
:10FAB000145CE40601D568702B76401C4C788442B7
:10FAC000F6DA887807E000BF19F80020D20601D5E1
:10FAD00070703376401CCA788242F5DACEE6F0B513
:10FAE000AD4B00260C7891F801C01D6810E08B78B2
:10FAF000CF780AE095F814E004FB0E3E30F91EE0E2
:10FB0000BEF1000F00DD76445B1C9F42F2DC641CFA
:10FB1000A445ECDC012A07D0032A05D0B5F806027B
:10FB2000B04207DA0120F0BDD1F80700B5F806129F
:10FB30008842F7DC0020F0BDF0B5984C954E04EB00
:10FB400001142178657805E0575CFF0600D5315433
:10FB5000491CC9B28D42F7D28E4DA1781A35E27890
:10FB600005E05C5CE40600D52954491CC9B28A4210
:10FB7000F7D2F0BDF0B50024069E2546631EC6F3FD
:10FB800007260AE000EB0417D7F80770AF4202D946
:10FB900063B23D460B70641CE4B2A642F2D8002466
:10FBA00021460DE000EB0115D5F80750A54205D917
:10FBB000994203D05F1C01D02C461170491CC9B278
:10FBC0008E42EFD8F0BD2DE9F04F87B0064614A85D
:10FBD0008946B0E882109846DDE912E30024601EF1
:10FBE0008DF818008DF810001198DFF8A8B1924632
:10FBF000012803D0032801D000270EE11A0E684D1A
:10FC0000C8B2022A08D001D302285AD2012A58D0F9
:10FC1000012856D00027D2E00228F5D156F8070F68
:10FC20004346316B32690844316A11448842524676
:10FC30001CDD00210846FFF77FFF434652460321A3
:10FC40000120FFF779FF544802218BF81810006853
:10FC500090F8F1170A2932D1417D037D69220931DB
:10FC6000594325F8112040F209311AE00121002002
:10FC7000FFF762FF4346524602210120FFF75CFF77
:10FC800002208BF818004448006890F8F1170A2900
:10FC900015D1417D037D09315943692225F8112091
:10FCA0006521427D037D09325A4305EB42021181F1
:10FCB000427D007D0932424305EB4200418107B09D
:10FCC00099E6CDE90031CDE9027C734604AA06A984
:10FCD0003046FFF74FFF9DF91800411C19D0C1B203
:10FCE000434652460020FFF727FF01208BF81800FB
:10FCF0009DF918005C46401C0BD09DF91000411C7A
:10FD000007D0C1B2434652460120FFF715FF02203B
:10FD100020762148006890F8F1170A29CFD1417D5B
:10FD2000037D09315943692225F81120427D037D65
:10FD300009325A4305EB42029DF9181011819DF9D1
:10FD40001010B5E7144806EB07110D460068027D58
:10FD5000144800EB4200119AFFF7C1FE012802D0BF
:10FD6000109801282AD12878594605E01AF8002071
:10FD7000D20600D50855401C6A788242F6DA054959
:10FD8000A8781A3116E000004E02100080D301203E
:10FD900060A20120D6531000280210004A4F100024
:10FDA00000DB01200A64100018F80020D20600D5FC
:10FDB0000855401CEA788242F6DA641C7F1C4F45E5
:10FDC000C0DB2CE0FF4806EB07110D460068027D02
:10FDD000FD4800EB4200119AFFF781FE012802D096
:10FDE0001098012818D12878594605E01AF8002003
:10FDF000D20600D50855401C6A788242F6DAA87807
:10FE0000F24905E018F80020D20600D50855401C3C
:10FE1000EA788242F6DA641C7F1C4F45D2DBEB485D
:10FE20008BF8184004764AE7F0B55378002712E0C3
:10FE30005D1C147805EB051609E000BF04EB4605D0
:10FE40006D1C10F805C08C4500D14755641C957891
:10FE5000A542F3DA5B1CD4789C42E9DAF0BDF0B538
:10FE6000D84A136893F8F1270A2A2DD10022D84CDA
:10FE7000D84D13E01E7D02F1010C06FB0CF6875CE9
:10FE800024F816701E7D02F1020C06FB0CF635F804
:10FE9000127004EB4606521C26F8027C5E7D9642E8
:10FEA000E8DC0020CC4D0CE002440E5C24F812602B
:10FEB0005E7D1F7D35F8102006FB0706401C24F8E8
:10FEC00016201A7D8242EFDCF0BD30B504460020DA
:10FED000034606E034F91350954200DD28445B1CCC
:10FEE000DBB28B42F6DB30BDF0B5B64D07460026DF
:10FEF0002868017DB848FDF7E5FF4FF00A0C90FB3C
:10FF0000FCF084B22868417DB248FDF7DBFF90FB2E
:10FF1000FCF0296880B291F80E22A2420FD991F824
:10FF20000F2282420BD264225443B4FBF0F091F8CA
:10FF30000D1280B2814202D90120B87106463046C6
:10FF4000F0BD2DE9F0419F4DA44A002429681278A4
:10FF5000B1F89202012A01D1B1F88B064A7D01B2B3
:10FF60000F469C48FFF7FAFB064628683946027D93
:10FF70009948FFF7F3FB012E01D0012800D101249D
:10FF800097492246A1F13C00FDF741FA012819D119
:10FF90009449002008700320F0F76FFB90493C2241
:10FFA0003C39914807F0A0FF40228D498F4807F067
:10FFB0009BFF0320F0F77CFBBDE8F04140F6170003
:10FFC000F8F715BCBDE8F0812DE9F0477D4A1068CF
:10FFD000037D90F887125B1EDEB2854B0C4693F8CA
:10FFE00000C0BCF1010F01D190F888427B4F3B78F3
:10FFF000012B01D190F88D4604B90C4690F8B91147
:020000021000EC
:100000009146890602D5B0F8895202E079490988FB
:100010008DB2BCF1010F05D0B0F8C121BA46012B59
:1000200003D008E0B0F8C321F8E790F8882690F8EC
:100030008706401EC6B268496648FDF79DF9DFF89D
:10004000A4810746334688F80000002229B25E48A2
:10005000FCF7E4FAD9F800104FF0000591F86912A6
:10006000890608D53FB9012805D16348634900785E
:100070000978084302D0624885702FE56048012264
:100080002146801CF2F742FE0128F6D15D4805703A
:1000900088F8005040F61800F8F7A9FB9AF800001D
:1000A00038B13346BDE8F047002257495748F4F7C6
:1000B0005FBABDE8F04754495448F3F756BE70B5EF
:1000C000404C45492068B0F89E62B0F8A0224148F3
:1000D000FDF774F9054631B23B48FCF7C1FA2168D7
:1000E0004FF0000491F86922120608D5012D06D1BF
:1000F00028B94148414A00781278104302D040485C
:10010000047170BD3E4891F89D120122001DF2F766
:10011000FDFD0128F5D13B4831493C2204703148AE
:100120003C390470304807F0DFFE40222C492F484C
:1001300007F0DAFEBDE8704040F61900F8F757BB4B
:100140002DE9F00F1F4C00268246246847F6FF7108
:100150003746B446084635460123DFF8789094F8D0
:1001600015800DE03AF913208A4200DA114639F978
:100170001320824200DA1046AA4200DD15465B1CBD
:100180009845EFDCB4F87E228A4200DA0126B4F802
:100190008012814200DA0127B4F88212281A8842BC
:1001A00001DA4FF0010C012E40D1012F3ED1BCF1FC
:1001B000010F3BD1164840F205420168114301602E
:1001C000144829E0280210000A641000F0531000BF
:1001D00000DB0120E8040120240501206202100058
:1001E000B00B0120300210006C040120A804012093
:1001F0004E0210001E0410005102100052021000A6
:10020000E00310004902100060A2012080D3012009
:100210003402100038021000016841F4000101604E
:10022000BDE8F00F511F0120F0F736B9BDE8F00F1F
:1002300070472DE9F041FF4C07460E462068FE4D01
:10024000DFF8F8C390F8B911C90612D590F89317E2
:1002500001F00F02417DFA48FDF70EFE287020687C
:1002600090F8931701F00F02017DF648FDF704FEA8
:1002700001E0002028708CF800002068F24D90F812
:100280006A02C00703D0287808B9FFF75AFE206831
:1002900090F86902000703D531463846FFF750FF52
:1002A0002068EA4E90F86912890601D5297831B1A3
:1002B00090F88006C00706D02878012803D130784E
:1002C00008B9FFF781FE206890F86912090601D588
:1002D000297831B190F88006800708D52878012860
:1002E00005D13078002802D1BDE8F041E7E669E6A3
:1002F0002DE9F04105460027142107F074FED4488B
:10030000CC4C00780028206819D0B0F8C56120686E
:10031000D04B427D6888304401B2CF48FDF7E1FD03
:1003200080462068CD4B027DA888304401B2CC487D
:10033000FDF7D7FD0146B8F1010F0ED010E0B0F87F
:10034000C361417DC448FDF7AAFD68802068017D36
:10035000C348FDF7A4FDA880D9E7012900D10127F2
:1003600038462FE62DE9F041164688460746002418
:1003700026E000251FE000BFC4EBC40208EB051017
:10038000D119837891F802C0634512D3C37891F8EC
:1003900003C063450DD80378BA5C934209D3427811
:1003A00049788A4205D8847322462946D020F8F736
:1003B00036F96D1CEDB2707AA842DDD8641CE4B247
:1003C000307BA042D5D8FDE52DE9FF4F82468B4614
:1003D0000020FF22CAEBCA01CD18DDF834E0AA7173
:1003E0000246DFF8509250E0029901EB021191F9B8
:1003F0000E40544547D10C784E7820E08B78641C31
:10040000CF7819E0D9F800C09CF814C004FB0C3C6C
:100410001FFA8CFC3EF91CC0BCF1000F0ADDD1F8BC
:100420000780C444C1F807C0B1F805C00CF1010C45
:10043000A1F805C05B1CDBB29F42E3D8E4B2A64240
:10044000DCD8D1F80730834202D9AA71D1F807006D
:10045000D9F8003093F8F1470A2C14D15E7D1C7D49
:10046000761D66437F4C652724F81670D1F8071077
:100470000A2691FBF6F15E7D1B7D761D06FB0323AC
:1004800004EB43035980521CD2B29BF809109142ED
:10049000AAD895F90610491C02D16420A871002041
:1004A00004B0BDE8F08F2DE9F0470446C0EBC4006E
:1004B0001844164690F906500F462A462146C72092
:1004C000F8F7ADF80020DFF86C9133E006EB00118F
:1004D00091F90E20A2422BD1A84201D1642209E059
:1004E000D1F8072064235A4306EB0513D3F80730ED
:1004F00092FBF3F2A1F80B20D9F8002092F8F13723
:100500000A2B15D1537D92F814C09B1D03FB0CF3ED
:10051000DFF850C14FF066082CF81380B1F80B30AB
:10052000517D127D891D01FB02010CEB41014B80C5
:10053000401CC0B2797A8142C8D89EE52DE9F04FBF
:100540009B46099BC1EBC10423444FF0000C93F977
:1005500006906446DFF8DCA048E000BF0BEB041314
:1005600093F90E508D423FD14C453DD0DAF8005002
:10057000B3F90B6095F83552AE4235DA01255D735B
:100580001D786D1CEEB2002714E09D780AE000BFD4
:1005900006EB061C05EB4C0C00F80C70A3F805707C
:1005A0004FF0010C6D1C93F80380EDB2A845EFD21B
:1005B000761CF6B25D78B542E7D2DAF8003093F8EF
:1005C000F1570A2D10D15E7D1D7DF61D6E43254D20
:1005D000672725F816705E7D63271B7DF61D06FBD9
:1005E000034305EB43035F80641CE4B2537AA342E8
:1005F000B4D8604655E72DE9FF4F4FF00008FBB037
:1006000092464646DFF82CB08EE07E9800EB06144A
:100610007C9894F90E10814278D102A84790A07876
:100620008DF80800E0788DF80A004FF00009207876
:100630001AE00000280210005102100052021000BF
:100640006C040120A804012062021000F7031000CE
:100650005502100090021000E80401208C021000E6
:100660002405012000DB01208DF8090060788DF859
:100670000B0002AB2FAA49467B98F8F744FC0746CB
:10068000DBF8000090F8F1170A290FD1427D017DB7
:1006900008324A43FE49682321F81230427D007D2A
:1006A000083202FB006001EB40004780012F39D97E
:1006B000F8485490A0788DF80800E0788DF80A008A
:1006C00020788DF8090060788DF80B00012519E07D
:1006D00059AB2946479A7B98F8F709FD49AA59A8CA
:1006E0004799F9F78DF94E99494501D98946A846A8
:1006F0002FA8B4F8051030F815006D1C0844A4F8B4
:100700000500EDB2BD42E3D9012409E00AE0A045AD
:1007100004D02146479A7B98FFF786FB641CE4B21D
:10072000BC42F4D9761CF6B29AF80900B0423FF602
:100730006CAF7FB0B5E62DE9F84F0446D6481646B3
:100740008B46D0F800A0227B0121C020F7F767FF7D
:10075000207B002846D00027224659463046FFF726
:1007600001FE0025DFF82C83DFF8309317E03346D5
:100770005A4621462846CDF80080FFF725FED9F8D5
:100780000010B1F83212814207D2C5EBC5003044E7
:100790008079642801D07F1CFFB26D1CEDB2207BF4
:1007A000A842E4D8C0B2B8421CD80120E0740025A9
:1007B00015E033465A4621462846FFF774FE5B464D
:1007C0002246294650460096FFF7B8FE5B46224671
:1007D000294650460096FFF70EFF6D1CEDB2207BB8
:1007E000A842E6D8BDE8F88F2DE9F34F8146AA4824
:1007F000FDB0002600686B90A6487790DEE000BF51
:100800007E994FF0000B01EB0614CDF828B1C4F827
:1008100007B0A4F805B0A0788DF80000E0788DF856
:10082000020020788DF8010060788DF803006B4697
:1008300030AA00216B98F8F766FB07469748D84620
:10084000006890F8F1170A290FD1417D027D083127
:1008500051438F4A682322F81130417D007D0831D1
:1008600001FB006002EB40004780012549E00020C9
:100870007190A0788DF80000E0788DF80200207863
:100880008DF801006078EA468DF80300E9B24BABC1
:1008900052466B98F8F72BFC00220521CB20F7F786
:1008A000BEFE6CAA51464BA8F9F7AAF8D4F8070087
:1008B00071990DF1C00A0844C4F807003AF8151000
:1008C00099F8060081420ED308F1010000F0FF08FC
:1008D0002079401C207171994A98814208D905F00D
:1008E000FF0B4A9104E0E9B26A466B98FFF79CFA65
:1008F0003AF81500B4F805106D1C0844A4F805007A
:100900006DB2BD42B3DDB8F1010F34D9012530E03D
:100910005D452CD0B8F1010F29D92079012826D9BD
:100920005E48006890F8F1170A2914D1417D027DD4
:1009300009315143564A692322F8113090F815C005
:10094000007D05EB86030CF1090C0CFB003002EB7B
:10095000400066218181E9B26A466B98FFF764FA2C
:10096000A8F1010000F0FF082079401E20716D1CE5
:100970006DB2BD42CCDD99F80A1001EB080089F890
:100980000A004648006890F8F1170A2914D1427D00
:10099000017D521D4A433E49652321F81230D4F8A7
:1009A00007200A2392FBF3F3427D007D521D02FBD8
:1009B000006001EB40004380761C76B299F8090094
:1009C000B0423FF71DAFB4E610B50228049C0FD12A
:1009D0003248C3F30741006890F80C22914209D8CD
:1009E00090F82510490703D52D490978012901D030
:1009F000002010BD2849007D264A096801EB40010E
:100A000002EB4000F3F7B1F900202070012010BD87
:100A1000F0B5224905460020C3F3072669241C4A85
:100A20000968012E03D01DD903461E4D5BE0022D3F
:100A300019D0012D16D191F8BA315B0612D591F873
:100A4000F13701200A2B0DD14B7D0D7D09336B430E
:100A500022F8134021244B7D097D09334B4302EBDF
:100A600043018C80F0BD104B1B78002BFAD00F4B4C
:100A70001B78012BF6D191F8F13701200A2BF1D127
:100A80004B7D0D7D09336B4322F813402C24E2E7A4
:100A900000DB01200A641000700210002802100020
:100AA0003C0410004A4F100055021000560210007E
:100AB00005EB03173F79012F13D991F8F1070A28A5
:100AC0000DD1487D0B7D09305843582322F8104042
:100AD000487D097D0930484302EB400083800120B6
:100AE000F0BD5B1CDBB29E42E2D8F0BD2DE9F043C5
:100AF000FF4D8846914628680026374690F8D9422F
:100B0000017D2246FB48FFF7E0F98446286822462B
:100B1000417DF948FFF7D9F910EB0C04F74831464D
:100B200003D00278012A02D004E0017002E02A68B2
:100B3000B2F8DA622A68D2F8D5329D1BF04BA54292
:100B400007D24FEA1864012C03D109F0FF04012CED
:100B500008D0017092F8C102800700D5197038469C
:100B6000BDE8F08301240470E648032701761A30BB
:100B70000176E548017092F8C1028007EFD51C703C
:100B8000EDE7090E05D0D2B2012A02D9DF48FFF7FE
:100B9000ABB9DE4800210160416070472DE9F041AA
:100BA0000746C07C00261C460D46012826D0384644
:100BB000FFF71AFE787A012826D9002222E000BF2A
:100BC00005EB0211097901291AD901212170C849BF
:100BD0000020096891F8F1270A2A0FD14B7D0A7D80
:100BE00009335343CA4A692422F813404B7D097DD7
:100BF000582409334B4302EB43018C80BDE8F0815C
:100C0000521CD2B29042DBD83046F7E72DE9F04FC4
:100C10008FB04FF000092021BE4807F006FABD480A
:100C20002221203007F001FABA484FF4C87142304F
:100C300007F0D9F9142107A807F0F7F9B148002403
:100C4000B038AB4D0460848084712868DFF8C0A29E
:100C5000B14A007D0AEB400102EB4000F3F785F852
:100C6000A549AE48FFF7E5FA2868DFF8B4B20DF100
:100C70002A0690F8B8110BADC9077DD0A9490978AB
:100C800019B190F8C112490676D507A8FFF730FBD5
:100C90000746012804D0A4480078012807D00CE0BA
:100CA00001469D48FDF7BBFE8BF8000005E0394684
:100CB0009948FDF7B4FE8BF80040DFF83482D8F88D
:100CC000000090F82500400708D59848894A8A49CD
:100CD00003789148FEF746FC9549087092480078E1
:100CE000012801D1012F7DD09BF8000000287AD087
:100CF000D8F8000090F8BA01C007F8D0012F71D0E1
:100D00008C4844707F499BF80020BDF81E00F239E2
:100D100003960091CDE90120D8F80000854F7D4B66
:100D2000427D75497878FEF7FCF98DF82300754906
:100D30009BF80020BDF82000D23903950091CDE941
:100D40000120D8F80000A1F577736A49027D787810
:100D5000FEF7E7F98DF8240001469DF82300F2F72D
:100D6000E5F88DF827009DF823009DF824104843EE
:100D7000C2B28DF8252000E01AE20121EE20F7F73B
:100D80004EFC9DF8250000286FD08DF834400020DF
:100D90005D4903908DF83040012008705D495D4841
:100DA0002031FFF75CF89BF8001007A8FDF743F827
:100DB0009DF82400574A574900909DF8233020326F
:100DC00001F14200FEF7DCFC524BBDF91C00203360
:100DD000504A5149FEF754FDD8F8000090F8BA0186
:100DE000000601E01DE075E103D54F4800780128B9
:100DF00022D0484907A84231FFF7F6FCDDE90A0195
:100E0000CDE9000107AF9BF800000ECFFFF700FE11
:100E10008DF830003648006890F8F1170A2925D07F
:100E200095E04448417829B101297FF46BAF022154
:100E3000417067E70121FBE7324B3649B03BA3F233
:100E4000FE3207A8FEF7C3F82E4A07A8B03AA2F56B
:100E50007771FFF770FC2B4A0CABB03AA2F57771B3
:100E600007A8FFF79BFE0390D4E7FFE0417D027DDA
:100E7000C91C514363232AF81130524600219DF8C2
:100E800025E062E01F4BC1EBC108B03B08EB030952
:100E9000437D90F814C0DB1C03FB0CF303EB8103D0
:100EA00002EB430399F802705F80437D90F814C011
:100EB000DB1C03FB0CF303EB810302EB430399F808
:100EC00003709F800F4B90F814C0B03B13F808706C
:100ED000437DDB1C03FB0CF303EB810302EB4303B9
:100EE000DF80437D99F80170DB1C90F814C023E08B
:100EF0002802100024050120E804012085021000CA
:100F000086021000D6531000B7031000AC02100088
:100F100000DB0120084F10000A641000740B012050
:100F20005B021000F70310004E0210005602100082
:100F30003C041000E003100003FB0CF303EB8103FF
:100F400002EB4303491C1F81C9B28E459AD80DA8F4
:100F50000290DDE90A01CDE900010DF11C085F46B0
:100F6000B8E80E009BF80000FFF72EFD692101286C
:100F70000DD09DF827209DF82600824223D89DF8A9
:100F8000252090421FD89DF83000C8B11BE0B24820
:100F9000006890F8F1270A2A0DD1427D037D0932BD
:100FA0005A432AF81210417D007D3722093141430E
:100FB0000AEB410082809DF834000FB0BDE8F08F4D
:100FC000387801280BD00398012808D0A348047072
:100FD000A148006890F8F1270A2A18D026E09E4818
:100FE000006890F8F1270A2A0DD1437D027D09336C
:100FF00053432AF81310417D007DDE23093141431C
:101000000AEB4100438095490120087029E0437DA7
:10101000027D093353432AF81310417D007D0931C5
:1010200041430AEB410040F24D1343809DF82410E8
:101030009DF82300F1F772FF012800D000208046C0
:10104000142207A902A806F094FF3978844BCDE951
:101050000081A3F120029DF8251002F14200FEF765
:10106000B2FD80484FF00309C470A9E07D4F2246CD
:1010700002217C70EE20F7F7D2FAD8F8000090F841
:101080006A1289070BD59DF8231000299DF82410BA
:1010900001D009B103E011B17349097809B1FC70BD
:1010A0008EE090F89412F878814202D9401CF870D2
:1010B00086E06E48FC70016841F4806101606C4814
:1010C000016841F4800101604FF480610120EFF775
:1010D000E3F975E0D8F80000664A007D0AEB4001AC
:1010E00002EB4000F2F741FE012F69D1D8F8000071
:1010F000414690F8C12253075F4A05D513781BB1CA
:101100005E4B1B78012B05D05C491278097811439E
:101110003FD055E0DFF84C81594B894688F80140B3
:101120009BF800C0BDF81E20CDE9003CCDE90226A9
:10113000427D5F46A3F5777352492046FDF7F1FFE4
:101140008DF823004E493A78BDF8200020310395F0
:101150000091CDE90120D9F80000414B4949427D79
:1011600098F80100FDF7DDFF8DF8240001469DF899
:10117000230000FB01F28DF82520F1F7D7FE8DF852
:1011800027000B9807AF00900FCFFFF7AFFC814609
:1011900016E090F8B811090612D590F8BA01800748
:1011A0000ED50B9807AF00900FCFFFF7EAFC07E0D2
:1011B00035490C7090F8C102800701D5334804709E
:1011C0009BF800105F46022943D12448007801288B
:1011D0003FD1B9F1030F3CD1DFF88880284B0DF1E6
:1011E000040A88F80140BDF81E200093AAE84600D2
:1011F000194E2046A3F5777331684A7D2149FDF7E2
:1012000090FF8DF823001E493A78BDF82000203168
:1012100003950091CDE901203068114B1C49027DF6
:1012200098F80100FDF77DFF01468DF824009DF838
:10123000230000FB01F28DF82520F1F777FE084B23
:101240008DF82700BDF91C00A3F120020949FEF723
:1012500017FB4846B1E6000028021000B703100053
:10126000284F1000E003100062021000340210004A
:101270003C0210000A6410005502100056021000D3
:10128000E4521000E80401204E0210008602100013
:1012900024050120FE48FF4A0068B0F819131180A8
:1012A000FD4990F81B0348817047FB48002181816C
:1012B000C170012101717047F7490020F44AC880CC
:1012C00008814861126892F83F331B090B61F34BA8
:1012D000886188701870F24B186058609860D86008
:1012E000487092F8C002C00703D0EA49B2F8070379
:1012F0004880DAE7F0B5E649E74E096891F83D2302
:10130000D20764D0E54A1778E64A1278AFB1012ACD
:1013100009D091F83F33B1F8584303F00F021D098B
:10132000B1F8563315E091F84133B1F8544303F066
:101330000F021D09B1F852330BE0012A19D091F8C0
:101340003E33B1F84C4303F00F024FEA1315B1F8E6
:101350004A3391F872C05FEACC7C14D0DFF848C3FE
:10136000BCF800C05FEA4C5C20D591F84213CFB9BD
:101370001AE091F84033B1F8504303F00F021D0911
:10138000B1F84E33E5E791F81BC15FEACC7C0DD094
:10139000DFF818C39CF800C0BCF1070F06D191F824
:1013A00043130FB10A0901E001F00F02984201DC7A
:1013B0003261F0BDA04201DB3561F0BDC01AA91A4F
:1013C0004843E11A90FBF1F010443061F0BD002079
:1013D000FBE7AF4930B409680022B1F8CA32834252
:1013E00005D291F8C0321B0701D5032212E0B1F8F3
:1013F000C832834205D291F8C0325B0701D5022280
:1014000008E0B1F8C632834204D291F8C0028007E6
:1014100000D50122A048A14C83789A4219D12278A4
:101420009A4222D0A24D2D782B430FD08269521EB2
:101430008261002A19DC8078207091F81001C006C2
:1014400013D5802130BC0520EFF726B88270826961
:10145000EFE762B1022A01D1012B08D091F8C41242
:1014600081618270002900DC227030BC704791F8E5
:10147000C512F5E770B5864900250968B1F8CA229A
:10148000824205D291F8C022120701D5032512E04D
:10149000B1F8C822824205D291F8C022520701D584
:1014A000022508E0B1F8C622824204D291F8C002B7
:1014B000800700D501257E4E784A774C3078012888
:1014C00001D0E8B117E01078C0B945B1A06918B1F2
:1014D000401EA06106D011E091F8C40200E0002097
:1014E000A0610BE0157091F81001C00606D58021AF
:1014F0000520EEF7D1FF3078012800D1A57070BD2E
:10150000A078107070BD624A00211268B2F8CA3229
:10151000834205D292F8C0321B0701D5032112E0A5
:10152000B2F8C832834205D292F8C0325B0701D5C7
:10153000022108E0B2F8C632834204D292F8C00217
:10154000800700D501215B48544A03785248012B9B
:1015500004D0002B01D10370117070470029FCD01A
:101560000378002BF9D10123F5E7F0B5DFF828C1A6
:10157000DFF82CE100239CF801000EF1080E40F684
:10158000FF713EF8106042480268184692F8064320
:10159000B2F8175304F00F04641C06E03EF8107014
:1015A000B94201DD39460346401C8442F6DC92F81C
:1015B000F107112803D1404846818181C581701A05
:1015C000A84208DD02F20732324832F81320428086
:1015D00001808CF80130F0BD2D4A126892F8C022CB
:1015E000D20607D5421A002A04DCC1EB8111084457
:1015F000C0F38F1070472DE9F04706462448A0B08D
:101600008021056895F8C30200F00F04641C684649
:1016100006F00BFD00236A46297D10E001FB03F76D
:10162000002009E007EB000852F820C036F91880C6
:10163000C44442F820C0401C8142F3DC5B1CA3423E
:10164000ECDB0020914606E059F8203093FBF4F3E0
:1016500049F82030401C8142F6DC134A002318462A
:10166000D2F800A04FE000BF4FF0000C67460BE03F
:1016700007FB010236F9128059F82020B8EB02026C
:1016800000D5524294447F1CA742F1DB16E00000D3
:101690002802100004251000F40310005502100069
:1016A000F00B01204B021000800210009402100089
:1016B000490210005602100000DB01209CFBF4F2EE
:1016C00095F87270FF0705D05FEA4A5717D595F86D
:1016D00076700CE095F81B71FF0710D0E54F3F784E
:1016E000072F0CD15FEA4A5709D595F81F714FEAC9
:1016F000171C0CFB02FC07F00F029CFBF2F29A4253
:1017000000DD1346401C8142AEDCB3F5803F04DBB4
:101710004FF6FF7020B0BDE8F08798B2FAE72DE9E8
:10172000F047D54EDFF854A30024306827460AF16D
:10173000080590F8149090F8C30200F00F0000F133
:10174000010814E007FB08F0CD4900FB09F001EBAC
:101750004000FFF750FF2AF8170035F81710FFF781
:101760003BFF25F81700A04200D904467F1C3068D3
:1017700090F8060300F00F00401CB842E2DCFFF7CF
:10178000F4FE3068BF4F90F80513890602D47978CB
:1017900035F811404FF000514FEA14224A738C7310
:1017A00090F8C112090603D52046FFF7ACFE09E008
:1017B00090F8C0028006204602D5FFF75BFE01E0EC
:1017C000FFF707FE306890F83D03800703D578786F
:1017D00035F8100000E02046FFF78CFD316891F8E5
:1017E000F107112897D1A848112201F20731028090
:1017F0004288521C4280A54A538883801288C28046
:101800007A780281A24A127802822A8842826A8801
:101810008282AA88C282EA880283BAF800304383AF
:10182000BAF802308383BAF80430C383BAF80620CA
:1018300002840A8842844A8882848A88C284C98849
:101840000185448567E72DE9FE4F8B488D4E4FF0AB
:1018500000040168DFF828A281460F7D91F8C312C9
:1018600001F00F05716905F1010591FBF5F205FB2A
:10187000121830E0874904FB07F201EB420B04FB2E
:10188000058202FB07F20AEB4202029290F8C022A4
:1018900012061AD57269002A17DD04FB05F27A4395
:1018A0000AEB420190F8BA21037D5207002AB0F9F1
:1018B000E822CDE90023B0F9E6325A46104602DAB2
:1018C000F2F7A5FC01E0F2F737FC7A0059460298DE
:1018D00006F00AFB641CD9F8000090F8061301F02A
:1018E0000F01491CA142C5DC70694FF0FF31401C5B
:1018F00001EB45017061814200DA75617069A842AF
:1019000002DBBDE8FE4F0AE7BDE8FE8F2DE9F34F8D
:10191000DFF86491DFF880A15A4CD9F8000083B059
:101920000F4690F8C1024FF00006C00778D0217929
:101930002020CDE90001514900251F233A461031EE
:101940000398F5F734FB2079012800D12671002196
:10195000DFF848B14FF0010C4B4640E047481030EB
:1019600030F81120039830F81100A2EB0000434A30
:1019700000B202F1500222F811001A6892F8C282F5
:101980005FEA887806D5DFF8188198F80080B8F10A
:10199000010F08D09BF80080B8F1000F10D0B8F10B
:1019A000010F2CD018E0B2F8EA82804500DA012558
:1019B000B2F8EC22524212B282420FDD01250DE054
:1019C000B2F8DD82804500DA0125B2F8DF2252420A
:1019D00012B2824200DD01258AF80060491CB9423A
:1019E000BCDBE078A84202D09BF80000C8B1A68119
:1019F00022487A001030039906F076FA26E0A68194
:101A0000E670B2F8E182804501DA8AF800C0B2F8E7
:101A1000E322524212B28242E0DD8AF800C0DDE7E2
:101A200013E0A089401C00B2A081D9F80010012D5C
:101A300091F8E51205D001F01F018142D8DCE57074
:101A4000D6E7B0EB511FFADAD2E7E670D9F800001A
:101A500090F8F10711280AD10B4842F20F718185E5
:101A6000E178C1859AF800100186A189418605B008
:101A7000BDE8F08F9402100028021000F00B012046
:101A80000A541000F403100000DB012004251000AC
:101A90005502100064050120590210005602100082
:101AA0005802100031B56846F9F7D7FBFE4C207894
:101AB000022805D19DF80000012801D102F0ABFFFA
:101AC0009DF80000207038BD10B5F9F79FFEBDE805
:101AD000104002F083BE10B5FAF763F8F7F7DEF9AD
:101AE00002F064FEFCF790F9BDE81040FFF7E4BB9C
:101AF000ED4900208860EEE7F8B50024FBF70EFF03
:101B0000EA4D26462B6893F8C91389061DD5E84986
:101B1000E84FDFF8A4C30A7852EA000E0CD197F818
:101B200000E0BEF1010F07D19CF800E0BEF1000F0C
:101B300002D001220A7008E0012A06D128B93A78B9
:101B40001AB99CF8002002B90E70DC490978022904
:101B500004D093F8F1170A2904D005E0002800D03A
:101B60000120F8BDD649C885E8B1CF4901288E804B
:101B700003D0032804D0B0B10FE0FFF793FF0AE0D1
:101B8000D048D24AD24900780090CF480378D14853
:101B9000FCF79BFC08B902F031FE286890F8F107C9
:101BA000182803D004E0FFF78FFF02E0FDF71AF9D1
:101BB00001242046F8BDBD4910B50C6814F82D3F2E
:101BC0006178A2886488A04201D9184610BD90426D
:101BD00001D2084610BD801A5B1A5843A21AB0FB06
:101BE000F2F0084410BD2DE9FC5FB04C834600269E
:101BF00022688A4640F6FF71537D107D5B1C43438B
:101C00009FB2AE4B35461B78042B7DD192F8243021
